:020000040000FA
:100000000002040000000000CE840000CE84000046
:10001000CE840000CE840000CE840000CE84000098
:10002000CE840000CE840000CE840000CE84000088
:10003000CE840000CE840000CE840000CE84000078
:10004000CE840000CE840000CE840000CE84000068
:10005000CE8400004A5A0000705A0000CE8400008E
:10006000CE840000CE840000CE840000CE84000048
:10007000CE840000CE840000CE840000CE84000038
:10008000CE840000CE840000CE840000CE84000028
:10009000CE840000CE840000CE840000CE84000018
:1000A000CE840000CE840000CE840000CE84000008
:1000B000CE840000CE840000CE840000CE840000F8
:1000C000CE840000CE840000CE840000CE840000E8
:1000D000CE840000CE840000CE840000CE840000D8
:1000E000CE840000CE840000CE840000CE840000C8
:1000F000CE840000CE840000CE840000CE840000B8
:10010000CE840000CE840000CE840000CE840000A7
:10011000CE840000CE840000CE840000CE84000097
:10012000CE840000CE840000CE840000CE84000087
:10013000CE840000CE840000CE840000CE84000077
:10014000CE840000CE840000CE840000CE84000067
:10015000CE840000CE840000CE840000CE84000057
:10016000CE840000CE840000CE840000CE84000047
:10017000CE840000CE840000CE840000CE84000037
:10018000CE840000CE840000CE840000CE84000027
:10019000CE840000CE840000CE840000CE84000017
:1001A000CE840000CE840000CE840000CE84000007
:1001B000CE840000CE840000CE840000CE840000F7
:1001C000CE840000CE840000CE840000CE840000E7
:1001D000CE840000CE840000CE840000CE840000D7
:1001E000CE840000CE840000CE840000CE840000C7
:1001F000CE840000CE840000CE840000CE840000B7
:10020000FFFFFF00FFFFFF00CE840000CE84000050
:10021000CE840000CE840000CE840000CE84000096
:10022000CE840000CE840000CE840000CE84000086
:10023000CE840000CE840000CE840000CE84000076
:10024000CE840000CE840000CE840000CE84000066
:10025000CE8400004A5A0000705A0000CE8400008C
:10026000CE840000CE840000CE840000CE84000046
:10027000CE840000CE840000CE840000CE84000036
:10028000CE840000CE840000CE840000CE84000026
:10029000CE840000CE840000CE840000CE84000016
:1002A000CE840000CE840000CE840000CE84000006
:1002B000CE840000CE840000CE840000CE840000F6
:1002C000CE840000CE840000CE840000CE840000E6
:1002D000CE840000CE840000CE840000CE840000D6
:1002E000CE840000CE840000CE840000CE840000C6
:1002F000CE840000CE840000CE840000CE840000B6
:10030000CE840000CE840000CE840000CE840000A5
:10031000CE840000CE840000CE840000CE84000095
:10032000CE840000CE840000CE840000CE84000085
:10033000CE840000CE840000CE840000CE84000075
:10034000CE840000CE840000CE840000CE84000065
:10035000CE840000CE840000CE840000CE84000055
:10036000CE840000CE840000CE840000CE84000045
:10037000CE840000CE840000CE840000CE84000035
:10038000CE840000CE840000CE840000CE84000025
:10039000CE840000CE840000CE840000CE84000015
:1003A000CE840000CE840000CE840000CE84000005
:1003B000CE840000CE840000CE840000CE840000F5
:1003C000CE840000CE840000CE840000CE840000E5
:1003D000CE840000CE840000CE840000CE840000D5
:1003E000CE840000CE840000CE840000CE840000C5
:1003F000CE840000CE840000CE840000CE840000B5
:100400006F032200007F220000018800000000002E
:100410000C000700E0E827000100200011000700A1
:10042000000020000000E000020032000000020096
:100430000000000016840200000000000040DA0006
:100440000000FE004440A900201F20000000E00042
:100450000300320000002000A00188004440A800F2
:100460000000060091018800800078000000EB0089
:1004700015003700E280400032A0B4009101BA00BC
:10048000E280400032A0B4009102BA00E280400055
:1004900032A0B4000002EB00472BDE00F507B200EB
:1004A000602CE10004003A000059EB008301E900F0
:1004B000FDFF3E00040037006128E100010032002A
:1004C0000082EB00040007001101BA000200E00006
:1004D000E8FF3A00000006003159BA008301E90044
:1004E0000C0032002159BA008301E90008003200F3
:1004F0000400E00003003A00E280400032A0B400B3
:10050000F5FF370011D9BA008301E900FAFF3A007C
:100510008100E800E180400032A0B4000000060045
:1005200000000000000000000000000000000000CB
:1005300000000000000000000000000000000000BB
:1005400000000000000000000000000000000000AB
:10055000000000000000000000000000000000009B
:10056000000000000000000000000000000000008B
:10057000000000000000000000000000000000007B
:10058000000000000000000000000000000000006B
:10059000000000000000000000000000000000005B
:1005A000000000000000000000000000000000004B
:1005B000000000000000000000000000000000003B
:1005C000000000000000000000000000000000002B
:1005D000000000000000000000000000000000001B
:1005E000000000000000000000000000000000000B
:1005F00000000000000000000000000000000000FB
:1006000000000000000000000000000000000000EA
:1006100000000000000000000000000000000000DA
:1006200000000000000000000000000000000000CA
:1006300000000000000000000000000000000000BA
:1006400000000000000000000000000000000000AA
:10065000000000000000000000000000000000009A
:10066000000000000000000000000000000000008A
:10067000000000000000000000000000000000007A
:10068000000000000000000000000000000000006A
:10069000000000000000000000000000000000005A
:1006A000000000000000000000000000000000004A
:1006B000000000000000000000000000000000003A
:1006C0000000000000000000889FBE008A9FBE005E
:1006D000010578000100E0000400350008003C003E
:1006E0000000E0002000320005003700600010002C
:1006F000E080180002003B0001F02C001A003700D7
:100700000004BE006011B8006B0920000982CF0010
:10071000020039000882CF000441B0006942520053
:100720000E00320008003B0082817100610164000C
:100730008904D1000884D3008B05E8000442E80056
:10074000F9FF3A00050037000804440089844C0092
:100750008B05E9000442E900FBFF3A002C01070089
:100760000AF0A70001F0A0004F05BE004F04BE0034
:1007700000000600F4FF2F004B013700140020009A
:1007800049013700889FBE008A9FBE008C1F7800F9
:10079000600107006701330003866C006450E100CC
:1007A0002E0032006420E100330032006150E1008D
:1007B0002F0032006120E1003100320085855500B4
:1007C000EB07B000090020000804200005003700F6
:1007D0000804440089844C000A00310006034300E9
:1007E00087834B000001530081815B00F8FF3300D9
:1007F0000203BE000800A0000804440089844C00E5
:10080000F6FF3900C639DD008301730001003200B4
:10081000130020008904D1000884D3000998A300A4
:10082000050032000800A7000300A0008904D100E1
:100830000884D3008B05E8008904D1000884D30024
:100840000001EB000281D200F100070001F0A100DD
:100850000CF0A70001F0A0003F0137006420E10088
:10086000410132000801BE000200BE00F7FF370060
:100870006120E1003C0132006000B800F3FF370066
:100880000000200001F82700F0FF370003F0A2006D
:10089000889FBE008A9FBE008C1F78001D01070044
:1008A000240133006450E1004F0032006420E10075
:1008B0005200320003826C0007003B000905D000A3
:1008C0000306D000820F54000C065D0002003900C0
:1008D0000200320089017800030678008582550005
:1008E00004003D000003FD008103FD008502EA00D5
:1008F0008B854200840F720002003B0060001000F4
:10090000E08018006011B8000005EB007A28E100D3
:100910000A00390006007800C75DDD00F707B20065
:10092000878075002D003700828171000A017800F0
:10093000610560008180D1000080D3008502E9005C
:10094000F9FF3B00060440008784480002003B009A
:1009500060041400E0841C000988A3000700320032
:100960008A81710082817100610164008904D10073
:100970000884D3008B05E800170037000978A3002E
:1009800013003A000B00E000130034008B05E9006F
:100990000804440089844C000A4474000978A300C8
:1009A0000D003A000B00E000070034008B05E90061
:1009B0000804440089844C0001003A000B00200028
:1009C0000978A300F7FF32000001EB0002003700B6
:1009D000828171000A0178008D0007000CF0A700E9
:1009E00001F0A000DC0037006420E10002003A00C2
:1009F000838F6C00DC0033000801BE000200BE00E3
:100A0000D5003700889FBE008A9FBE008C1F7800EB
:100A1000C0000700C700330003866C006450E1008B
:100A2000240032006420E100270032006150E10020
:100A3000220032006120E100210032008B8542005B
:100A4000EB07B1000134B800003AB80008044200D6
:100A500089844A00013AB8000030B800888040001C
:100A600009014A0004003300000040008180480072
:100A7000020149008B05E900C909DD00830170000E
:100A80000100320013002000C814DE004814DD000D
:100A90004709DE001200B200C808DE0008847000BA
:100AA0005B00070001F0A1000CF0A70001F0A0001E
:100AB000A90037006120E100AB0032000801BE0050
:100AC0000200BE00F7FF37006150E100FCFF3A0072
:100AD000A50037000001BE00A60007000470A700B3
:100AE00003F0A10003F8A30013003A006509B10068
:100AF00010003200090035006928E10002003500CD
:100B0000010028000000050000004000818048002E
:100B10008502E900FCFF3A0000000600F88F420061
:100B2000050035008100D1000080D3008502E80077
:100B3000FCFF3A00000006008000EB00000005000A
:100B40006022B800060220000000D0008180D200A0
:100B50000482D2008582D2000000A000020252006E
:100B600083825A00030031000202420083824A005D
:100B70000000A1000603E900F3FF3A0000000600B0
:100B8000EFFF07000400BE00000006000001BE00E9
:100B9000780007000470A70003F0A1006509B10008
:100BA000160032000D0035006828E100060035000F
:100BB000F0FF2F00F1FF27000300E00013003B00CF
:100BC000010028000000050000004000818048006E
:100BD0008502E900FCFF3A0008003700F88F420068
:100BE00002003C008000EB00000005008100D10005
:100BF0000080D3008502E800FCFF3A000300E0001B
:100C000002003B0060001000E080180000000600B9
:100C100081002000618055000B003D000B0020008A
:100C200061FE2F000100E1001D003400828171008F
:100C3000610164008904D1000884D3000000E80049
:100C4000FAFF3A00710020006100640003007000A8
:100C5000020060000900320061044400E0844C009E
:100C60000988A500050032008B05E8006808E1004E
:100C700002003A008904D1000884D300F20F20005A
:100C80000258E10005003D00C75DDD00F907B20034
:100C90008980750008007800000006000BF8270026
:100CA0008B00780000000500889FBE008A9FBE0070
:100CB000841F7800170007004F00780011003300F0
:100CC000F0FF2F00838F6C0006003B0004056500D9
:100CD0000A00A7000800370009F0A6001000200055
:100CE00008003700820F5400838F5C000300390036
:100CF0001000200001003E000000200009F0A700C5
:100D00000000EA004F05BE004F04BE000000E000F6
:100D1000000006000004BE00160007000003BE002D
:100D20000405BE000200BE0012000700844F7500DB
:100D3000000006000200BE006450E100050036001D
:100D40006420E100020036000968A30001003A00B7
:100D50000800BE000160A0004F0678004F05BE00ED
:100D60004F04BE0000000600F0FF2F00F1FF270037
:100D7000F9FF3700C70ADE00F107B200F50FB20035
:100D800008003200E1CF4200020032000170A000F2
:100D900024000500810F70000100320004080500E6
:100DA00044000500810F700002003A0014000500A5
:100DB0008502E9000000400081C04800FCFF3B00C4
:100DC0000170A000240005004C4500005400000004
:100DD0004946000000540000484500004E00000055
:100DE000454C000053450000004700004F540000F0
:100DF0004F000000474F0000535500004200000024
:100E00005245000054550000524E000000520000B0
:100E1000454D000000500000524900004E540000B3
:100E2000004900004E5000005554000000460000EC
:100E30004F520000005400004F0000004E450000DB
:100E400058540000005200004541000044000000DA
:100E50004441000054410000005300005441000090
:100E60005254000052000000535400004152000050
:100E700054000000535400004F5000005200000086
:100E8000535400004F50000000530000454E000036
:100E90004400000052450000434500004956000050
:100EA00045000000434C00004B000000444100009E
:100EB0005400000042490000545200004541000027
:100EC0004400000041440000430000004155000080
:100ED00058500000494E00000050000053550000DB
:100EE00000500000554C00004C5500005000000020
:100EF000444500004C4100005900000041550000ED
:100F00005800000046520000455100000044000017
:100F100055540000590000004D41000043520000AC
:100F20004F000000454E0000440000000052000049
:100F3000554E0000004C00004953000054000000D2
:100F4000455800004954000000440000454200009C
:100F500055470000004E000045570000000000000B
:100F60003E2000000008000020080000001B0000D8
:100F70005B440000001B00005B0000004400000018
:100F80001B5B0000430000001B5B0000324B0000B5
:100F90000D00000043000000001B00005B32000059
:100FA00044000000203D00002000000056520000D8
:100FB00045470000207400006F6F0000206C0000A7
:100FC0006F7700002C20000069730000207400007F
:100FD0006865000072650000206100002073000059
:100FE000686F0000727400003F0000002E200000B7
:100FF0003C0000003E0000002E200000000D00001C
:101000000A280000002900003E20000000420000E5
:1010100075730000205000006972000061740000C8
:101020006520000076310000610000004669000084
:10103000726D00007761000072650000207600008C
:10104000352E0000392D0000657800007472000014
:101050006173000020280000723500003339000061
:101060002920000000200000283200003446000043
:101070004A360000344700004130000030320000A2
:101080002000000041330000004200003400000056
:10109000423500000042000038000000554E0000BC
:1010A0004B0000002900000049090000004F00002B
:1010B0000900000048090000004C00000900000081
:1010C000456E00007465000072200000726100002F
:1010D00077200000766100006C750000652000003C
:1010E000666F0000722000004252000047000000BE
:1010F0003062000000300000303000002C000000A2
:101100003030000000300000313200003334000085
:1011100035360000373800003941000042430000F6
:10112000444500004630000078000000002900001F
:10113000002000005700000020520000004900007D
:1011400032430000310000000808000008080000D9
:101150000800000000000000204800007A000000A5
:101160000000000042420000494F00003100000032
:1011700052410000573100000000000031410000E2
:101180004C530000000000004F43000044310000B9
:101190000000000000000000000000002900000026
:1011A0000000000000000000000000002800FA001D
:1011B0000000EB00600F98000000EB0080578800F3
:1011C0000000EB00705788007057800020079800DF
:1011D0000000EB00100798000000EB00000F780003
:1011E0000000EB00A04088000000EB009057880052
:1011F0000000EB00400798000000EB00000F980093
:10120000140037000000EB00600798000B00370067
:101210000E089000EE0090004500DD0081004000C7
:1012200040AF2000808040000040EB008048780004
:101230006E0090000000E800600798006E009000CB
:10124000FF0F5000F2FF34000E0890000000E8008D
:10125000000F98000E089000E40F5000E9FF3400E2
:101260000000EB00A05C8800A1408000E0022000AC
:101270000088B900610220008080400000832000C7
:10128000008040009655020000000000D140800020
:1012900000202000008060000000E0000400320018
:1012A00071002000C05920002880020000000000CA
:1012B000007B280096550200000000003204370031
:1012C000A05C80000000E00063003200A05C8000B1
:1012D0000000E900A05C88000000EB0060079800B7
:1012E0001E00370072578000A05C8000EE00900066
:1012F0004500DD008100400040AF2000008040003C
:1013000090407800E09E20000000410001487800F5
:10131000A05C8000EE0090004500DD0081004000F0
:1013200040AF20000080400010407800F2590200D9
:1013300000000000705780000000E800705788002F
:101340006E0090000000E800600798007157800070
:10135000F00F20000080600070578800A05C8000C3
:10136000EE0090004500DD008100400040AF20000D
:1013700000804000104078000004E000D9FF3A00EF
:101380000000EB00A05C880033003700A09C200028
:1013900010407800644060000004E0002E0032003D
:1013A000A1408000E00220000088B900FA0040005F
:1013B0000083200000804000100078000000010041
:1013C0000000E00024003200A1408000E002200084
:1013D0000088B90061022000808040000083200066
:1013E000008040009655020000000000007B2800AD
:1013F0009655020000000000815780007057800061
:10140000808F5000140032008057800060079800E1
:101410000D003700EE009000E09E200000804000AC
:1014200010407800F259020000000000EE00900029
:10143000F00F200000806000600798006E009000B0
:101440000000E80060079800EE00900070578000F0
:10145000808F5000EFFF3A00D459020000000000D6
:101460000004E000C9FF320022C2BF0062406000F9
:101470000004E0000500320010118000D1FF2F00B1
:101480000100600010118800BF033700E05902001E
:1014900000000000604F98006E4890000080FB0044
:1014A0006101B9000217980013179800F007200097
:1014B000010020000E1190009E119000800F51003D
:1014C000818F59003C033E000E1090009E1090004A
:1014D000006001002D033700E20237003E013700B3
:1014E00035033700D8003700F902370053013700C1
:1014F00031033700770037002F0337000F03370021
:101500002D0337002C0337000C033700FE01370092
:10151000290337005A013700270337002603370015
:101520002503370024033700230337002203370045
:1015300021033700200337001F0337001E03370045
:10154000020137001C0337001B0337001A03370062
:101550001903370018033700170337001603370045
:101560001503370014033700130337001203370045
:1015700011033700100337000F0337000E03370045
:101580000D0337000C0337000B0337000A03370045
:101590000903370008033700070337000603370045
:1015A0000503370004033700030337000203370045
:1015B0000103370000033700FF023700FE02370047
:1015C000FD023700FC023700FB023700FA02370049
:1015D000F9023700F8023700F7023700F602370049
:1015E000F5023700F4023700F3023700F202370049
:1015F000F1023700F0023700EF023700EE02370049
:10160000ED023700EC023700EB023700EA02370048
:10161000E9023700E8023700E7023700E602370048
:10162000E5023700E4023700E3023700E202370048
:10163000E1023700E0023700DF023700DE02370048
:10164000DD023700DC023700DB023700DA02370048
:10165000D9023700D8023700D7023700D602370048
:10166000D5023700D4023700D3023700D202370048
:10167000D1023700D0023700CF023700CE02370048
:10168000CD023700CC023700CB023700CA02370048
:10169000C9023700C8023700C7023700C602370048
:1016A000C5023700C4023700C3023700C202370048
:1016B000C1023700C0023700BF023700BE02370048
:1016C000BD023700BC023700BB023700BA02370048
:1016D0005D003700815780002E009000810F500080
:1016E00055003200715780002E009000810F50008D
:1016F00010003A00705780008000E900F00F2000D1
:10170000008060007057880071578000E09E2000C4
:10171000808040000040EB008048780071578000D6
:1017200021079800307B2800965502000000000039
:10173000150337000000EB00000F98002E0090000A
:101740008000E900F00F2000008060002007980072
:10175000707B280096550200000000002E019000CA
:1017600062079800210037006E0190006E00900023
:101770008000E800E09E200000804000904078005B
:10178000E09E20000000410001487800EE0090003B
:10179000E09E200000804000104078000004E0003F
:1017A00007003200EE009000E09E20000080400024
:1017B00010407800F25902000000000003003700DA
:1017C00000C2B300F2590200000000000E089000B1
:1017D0000000E800000F98006E0090008000E80014
:1017E000F00F20000080600060079800EE0090007D
:1017F00070578000808F5000DBFF3A0070578000E8
:101800008000E900F00F2000008060007057880021
:10181000B07B280096550200000000000E089000E2
:101820002E58020000000000E07B280096550200C0
:1018300000000000D402370070C0B300F25902006B
:1018400000000000D0023700715780002E00900089
:10185000810F5000390032000000EB00000F9800AB
:10186000AE01900063079800210037006E019000E0
:101870006E0090008000E800E09E200000804000A4
:1018800090407800E09E2000000041000148780070
:10189000EE009000E09E20000080400010407800A4
:1018A0000004E00007003200EE009000E09E2000FF
:1018B0000080400010407800F25902000000000053
:1018C0000300370000C2B300F2590200000000001C
:1018D0000E0890000000E800000F98006E009000D5
:1018E0008000E800F00F2000008060006007980092
:1018F000EE00900070578000808F5000DBFF3A00B0
:10190000705780008000E900F00F20000080600028
:1019100070578800B07B2800965502000000000038
:101920000E0890002E58020000000000E07B280006
:1019300096550200000000009302370070C0B3000B
:10194000F2590200000000008F023700E059020047
:1019500000000000604F9800EE489000B0C5B30052
:1019600080CF500088023A00E059020000000000D9
:10197000604F98006E4890000080FB00700F980048
:1019800020042000FE089000808F5000DE0032000E
:10199000200420007E099000800F510005003C00CB
:1019A00010042000FE099000808F510034003200A6
:1019B0007502370030042000FE089000808F500030
:1019C0001E003200400420007E099000800F51006C
:1019D000010032006C0237004E009000E40F50000E
:1019E0000500340028730200000000000000EB0036
:1019F0004007980064023700815780002E00900055
:101A0000810F5000090032002E0090008000E90094
:101A1000F00F20000080600020079800707B2800F5
:101A200096550200000000005702370070C0B30056
:101A3000F259020000000000530237007157800085
:101A40002E009000810F5000090032002E009000FF
:101A50008000E800F00F2000008060002007980060
:101A6000007C280096550200000000004602370066
:101A700070C0B300F25902000000000042023700BB
:101A80000000EB00000F7800805780000000E900A4
:101A900080007800F00F2000008060006007980050
:101AA0008D003700EE009000E09E20000080400096
:101AB000104078000004E00082003A006E009000C0
:101AC0008000E900F00F200080806000E09E200090
:101AD00000804000104078000004E00079003200EF
:101AE0001E0FE8001E0090009E0F100075003600CB
:101AF0001E0090000000E800100798008157800049
:101B000070578000808F5000140032000A003700A8
:101B100071578000E09E2000808040000040EB0074
:101B200080487800705780008000E900F00F2000A6
:101B300000806000705788007157800080578000D7
:101B4000808F5000F2FF3A0071578000E09E200025
:101B5000808040000040EB00804878006E009000DC
:101B60008000E900F00F200000806000000F980066
:101B7000110037008E089000E09E20000080400099
:101B8000104078000004E00006003A000E089000C3
:101B90008000E800F00F20000080600050079800EF
:101BA000090037000E0890008000E900F00F2000C7
:101BB00000806000000F98008E0890007057800031
:101BC000808F5000EBFF3A00407C280096550200C1
:101BD00000000000A1408000E00220000088B90061
:101BE00061022000808040000083200000804000CF
:101BF0009655020000000000D14080000020200027
:101C0000008060000000E00004003200710020004D
:101C1000C05920002880020000000000007B28003E
:101C20009655020000000000DE019000030F9800AE
:101C3000180037008E089000E09E200000804000D1
:101C400010407800F2590200000000007257800036
:101C50008E089000E09E20000080400090407800B8
:101C6000E09E20000000410001487800705780008D
:101C70008000E800F00F20000080600070578800AE
:101C80000E0890008000E800F00F20000080600047
:101C9000000F98008E0890006E009000808F50001A
:101CA000E4FF3A0071578000E09E200080804000F1
:101CB0000040EB00804878007057800020079800B3
:101CC000090037006E0090008000E900F00F20004E
:101CD0000080600060079800EE0090007057800060
:101CE000808F50006FFF3A00EE0090007057800028
:101CF000808F5000A4013A0070C0B300F259020076
:101D000000000000A00137000000EB00000F780089
:101D1000805780000000E90080007800F00F20006C
:101D200000806000600798008E003700EE00900091
:101D3000E09E200000804000104078000004E00099
:101D400083003A006E0090008000E900F00F200050
:101D500080806000E09E20000080400010407800FD
:101D60000004E0007A0032001E0FE8001E00900020
:101D70000000E9009E0F500075003A001E00900020
:101D80000000E9001007980081578000705780001C
:101D9000808F5000140032000A0037007157800015
:101DA000E09E2000808040000040EB0080487800EA
:101DB000705780008000E900F00F20000080600074
:101DC000705788007157800080578000808F5000C6
:101DD000F2FF3A0071578000E09E200080804000B2
:101DE0000040EB00804878006E0090008000E90021
:101DF000F00F200000806000000F980011003700F5
:101E00008E089000E09E2000008040001040780086
:101E10000004E00006003A000E0890008000E80090
:101E2000F00F200000806000500798000900370084
:101E30000E0890008000E900F00F20000080600094
:101E4000000F98008E08900070578000808F50001F
:101E5000EBFF3A00407C280096550200000000008D
:101E6000A1408000E00220000088B900610220004B
:101E700080804000008320000080400096550200D2
:101E800000000000D14080000020200000806000A1
:101E90000000E0000400320071002000C059200062
:101EA0002880020000000000007B280096550200F8
:101EB00000000000DE009000010F980018003700BD
:101EC0008E089000E09E20000080400010407800C6
:101ED000F259020000000000725780008E08900046
:101EE000E09E20000080400090407800E09E2000AE
:101EF0000000410001487800705780008000E80031
:101F0000F00F200000806000705788000E089000DD
:101F10008000E800F00F200000806000000F9800B3
:101F20008E0890006E009000808F5000E4FF3A0011
:101F300071578000E09E2000808040000040EB0050
:101F40008048780072578000220798000900370007
:101F50006E0090008000E900F00F2000008060001B
:101F600060079800EE00900070578000808F50004E
:101F70006EFF3A00EE00900070578000808F500096
:101F800001013A001E009000E10F500031003A00BC
:101F9000407C28009655020000000000A14080000F
:101FA000E00220000088B90061022000808040002B
:101FB00000832000008040009655020000000000D1
:101FC000D140800000202000008060000000E00080
:101FD0000400320071002000C05920002880020057
:101FE00000000000007B2800965502000000000061
:101FF0000A00370071578000E09E2000808040007A
:102000000040EB0080487800705780008000E900B5
:10201000F00F20000080600070578800715780002A
:1020200080578000808F5000F2FF3A007157800087
:10203000E09E2000808040000040EB008048780057
:1020400073578000230798000000EB0010079800EA
:10205000CD00370070C0B300F2590200000000004C
:10206000C9003700815780002E009000810F50007A
:1020700013003200815780002E00900001005000B4
:1020800080007800F00F200000806000000F9800B2
:10209000B07B280096550200000000000E0890005A
:1020A0002E58020000000000E07B28009655020038
:1020B000000000008057800020079800B200370021
:1020C00070C0B300F259020000000000AE003700FB
:1020D000715780002E009000810F500013003200D5
:1020E000715780002E009000008050008000780022
:1020F000F00F200000806000000F9800B07B2800E7
:1021000096550200000000000E0890002E580200B4
:1021100000000000A07C280096550200000000008E
:1021200071578000210798009700370070C0B300F6
:10213000F259020000000000930037001000200058
:10214000600F98000000EB001007980071578000A6
:10215000E09E2000808040000040EB008048780036
:10216000705780008000E800F00F200000806000C1
:10217000705788007257800022079800C07C2800A2
:10218000C2550200000000007F0037004E009000A2
:102190000000E800400798004E009000F40F500047
:1021A00079003A0052600200000000000000EB00DD
:1021B0004007980074003700705780008000E800E6
:1021C000F00F20008080600080578000808F5000DA
:1021D0006A0032006E489000FF4F500067003600E2
:1021E000EE489000E0C7B30080CF500063003E008F
:1021F000715780002E009000808F500015003A002B
:102200006E489000F25902000000000071578000F3
:102210006E499000E09E2000008040000248780057
:10222000705780008000E800F00F20000080600000
:102230007057880071578000E09E20008080400029
:102240000040EB0080487800735780002307980017
:102250004D003700715780002E0090000080500024
:1022600080007800F00F200000806000000F9800D0
:10227000B07B280096550200000000000E08900078
:102280002E58020000000000A07C28009655020095
:102290000000000070578000600798001D003700A4
:1022A0006E0090000001E800EE009000E09E20002B
:1022B0000080400090407800E09E20000000410037
:1022C00001487800EE009000E09E20000080400071
:1022D000104078000004E00009003200EE00900099
:1022E000E09E20000080400010407800F25902007B
:1022F00000000000D07C280096550200000000007D
:102300006E0090008000E900F00F20000080600067
:10231000600798006E0190002E0090008000E90098
:10232000F00F200000806000800F5100DCFF3A00B9
:102330006E489000F259020000000000AE009000CC
:102340006E499000E09E2000008040000248780026
:102350002E0090008000E800F00F20000080600058
:1023600020079800705780008000E800F00F2000E0
:1023700000806000705788000300370070C0B30011
:10238000F2590200000000006E0890000000E0001A
:10239000CBFB320070578000400F980080578000C0
:1023A000300F98000000EB00600F98000000EB0079
:1023B000500F98000000EB0090578800D14080003B
:1023C00000202000008060000000E000D004320007
:1023D000863402000000000051002000305A200026
:1023E000B28002000000000010002000500F980092
:1023F000C704370081578000E09E20000080400025
:1024000010407800604F98006E4890000080FB00FC
:102410006101B9002217980033179800D0072000F7
:10242000010020002E119000BE119000800F51007D
:10243000818F59008A043E002E109000BE1090003B
:1024400000600100880437008504370084043700E9
:10245000830437008204370081043700800437008A
:102460007F0437007E0437007D0437007E04370088
:102470007B0437007A0437007B0437007804370088
:10248000770437007604370075043700740437008A
:10249000730437007204370071043700700437008A
:1024A0006F0437006E0437006D0437006C0437008A
:1024B0006B0437006A04370069043700680437008A
:1024C0006704370068043700450437008502370089
:1024D000E4003700ED0037009C0137008A01370027
:1024E0005F0437005E0237005D0437005C0437008C
:1024F0005D0437005C043700F10337000A0437003D
:10250000D5033700FE023700FD023700FC0237001A
:10251000FB023700FA023700F9023700F8023700F1
:10252000F7023700F6023700F50237004C04370097
:102530004B043700A50137008F00370048043700EF
:102540003E003700FF003700F10037004404370039
:102550006400370069013700410437004004370048
:102560003F0437003E0437003D0437003C04370089
:102570003B04370066003700390437003804370061
:102580003704370036043700350437003404370089
:10259000830137003204370031043700300437003C
:1025A000FE0037002E0437002D0437002C043700BE
:1025B000AF023700B5033700BF023700E903370029
:1025C000CC03370026043700C4003700260037004C
:1025D000390037003B01370021043700280037005D
:1025E0002A0037001E043700170037001C0437008C
:1025F0001B04370053003700190037001804370058
:102600001B00370016043700150437003803370065
:102610005F0137001204370011043700160037003D
:10262000140137000E0437000D0437000C04370086
:10263000980237006B003700A8023700C8800200FC
:10264000000000000804370077070700A040800062
:102650000000E00004043200F00707000204370025
:102660002C0607000004370014090700FE0337009A
:10267000EE080700FC03370062080700FA03370082
:10268000AA5D020000000000F7033700A0408000B0
:102690000000E00005003A00D1012000305D20007C
:1026A000B280020000000000EF033700125C02005D
:1026B00000000000EC033700A09C200010407800D0
:1026C0000000A1000010A100A19C2000804878001B
:1026D00061012000805A2000B2800200000000004A
:1026E000E1033700A09C2000104078000000A0000B
:1026F0000010A100A19C200080487800510120001A
:10270000E05B2000B280020000000000D60337002A
:10271000A09C2000104078000030A000A19C200068
:1027200080487800C1012000B07E2000288002008F
:1027300000000000C07C2800C2550200000000001C
:10274000C9033700A09C2000104078000030A10091
:10275000A19C200080487800B1012000007D20006D
:102760002880020000000000C07C2800C255020042
:1027700000000000BC033700805780008000E800A4
:10278000F00F20000080600080578800D10507000E
:10279000E9030700600798006E009000905802005F
:1027A00000000000207D2800965502000000000077
:1027B0006E0090002E58020000000000207D2800CE
:1027C00096550200000000006E009000F6550200D1
:1027D00000000000C07C2800C2550200000000007C
:1027E000A1033700805780008000E800F00F200030
:1027F0000080600080578800B6050700CE03070000
:10280000600798006E0090000080FB00467E02008A
:1028100000000000600798006E00900090580200D1
:1028200000000000207D28009655020000000000F6
:102830006E0090002E58020000000000207D28004D
:1028400096550200000000006E009000F655020050
:1028500000000000C07C2800C255020000000000FB
:10286000810337005100200030632000B280020055
:102870000000000023C2BF00614060000004E000CF
:10288000FCFF32000000FE00770337005881020091
:10289000000000000000E00073033200A1002000EF
:1028A00080632000B280020000000000400620008B
:1028B000E47D020000000000367C02000000000001
:1028C00023C2BF00614060000004E000FCFF320052
:1028D00081BF2A0001400100630337003B05070068
:1028E0000000E800000F980002003700E85E0200D8
:1028F000000000000E0890000000E900000F9800A2
:102900000E0890000000E000F8FF3A005603370080
:102910002E0507000000E800000F980002003700B5
:10292000C65E0200000000000E0890000000E900F2
:10293000000F98000E0890000000E000F8FF3A0039
:1029400049033700210507000000E800000F980048
:102950000B00370061012000206420002880020065
:10296000000000000A5F0200000000008055020025
:1029700000000000C07C2800C255020000000000DA
:102980000E0890000000E900000F98000E0890006B
:102990000000E000EFFF3A0033033700A040800062
:1029A0000000E00005003A00D1012000305D200069
:1029B000B2800200000000002B033700C082A90093
:1029C000C282A800C8A2A900CAA2A80021E3A80048
:1029D00020002000E47D020000000000A0C0B30041
:1029E000867C02000000000080007800001B2000B0
:1029F000808F50000F00360090C0B300867C02002C
:102A00000000000080007800702B2000808F5000B4
:102A10000800360011012000806520002880020097
:102A200000000000C07C2800C25502000000000029
:102A30000E003700C082A900C282A900C8A2A90066
:102A4000CAA2A900607D2800C25502000000000053
:102A50002101200090662000288002000000000074
:102A6000C07C2800C25502000000000021E3A9003C
:102A7000FD023700A04080000000E00005003A00A1
:102A8000D1012000305D2000B28002000000000073
:102A9000F5023700C082A900C282A900C8A2A9001D
:102AA000CAA2A9002101200090662000288002000F
:102AB00000000000C07C2800C25502000000000099
:102AC000E9023700F1002000A03920002880020030
:102AD00000000000A07C02000000000011002000A7
:102AE000903A20002880020000000000C07C2800EE
:102AF000C255020000000000DB023700B27C020079
:102B000000000000D8023700B0040700000F980052
:102B10006100200070682000288002000000000092
:102B20000E089000D0570200000000002100200095
:102B3000D0682000B2800200000000000E08900063
:102B4000107E020000000000C70237009F0407004B
:102B5000000F9800610020007068200028800200AB
:102B6000000000000E089000D05702000000000096
:102B70002100200090EC2000B28002000000000044
:102B80000E089000E47D020000000000B60237004D
:102B9000D04080000090A000D0408800B2023700F2
:102BA000A04080000000E00005003A00D1012000B4
:102BB000305D2000B280020000000000AA02370051
:102BC0003E5F020000000000A70237001000200056
:102BD0009057880010002000600798001000370010
:102BE000815780006E00900080804000F00F200030
:102BF00080806000E09E20000080400090407800CF
:102C0000E0C3B30080CF500002003A000000EB00A8
:102C1000905788006E0090000000E8006007980060
:102C2000815780006E00900080804000F00F2000EF
:102C300080806000E09E200000804000104078000E
:102C40000004E000E6FF3A00EE00900020022000C1
:102C5000808F500002003400100020009057880040
:102C6000905780000000E0007F023A00805780000B
:102C70008000E800F00F200000806000805788008E
:102C8000AD0207006007980081578000F00F200018
:102C900080806000E09E200000804000904078002E
:102CA000D0C3B30080CF500040003A006E009000C7
:102CB0000000E0003A0034006E009000E50F500084
:102CC00037003C00805780008000E800F00F2000B3
:102CD00000806000805788006E0090000000E900CE
:102CE000600798000000EB00000F98000B00370011
:102CF0006E0090008E0890004500DD0081004000CD
:102D000040AF2000808040000040EB008048780009
:102D10000E0890000000E800000F98000E089000D8
:102D2000FF0F5000F2FF34000000EB00000F98008E
:102D300013003700EE0190000E0A900081578000CA
:102D4000E09E200000804000104178004518DD0022
:102D50008400400040AF200000804000024878001E
:102D60000E0890000000E800000F980080578000D7
:102D70008000E800F00F200000806000805788008D
:102D800081578000E09E2000008040009040780045
:102D9000E0C3B30080CF5000E6FF3A0032023700B4
:102DA00010002000905788002F0237006E0090001E
:102DB0000000E0001B003A000000EB00000F98004C
:102DC000140037000E0890000040E8002E58020062
:102DD00000000000607F28009655020000000000FF
:102DE0000E0890004500DD008000780040AF200014
:102DF000008040009655020000000000A07F2800DF
:102E0000C2550200000000000E0890000000E8001B
:102E1000000F98000E089000E40F5000E9FF340006
:102E2000110237006E0090000000E000090034003D
:102E30006E009000E50F500006003C00C07C2800AA
:102E4000C255020000000000EE009000A15C880066
:102E5000050237001000200090578800020237005A
:102E6000805780008000E800F00F200000806000A4
:102E70008057880030020700200F980015040700D3
:102E800081578000F00F200080806000E09E2000CD
:102E9000008040009040780090C2B30080CF500086
:102EA0000D003A00A1408000E00220000088B90037
:102EB000FC0040000083200000804000900078006B
:102EC0002E08900001000100C07C2800C2550200BD
:102ED00000000000E4013700100020009057880037
:102EE000E1013700100020009057880010002000FA
:102EF0006007980010003700815780006E00900036
:102F000080804000F00F200080806000E09E200064
:102F1000008040009040780020C2B30080CF500075
:102F200002003A000000EB00905788006E0090000D
:102F30000000E80060079800815780006E00900054
:102F400080804000F00F200080806000E09E200024
:102F500000804000104078000004E000E6FF3A00E6
:102F6000905780000000E000BF013A00710020008F
:102F7000F0682000288002000000000020C2B3009A
:102F8000F259020000000000220037008157800043
:102F9000F00F20000080600080578800815780007B
:102FA000E09E20000080400010407800F2590200AE
:102FB0000000000081578000E09E2000008040005B
:102FC000104078000000FB00200F9800A09C20001B
:102FD00010407800684060000004E0000400320007
:102FE0002E089000467E020000000000200F98008E
:102FF000A1408000E00220000088B900E800400005
:103000000083200000804000900078002E0890008F
:1030100001000100805780000000E8008057880010
:1030200081578000F00F200080806000E09E20002B
:10303000008040009040780020C2B30080CF500054
:10304000D2FF3A0080578000F10F2000010060009D
:103050008057880020C2B300F2590200000000002F
:10306000C07C2800C2550200000000007E0137002D
:10307000A1408000E00220000088B90080007800B4
:103080000083200000804000100078000000010054
:1030900075013700A1408000E00220000088B900DF
:1030A0008080E8000083200000804000100078004D
:1030B000000001006C013700A1408000E002200008
:1030C0000088B900E4004000008320000080400038
:1030D000100078000000010063013700A14080006B
:1030E000E00220000088B900E600400000832000D4
:1030F0000080400010007800000001005A013700F5
:1031000071002000F068200028800200000000000C
:1031100089010700200F9800805780000000E90017
:103120008057880081578000F00F200000806000E9
:1031300080578800250307000000E800000F980072
:1031400045030700300798003E0090000000E000B3
:103150005D0032003E00900080407800909B20008F
:10316000014878003E009000E80F5000060034004F
:10317000A09C2000104078000050A000A19C2000DE
:103180008048780050003700A09C20001040780054
:103190000050A100A19C2000804878004A00370020
:1031A0002E0890003E7D020000000000A09C200040
:1031B000104078000042B2000004E00004003A0031
:1031C000909B200010407800E84F500009003A0022
:1031D000A09C2000104078000042B2000004E000F3
:1031E0000B003200909B200010407800F04F500000
:1031F00007003200B0C3B300F25902000000000023
:10320000909B2000104078002E5802000000000023
:10321000A09C200010407800684060000004E0009E
:10322000040032002E089000467E020000000000DC
:10323000200F9800A1408000E00220000088B90023
:10324000E8004000008320000080400090007800EB
:103250002E08900001000100100F980000C2B3007A
:10326000F259020000000000A09C200010407800ED
:103270000044B2000004E0001300320061002000AE
:10328000606920002880020000000000A09C20004F
:1032900010407800684060000004E0000400320044
:1032A0001E089000467E020000000000100F9800EB
:1032B0001E0890003E7D02000000000000C2B30026
:1032C000F2590200000000000E0890000000E90022
:1032D000000F98000E0890000000E000B0FF3A00D8
:1032E000C07C2800C255020000000000DE0037004C
:1032F00061002000606920002880020000000000BA
:10330000B20207000000E800000F9800D202070098
:10331000300798003E0090000000E00044003200BA
:103320003E00900080407800909B2000014878008B
:103330003E009000E80F500006003400A09C2000E2
:10334000104078000050A000A19C20008048780028
:1033500037003700A09C2000104078000050A100EA
:10336000A19C20008048780031003700A1408000F7
:10337000E00220000088B900EA004000008320003D
:10338000008040001000780000000100100F98003D
:10339000A09C200010407800684060000004E0001D
:1033A000040032001E089000467E0200000000006B
:1033B000100F98001E0890003E7D020000000000E3
:1033C000A09C2000104078000042B2000004E00001
:1033D00004003A00909B200010407800E84F500015
:1033E00009003A00A09C2000104078000042B20082
:1033F0000004E0000B003200909B20001040780099
:10340000F04F500007003200B0C3B300F259020081
:1034100000000000909B2000104078002E58020011
:103420000000000000C2B300F259020000000000DA
:103430000E0890000000E900000F98000E089000B0
:103440000000E000C9FF3A00C07C2800C25502001D
:10345000000000008400370081002000C0692000C7
:10346000B280020000000000A1408000E0022000C5
:103470000088B900EC00400000832000008040007C
:103480001000780000000100770037008100200064
:10349000406A2000B280020000000000A1408000CD
:1034A000E00220000088B900EE0040000083200008
:1034B0000080400010007800000001006A00370022
:1034C000E1002000C06A2000B2800200000000007D
:1034D000A1408000E00220000088B900F000400018
:1034E00000832000008040001000780000000100F0
:1034F0005D003700E1002000A06B2000B2800200D8
:1035000000000000A1408000E00220000088B90017
:10351000F20040000083200000804000100078008E
:103520000000010050003700C1002000B0672000FB
:103530002880020000000000A1408000E00220007E
:103540000088B900F40040000083200000804000A3
:10355000100078000000010080550200000000000B
:103560004100370019020700000F9800D100200029
:10357000806D200028800200000000000E089000EE
:103580003E7D0200000000000E0890000000E800F0
:10359000000F980008003700A1408000E0022000E2
:1035A0000088B900F6004000008320000080400041
:1035B00010007800000001000E0890000000E900F3
:1035C000000F98000E0890000000E000F2FF3A00A3
:1035D000C07C2800C2550200000000002200370015
:1035E000FA0107000000E800000F9800A100200089
:1035F000506E200028800200000000000D003700FF
:10360000A1408000E00220000088B900F8004000DE
:1036100000832000008040001000780000000100BE
:10362000805502000000000000C2B300F259020001
:10363000000000000E0890000000E900000F980054
:103640000E0890000000E000EDFF3A0001012000AC
:10365000806C2000B28002000000000002003700F1
:103660001000200090578800805780008000E800FC
:10367000F00F200000806000805788009057800085
:103680000000E0001C00320051012000F06E20001C
:103690002880020000000000BE08900080578000D3
:1036A000808F5000070031008057800080407800F4
:1036B0003E08900000C050002E580200000000009C
:1036C0000600370080578000804078003E08900058
:1036D00000C050002E580200000000000000EB0067
:1036E0009057880010002000500F9800C07C2800E0
:1036F000C255020000000000815780007057800012
:10370000808F500002003A0010002000500F9800F7
:103710005E0890000000E00036FB32004E0890008A
:10372000805788004E089000705788000000EB001A
:10373000600F9800CCF637000600FA000000EB009E
:10374000100798000000EB00000F78008157800000
:103750001E00900080804000F00F200080806000FC
:10376000E09E2000008040009040780000C3B3003D
:1037700080CF500043003400815780001E0090002D
:1037800080804000F00F200080806000E09E2000DC
:10379000008040009040780090C3B30080CF50007C
:1037A00038003C00815780001E009000808040005F
:1037B000F00F200080806000E09E2000008040002C
:1037C000104078008000FB0000FD2F00008F4000BB
:1037D0001E0090000000E80010079800120037005B
:1037E0001E0078006A00B900000F78008157800041
:1037F0001E00900080804000F00F2000808060005C
:10380000E09E200000804000104078000000FB0097
:103810009E00400000FD2F00008F40001E00900021
:103820000000E80010079800815780001E009000FB
:1038300080804000F00F200080806000E09E20002B
:103840000080400090407800F0C2B30080CF50006C
:1038500051013400815780001E009000808040009C
:10386000F00F200080806000E09E2000008040007B
:103870009040780090C3B30080CF5000D8FF340050
:1038800045013700815780001E0090008080400075
:10389000F00F200080806000E09E2000008040004B
:1038A0009040780000C3B30080CF500035013A004B
:1038B0001E0090000000E80010079800815780006B
:1038C0001E00900080804000F00F2000808060008B
:1038D000E09E2000008040009040780020C6B300A9
:1038E00080CF50000B003200815780001E009000F6
:1038F00080804000F00F200080806000E09E20006B
:10390000008040009040780020C4B30080CF500079
:103910002D003A001E0090000000E80010079800FB
:10392000120037001E00780000004000000F7800F1
:10393000815780001E00900080804000F00F200022
:1039400080806000E09E20000080400010407800F1
:103950000000FB009E00400000FD2F00008F400093
:103960001E0090000000E8001007980081578000BA
:103970001E00900080804000F00F200080806000DA
:10398000E09E2000008040009040780010C3B3000B
:1039900080CF5000E3FF3200815780001E0090006E
:1039A00080804000F00F200080806000E09E2000BA
:1039B000008040009040780000C3B30080CF5000EA
:1039C000D8FF3200F4003700815780001E009000BD
:1039D00080804000F00F200080806000E09E20008A
:1039E000008040009040780080C7B30080CF500036
:1039F0000B003200815780001E0090008080400044
:103A0000F00F200080806000E09E200000804000D9
:103A10009040780080C5B30080CF50008E003A00FF
:103A20001E0090000000E8001007980047003700D3
:103A30001E0078004400DD00000F780081578000F0
:103A40001E00900080804000F00F20008080600009
:103A5000E09E20000080400090407800F0C2B3005B
:103A600080CF500018003400815780001E00900065
:103A700080804000F00F200080806000E09E2000E9
:103A8000008040009040780090C3B30080CF500089
:103A90000D003C00815780001E0090008080400097
:103AA000F00F200080806000E09E20000080400039
:103AB000104078000000FB009E00400000FD2F0039
:103AC000008F40001E003700815780001E009000CC
:103AD00080804000F00F200000816000815780004E
:103AE0001E00900080804000F00F20008080600069
:103AF000E09E2000008040009040780000C2B300AB
:103B000080C07000E09E2000000041000148780065
:103B1000815780001E00900080804000F00F200040
:103B200080806000E09E200000804000104078000F
:103B30000000FB009E00400090FA2F00008F400024
:103B40001E0090000000E8001007980081578000D8
:103B50001E00900080804000F00F200080806000F8
:103B6000E09E20000080400090407800F0C2B3004A
:103B700080CF50000B003400815780001E00900061
:103B800080804000F00F200080806000E09E2000D8
:103B9000008040009040780090C3B30080CF500078
:103BA000A3FF3400815780001E00900080804000F9
:103BB000F00F200080806000E09E20000080400028
:103BC0009040780000C4B30080CF50000B00340058
:103BD000815780001E00900080804000F00F200080
:103BE00080806000E09E20000080400090407800CF
:103BF00060C4B30080CF50008DFF34008157800037
:103C00001E00900080804000F00F20008080600047
:103C1000E09E2000008040009040780000C6B30085
:103C200080CF50005C003400815780001E0090005F
:103C300080804000F00F200080806000E09E200027
:103C4000008040009040780060C6B30080CF5000F4
:103C500077FF340050003700815780001E0090002D
:103C600080804000F00F200080806000E09E2000F7
:103C70000080400090407800F0C2B30080CF500038
:103C800045003400815780001E0090008080400075
:103C9000F00F200080806000E09E20000080400047
:103CA0009040780090C3B30080CF50003A003C00B1
:103CB000815780001E00900080804000F00F20009F
:103CC00080806000E09E200000804000104078006E
:103CD0008000FB0000FD2F00008F40001200370025
:103CE0001E0078006A00B900000F7800815780003C
:103CF0001E00900080804000F00F20008080600057
:103D0000E09E200000804000104078000000FB0092
:103D10009E00400000FD2F00008F40001E0090001C
:103D20000000E80010079800815780001E009000F6
:103D300080804000F00F200080806000E09E200026
:103D40000080400090407800F0C2B30080CF500067
:103D500011003400815780001E00900080804000D8
:103D6000F00F200080806000E09E20000080400076
:103D70009040780090C3B30080CF5000D8FF34004B
:103D80000500370010002000905788000000EB006D
:103D9000200798000A003700815780001E0090001D
:103DA000008040008057880081578000F00F20007D
:103DB00000806000805788001E007800200798006F
:103DC0002E0090000080FA00000006000400FA00B7
:103DD000805780008000E800F00F200080806000A5
:103DE000E09E20000080400090407800A0C3B30017
:103DF00080CF500013003A00805780000080E80018
:103E00008057880081578000F00F200000806000FC
:103E10008057880048FE0700000F78008057800018
:103E20000000E9008057880081578000F00F2000D3
:103E300000806000805788001E00780010079800FE
:103E40000200370010002000100798001E009000AC
:103E50000080FA00000006000400FA00805780008D
:103E60008000E800F00F200080806000E09E2000CD
:103E70000080400090407800B0C3B30080CF500075
:103E80000F003A00805780008080E800F00F20008B
:103E9000008060008057880027FE0700000F780030
:103EA000805780008000E900F00F20000080600053
:103EB000805788001E007800100798000200370025
:103EC0000000EB00100798001E0090000080FA0030
:103ED000000006000000FA0005003700805780004F
:103EE0008000E800F00F200000806000805788000C
:103EF00081578000E09E20000080400090407800C4
:103F000000C2B30080CF5000F4FF32000080FA00FE
:103F1000000006000400FA000000EB00000F78002B
:103F2000805780008000E800F00F200000806000D3
:103F300080578800E7FF0700FFFD0700000F7800AB
:103F40001E00E0004D003A000000EB001007980052
:103F5000130037001E0090000040E8002E580200B9
:103F600000000000C07F28009655020000000000FD
:103F70009E009000E00220000088B900610220004D
:103F8000808040000083200000804000C255020075
:103F9000000000001E0090000000E80010079800DC
:103FA0001E009000E50F5000EAFF34007101200070
:103FB00040702000B2800200000000000000EB0012
:103FC000905788001300200062002000110020009C
:103FD0001000200055000700000FE900E0FF2F004F
:103FE0009E0F1000030032000080EB009E0F1000B7
:103FF00005003A00E1002000B0712000B28002000C
:104000000000000042003700A1408000E0022000D4
:104010000088B90001022000808040000083200059
:10402000008040001000780000000100367C020093
:10403000000000001E007800A0408800A140800021
:10404000E00220000088B900FE004000008320004C
:104050000080400010007800000001001E00E00019
:1040600001003200CA82A80051002000305A20000E
:10407000B280020000000000250037001E0FE9009A
:10408000500020009E0F10001D003C00A140800049
:10409000E00220000088B90001022000808040007A
:1040A0000083200000804000100078000000010024
:1040B000367C0200000000001E007800A04088004E
:1040C000A1408000E00220000088B900FE0040000E
:1040D00000832000008040001000780000000100F4
:1040E0001E00E00001003200CA82A800510020003A
:1040F000305A2000B28002000000000004003700A7
:104100005101200090722000B280020000000000E7
:10411000705780008000E900F00F200000806000F0
:10412000805788000080FA00000006001E00FA0098
:10413000100F9800210F9800320F9800430F98003D
:104140000000EB00400798000000EB0020079800FB
:104150000000EB00100798000000EB00000F780053
:10416000F07F280096550200000000001E08900015
:104170002E580200000000003080280096550200F2
:104180000000000067003700E05902000000000056
:10419000204F98002E4890000000FB00600F980010
:1041A0006E089000ED0F500029003200EE089000DC
:1041B000ED8F500007003C006E099000E80F5100A1
:1041C0000D0032006E089000EA0F5000200032000F
:1041D00035003700D0022000EE089000808F50009C
:1041E0001E003200800720006E099000800F5100F1
:1041F000270032002C0037004E0090000000E00045
:10420000070032004E0090000000E90040079800CF
:10421000307B280096550200000000004100370066
:104220001E00E000060032000000EB00000F7800E6
:10423000307B28009655020000000000390037004E
:1042400070C0B300F25902000000000035003700D2
:104250001000200020079800320037004E00900028
:104260000000E00006003A00D0C2B300F25902009C
:104270000000000010002000000F78002900370027
:1042800070C0B300F25902000000000025003700A2
:104290004E0890000000E000030032000080EB00B8
:1042A000500F98005D003700AE489000F0C2B30098
:1042B00080CF500018003400AE48900090C3B30087
:1042C00080CF500014003C004E009000E30F5000DF
:1042D0000600340070C0B300F25902000000000074
:1042E00040002000400798000E0037002E48900044
:1042F000F259020000000000CE0090006B00470061
:104300002E499000827078004E0090000000E80076
:10431000400798000300370070C0B300F259020054
:10432000000000002E0090000000E00096FF320028
:10433000C07C2800C2550200000000004E00900022
:104340000000E00003003A001E089000500F9800A3
:10435000320037000000EB00100798004E0090007C
:104360000000E90040079800CE0090003107980057
:10437000110037001E0090006A00B9001007980075
:10438000BE0090004E009000808050006B004700FF
:10439000614078008000FB001E009000808040009B
:1043A00000FD2F0000804000100798004E00900094
:1043B0000000E900400798004E0090000000E00077
:1043C000ECFF3D009E0090002E089000808F500072
:1043D0000D0035009E0090003E089000808F500038
:1043E00009003C001E00E000040032001E009000A6
:1043F0000000EA00500F9800080037001E019000EE
:10440000520F980005003700B1012000E0EA2000BB
:10441000B28002000000000049FF37005E089000F3
:104420000080FA00000006000400FA0070802800F6
:10443000C25502000000000060812800965502006D
:1044400000000000B0C5B300F259020000000000F7
:104450000000EB00000F78000F0037001E00E000A6
:104460000300320000C2B300F25902000000000055
:104470009E007800E00220000088B9006102200060
:10448000808040000083200000804000965502009C
:10449000000000001E0FE800500020009E0F1000DA
:1044A000EEFF3600D0C5B300F25902000000000054
:1044B000D100200070802000288002000000000051
:1044C000A1BF2A000000EB004C5B020000000000CE
:1044D000000F78001E0078004800DE002E58020011
:1044E00000000000E0C2B300F2590200000000002A
:1044F0001E0078002E58020000000000C07C28003A
:10450000C25502000000000061002000007620007B
:104510002880020000000000B0408000E85802003F
:10452000000000007100200070EA200028800200D6
:1045300000000000C0408000E858020000000000B9
:10454000308328009655020000000000C140800022
:1045500011079800200423009E009000808F5000D7
:1045600016003200200423009E009000808F50002F
:1045700005003E00300023009E009000808F500018
:104580000A00320019003700300423009E0090001A
:10459000808F50000D003200600423009E009000C8
:1045A000808F50000D00320010003700208428005A
:1045B00096550200000000000F00370050842800CC
:1045C00096550200000000000B0037008084280090
:1045D000965502000000000007003700B084280054
:1045E000965502000000000003003700E084280018
:1045F000965502000000000020852800C2550200E8
:1046000000000000E101200060762000B28002007E
:10461000000000000080FA00000006000000FA0020
:10462000510020002092200028800200000000009D
:10463000C1BF2A000000EB004C5B0200000000003C
:10464000E858020000000000610020007092200085
:104650002880020000000000E1BF2A000000EB00FB
:104660004C5B020000000000E8580200000000005F
:10467000C07C2800C255020000000000C1002000DC
:1046800040782000B2800200000000005D000700BA
:10469000CAC2BF000042B2000004E00005003200C0
:1046A0001101200080652000288002000000000029
:1046B00004003700210120009066200028800200BD
:1046C00000000000C0C2B300F25902000000000068
:1046D00000C2B300F259020000000000A09C2000BC
:1046E00010407800704060000004E00005003200D7
:1046F0002102200000792000B280020000000000AA
:1047000004003700E1012000207B2000B28002007D
:1047100000000000A09C200010407800684060006D
:104720000004E00005003A00B1012000007D2000F7
:10473000288002000000000004003700C1012000B2
:10474000B07E20002880020000000000C0C2B3003C
:10475000F25902000000000000C2B300F25902004A
:1047600000000000B1012000C020210028800200CC
:1047700000000000909B2000104078002E5802009E
:1047800000000000C07C2800C255020000000000AC
:10479000A09C20001040780063406000E14F500072
:1047A00005003A0051012000E05B2000B2800200C9
:1047B000000000000400370061012000805A200042
:1047C000B280020000000000A1408000E002200052
:1047D0000088B90041022000808040000083200052
:1047E000008040001000780000000100C10020009F
:1047F00040782000B2800200000000000080FA0033
:10480000000006000000FA00A1002000A005210021
:10481000B28002000000000061042000200B210093
:10482000B280020000000000A1012000400621002B
:104830002880020000000000A1408000E00220006B
:104840000088B90021022000808040000083200001
:10485000008040001000780000000100A10020004E
:10486000E007210028800200000000000040200036
:1048700050000700001020004E000700002020001C
:104880004C000700000420004A0007000008200038
:1048900048000700C07C2800C2550200000000004C
:1048A00041002000800F210028800200000000004D
:1048B00021E3A800A0C0B300867C02000000000035
:1048C000325902000000000011002000903A200040
:1048D000288002000000000090C0B300F2590200DE
:1048E0000000000090C0B300867C020000000000C1
:1048F000325902000000000011002000903A200010
:10490000288002000000000090C0B300F2590200AD
:1049100000000000C0C0B300867C02000000000060
:10492000325902000000000011002000903A2000DF
:10493000288002000000000090C0B300F25902007D
:1049400000000000B0C0B300867C02000000000040
:10495000325902000000000011002000903A2000AF
:10496000288002000000000090C0B300F25902004D
:104970000000000021E3A900004020001C00070007
:10498000001020001A000700002020001800070077
:104990000004200016000700000820001400070093
:1049A000C07C2800C2550200000000000080FA0010
:1049B000000006000200FA00000F78004016800098
:1049C0001E0060000000E000040032004085280066
:1049D0009655020000000000030037007085280093
:1049E00096550200000000000080FA00000006005A
:1049F0000200FA00000F7800501680001E006000D0
:104A00000000E00004003200A08528009655020056
:104A10000000000003003700D085280096550200F2
:104A2000000000000080FA00000006000200FA000A
:104A3000805780008000E800F00F200000806000B8
:104A40008057880023FD07003BFB0700000F78001C
:104A50001E00E00006003400400020009E0F100001
:104A600003003C001E00E900904088000D00370064
:104A70000000EB00905788002102200040812000B8
:104A8000B2800200000000008001EB004200200024
:104A90001100200010002000A4FD07000000E90024
:104AA000904088002101200060832000B280020035
:104AB000000000000080FA00000006000200FA007A
:104AC000805780008000E800F00F20000080600028
:104AD00080578800FFFC070017FB0700104798006D
:104AE0001E4090000004E000090032001E409000CB
:104AF000EA4F500006003E001E4090000040E900D2
:104B00008040780000812000014878000F003700C5
:104B10000000EB0090578800D1082000308720006B
:104B2000B2800200000000008001EB00A200200023
:104B300011002000900020007CFD07000040E900EB
:104B4000804078000081200001487800008120002A
:104B500010407800E94F500010003A00DDFC0700DB
:104B6000F5FA0700004F78001E04E0000B003A0041
:104B70000000EB009057880000862800C255020014
:104B8000000000008001EB00F2FF27008000EB0036
:104B90002002200065FD0700004F78004101200041
:104BA00000902000B28002000000000011012000EF
:104BB000B01F2100B28002000000000023C2BF002D
:104BC000614060000004E000FCFF32000081200032
:104BD00010407800E94F500003003A001E40780072
:104BE000105A020000000000107D020000000000CA
:104BF00000003700D4590200000000000004E0006B
:104C0000FCFF3200E0590200000000008040780004
:104C100000C2B30080CF500001003200F5FF370022
:104C20000080FA00000006000000FA0031618000F8
:104C3000E0C22000008040009040780030C8B300FF
:104C400080CF50000E003A00306180000000E80084
:104C50003061880003003700306180000000E80008
:104C60003061880031618000E0C220000080400097
:104C70009040780000CEB30080CF5000F6FF3600A1
:104C80000080FA00000006000A00FA0030079800D1
:104C90000000EB0020079800AE009000E0C220006A
:104CA000008040009040780000CEB30080CF5000DC
:104CB00003003E000080EB0040079800230037000F
:104CC000AE009000E0C2200000804000104078005C
:104CD0008080FB0000F22F00008040001007980049
:104CE0002E0090008000E800E0C22000008040001C
:104CF000104078000080FB004801DD002E0090008D
:104D00008080E800E0C22000008040001040780071
:104D10000080FB00000F41009E0078003E009000E4
:104D2000808F500003003A002E009000400798004A
:104D3000060037009E0090002E009000008040008A
:104D40006300400020079800D3FF37004E0090001A
:104D50000080FA00000006000600FA00881F7800B4
:104D60000000EB00000F780031618000E0C22000FD
:104D7000008040009040780080C2B30080CF500097
:104D800010003A00306180000000E80030618800C7
:104D90001F010700000F780031618000E0C2200091
:104DA000008040009040780090C2B30080CF500057
:104DB000AC003A00306180000000E80030618800FB
:104DC000A800370031618000E0C220000080400070
:104DD0009040780000C4B30080CF50001600360029
:104DE00031618000E0C220000080400090407800E7
:104DF000A0C5B30080CF50000F003E00326180009C
:104E0000E0C2200000004100104078008080FB00DC
:104E1000F0FB2F00008040008000400060BC2000BC
:104E20000080400010007800200798000200E80091
:104E3000306188008D00370031618000E0C22000C1
:104E4000008040009040780000C8B30080CF500040
:104E50007600360031618000E0C220000080400012
:104E6000104078000080FB00100798000100E80067
:104E700030618800700920009E009000808F5000F3
:104E800041003200700920009E009000808F500089
:104E90000D003C00400920009E009000808F5000D3
:104EA00016003200600920009E009000808F5000A4
:104EB0002B003200300920009E009000808F5000AF
:104EC0001800320048003700A00920009E00900022
:104ED000808F500036003200D00920009E009000E4
:104EE000808F50001A003200800920009E00900040
:104EF000808F5000350032003B003700A140800019
:104F0000E00220000088B900EA0040000083200091
:104F1000008040001000780000000100000F7800C1
:104F200050003700A1408000E00220000088B90056
:104F3000E80040000083200000804000100478005A
:104F40008400070008000100000F780045003700CA
:104F50000A5F020000000000000F780041003700E7
:104F6000A1408000E00220000088B900F400400069
:104F70000083200000804000100078000000010045
:104F8000000F780037003700A1408000E0022000C9
:104F90000088B900F8004000008320000080400035
:104FA0001000780000000100000F78002D0037008D
:104FB000CAC2BF000080FB004500DE006140600007
:104FC0000080FB00000F78002600370021E3A800D6
:104FD000C0C0B300867C020000000000000F780013
:104FE00021E3A9001F0037000000EB00000F78004C
:104FF0001C0037001E0078006A00B900000F78001E
:1050000031618000E0C22000008040001040780044
:105010000080FB009E00400000FD2F00008F40003C
:10502000306180000000E80030618800316180005C
:10503000E0C220000080400090407800F0C2B30041
:1050400080CF50000700360031618000E0C22000B0
:10505000008040009040780090C3B30080CF5000A3
:10506000E4FF36001E007800200798002E00900014
:105070004F0478000080FA00000006000600FA00E5
:1050800035FF0700000F7800000037003161800015
:10509000E0C220000080400090407800A0C2B30031
:1050A00080CF50000A00320031618000E0C2200051
:1050B0000080400090407800F0C2B30080CF5000E4
:1050C000030032001E007800200798001E00370001
:1050D00031618000E0C22000008040001040780074
:1050E0000080FB00100798000100E8003061880094
:1050F000A00220009E009000808F5000050032002A
:10510000F00220009E009000808F500007003200C7
:10511000DEFF370010FF0700800078001E007800D7
:105120000180B900000F7800D8FF37000AFF0700A0
:10513000000178001E007800110009000200D8006C
:10514000000F7800D1FF37002E0090000080FA0099
:10515000000006000600FA00C8FF0700000F7800F4
:105160000000370031618000E0C220000080400074
:1051700090407800D0C2B30080CF50000A003200C7
:1051800031618000E0C22000008040009040780043
:10519000B0C2B30080CF5000030032001E00780080
:1051A000200798001700370031618000E0C220001E
:1051B00000804000104078000080FB00100798003D
:1051C0000100E80030618800B00220009E009000DD
:1051D000808F500008003200D00220009E00900016
:1051E000808F500001003200DEFF3700A3FF070070
:1051F0001E0F1000DBFF3700A0FF07001E0F40004E
:10520000D8FF37002E0090000080FA000000060052
:105210000C00FA0032618000E0C220000000410072
:10522000104078008080FB00F0FB2F0000804000E1
:105230008000400060BC20000080400090007800AA
:10524000210798000200E800306188000000EB00B0
:10525000000F78000B0037009E017800326180005B
:10526000E0C220000000410010407800804078003B
:1052700066004700817178000200E8003061880014
:105280001E0FE80031618000E0C220000080400075
:105290009040780000C4B30080CF50000700360073
:1052A00031618000E0C22000008040009040780022
:1052B000A0C5B30080CF50000E00360031618000E1
:1052C000E0C220000080400090407800F0C2B300AF
:1052D00080CF5000E0FF360031618000E0C2200046
:1052E000008040009040780090C3B30080CF500011
:1052F000D9FF3E0097FF070010079800660047009F
:10530000104078000000FB0050079800C003200008
:10531000DE009000808F500032003200C003200079
:10532000DE009000808F500005003C00100220003D
:10533000DE009000808F5000410032004E003700A8
:10534000D0032000DE009000808F50000500320066
:10535000E0032000DE009000808F50000A00320041
:10536000450037000000EB0040079800AE009000B9
:105370001E009000808F500041003A001100200074
:10538000410798003E0037006600470090409000BB
:10539000D0C3B30080CF500009003A000000EB00FA
:1053A00040079800AE0090001E009000808F5000D3
:1053B000330035001100200041079800300037000D
:1053C0000000EB0040079800AE0090001E00900027
:1053D000808F50002A0034001100200041079800FF
:1053E000270037006600470090409000D0C3B3000C
:1053F00080CF500009003A000000EB004007980001
:10540000AE0090001E009000808F50001C003C00F9
:105410001100200041079800190037000000EB0040
:1054200040079800AE0090001E009000808F500052
:1054300013003D00110020004107980010003700C4
:105440006600470090409000D0C3B30080CF50006A
:1054500009003A000000EB0040079800AE00900001
:105460001E009000808F50000500320011002000C7
:1054700041079800020037000000EB004007980049
:105480004E0090000080FA00000006001C00FA00A8
:10549000881F78000000EB00306188000000EB00FE
:1054A000300798000000EB00200798000000EB0098
:1054B000100798000000EB00406188000000EB003E
:1054C000506188000000EB00606188000000EB0084
:1054D00050079800D04080000080A000D040880095
:1054E0000000EB0040079800090037004E009000D4
:1054F0008000400060BC2000808040000000EB0085
:10550000800878004E0090000000E80040079800F6
:105510004E009000F90F5000F4FF340035043700BE
:105520001E0090000000E00021003A003161800080
:10553000E0C220000080400090407800F0CDB30031
:1055400080CF500003003E0020002000300798006C
:105550002B04370031618000E0C220000080400051
:10556000104078008080FB0000F22F000080400097
:1055700060079800306180008000E800E0C22000F1
:1055800000804000104078000080FB004801DD00F2
:10559000306180008080E800E0C220000080400090
:1055A000104078000080FB00000071005007980058
:1055B0000000EB001007980030618000E30040001D
:1055C000E0C2200000804000104078000080FB0016
:1055D0006101B90000F82F00F1FF2F000201400027
:1055E00083814800420F9800530F9800100220005A
:1055F000010020004E099000DE099000800F51004C
:10560000818F5900EF033E004E089000DE089000A5
:10561000006001002100370035003700E903370042
:10562000E80337007100370081003700A30037001E
:10563000B7003700BE0037003B0137008801370054
:10564000E0033700EE0137003502370099023700DA
:10565000AF0237009F023700CB023700BB02370092
:10566000D8023700D70337007C03370060033700C8
:10567000D4033700D303370004033700F0023700A8
:10568000A3033700AE033700DE02370016033700EE
:1056900036033700B6033700C70337001000200079
:1056A000200798003061800066004000306188006B
:1056B000306180008080E900E0C22000008040006E
:1056C000104078008080FB00F0FB2F000084400039
:1056D000A0FE0700000178008800440060BC2000A4
:1056E00000804000020878004FFD0700B703370034
:1056F0001000200020079800306180006400400006
:1057000030618800C2FE07000000E0001C0032008B
:1057100031618000310F9800E0C220003E09900006
:1057200000004100904078008041EB004357980012
:1057300020C8B30080CF500002003A0010C0B30070
:1057400040579800BE0890000100E80030618800D2
:105750004E5190000204E0009C0332001000200033
:1057600010079800306180006300500030618800AD
:1057700096033700306180000000E8003061880047
:1057800031618000E0C2200000804000904078003D
:1057900030C8B30080CF5000070032003161800074
:1057A000E0C22000008040009040780000CEB300AE
:1057B00080CF5000EFFF360031618000E0C2200052
:1057C000008040009040780030C8B30080CF500087
:1057D0007E033A001000200010079800306180001E
:1057E0000080E90030618800780337001000200055
:1057F000200798003061800064004000306188001C
:1058000054FE070020FD0700000F78008081EB00A8
:105810009E8F1100030032001E0078003061880066
:105820006A033700600020003007980067033700E4
:1058300010002000200798003061800064004000C4
:105840003061880050618000E90F500018003C0072
:1058500052618000316180006E0090000080400045
:105860008001E90082004100A0BF200000804000CC
:1058700003087800506180000000E8005061880053
:1058800034FE070000FD0700000F78008080EB0069
:105890009E8F1000030032001E01780032618800E4
:1058A0004A033700600020003007980047033700A4
:1058B0007000200030079800440337000070280073
:1058C00096550200000000001000200020079800FC
:1058D000506180000000E0000A003200506180004A
:1058E0000000E900506188005061800080004000A5
:1058F000A0BF2000008040001000780030618800C8
:105900003203370080002000300798002F03370053
:105910001000200020079800316180006E00900088
:10592000008040006300400030618800270337009A
:1059300010002000200798003061800064004000C3
:10594000306188005700370031618000E0C22000DC
:10595000008040009040780020C2B30080CF50000B
:105960001F003A00306180000000E80030618800CC
:1059700010003700D04080000080A100D040880097
:1059800031618000E0C220000080400010407800BB
:10599000004178000100E800306188000240780092
:1059A000F259020000000000D04080000080A000FA
:1059B000D040880031618000E0C2200000804000BB
:1059C0009040780020C2B30080CF5000E9FF3A0039
:1059D000306180000000E80030618800310037004D
:1059E00031618000E0C220000080400090407800DB
:1059F00000C4B30080CF5000070036003161800042
:105A0000E0C220000080400090407800A0C5B300B4
:105A100080CF50000D00360031618000E0C22000D0
:105A200000804000104078000004E00013003D00BA
:105A300031618000E0C2200000804000904078008A
:105A4000F0CDB30080CF50000C003E00C1FD070038
:105A5000000F7800D04080000080A100D040880076
:105A60001E007800D057020000000000D0408000E7
:105A70000080A000D04088000A003700316180001B
:105A8000E0C220000080400090407800B0C3B30026
:105A900080CF500003003A00306180000000E80031
:105AA0003061880031618000E0C220000080400049
:105AB00090407800F0CDB30080CF500007003E004A
:105AC00031618000E0C220000080400090407800FA
:105AD00030C8B30080CF50009BFF3A003061800097
:105AE0008000E900E0C22000008040009040780083
:105AF000B0C3B30080CF500009003200D040800016
:105B00000080A100D040880060792800C2550200C2
:105B100000000000D04080000080A000D04088003D
:105B200041FC0700A9023700100020002007980060
:105B3000D04080000080A100D0408800306180000B
:105B4000640040003061880031618000E0C22000C4
:105B5000008040009040780020C2B30080CF500009
:105B600018003A00306180000000E80030618800D1
:105B70000A00370031618000E0C220000080400050
:105B800010407800004178000100E8003061880092
:105B900002407800F25902000000000031618000EC
:105BA000E0C22000008040009040780020C2B30096
:105BB00080CF5000EFFF3A00306180000000E80025
:105BC0003061880031618000E0C220000080400028
:105BD00090407800C0C2B30080CF500004003A006B
:105BE000306180000000E80030618800020037006A
:105BF000300020003007980031618000E0C22000B2
:105C000000804000104078008080FB00F0FB2F00F7
:105C1000008440008001EB00F2FF27008000EB00D1
:105C20000000EB0096200200000000000001780058
:105C30008800440060BC200000804000020878001A
:105C4000306180000000E80030618800F6FB07004A
:105C5000D04080000080A000D04088005B02370068
:105C60001000200020079800306180006400400090
:105C70003061880040618000E30F500004003C0068
:105C8000406180000000E8004061880002003700A9
:105C9000400020003007980042618000336180009E
:105CA000E0C2200000804100104078008080FB00AE
:105CB00000FC2F00008240006610B9008080E800E0
:105CC000E0C0200000804000040878000300E800E5
:105CD0003061880031618000E0C220000080400017
:105CE00090407800D0C3B30080CF500011003A003C
:105CF000306180000000E800306188004061800071
:105D00006600B9008080E800E0C02000008040000C
:105D1000100078000004E9000EFD07000001780083
:105D20008800440060BC2000008040000208780029
:105D300002003700300020003007980033618000F7
:105D4000130F9800E0C220009E08900000804000E1
:105D5000904078000041EB0002579800B0C8B300B3
:105D600080CF500002003A0013C0B30003579800E0
:105D70009E0890000100E800306188000E519000FC
:105D80000204E0000900320048618000F1FC0700D5
:105D9000000178006640B900E4004000E0C0200047
:105DA0000080400002087800020037003000200028
:105DB0003007980031618000E0C220000080400080
:105DC00090407800F0CDB30080CF5000080036003E
:105DD00040618000326180006600B9008000780078
:105DE000E0C0200000804000020878000200370078
:105DF00030002000300798008BFB0700F3013700CC
:105E000010002000200798003061800064004000EE
:105E10003061880032618000E0C220000000410053
:105E2000104078008080FB0000FC2F00008F4000B5
:105E30000200E80030618800500020003007980020
:105E40000000EB00400798002F0037004E00900044
:105E50006600B9008080E800E0C0200000804000BB
:105E6000100078009E0F500024003A001E00E90048
:105E70008000400060BC20000080400010017800DD
:105E80004E0090006600B900E4004000E0C0200031
:105E90000080400010007800800F510012003D008B
:105EA0009E00E9000181400060BC2000000041002C
:105EB000100078000001E8008180400060BC2000F4
:105EC00000804000020878004E0090006600B90093
:105ED00080007800E0C020000080400010007800C2
:105EE0003061880003003700406180000000E90055
:105EF000406188000000EB00300798004E009000E1
:105F00000000E80040079800416180004E009000CA
:105F1000810F5000CDFF340043FB0700AB01370079
:105F200010002000200798003061800064004000CD
:105F300030618800606180000000E00027003A00C6
:105F40000000EB00400798000A003700CE009000E8
:105F5000E0C2200000804000104078008080FB00FC
:105F60004E0090008080400030F22F000080400002
:105F7000400798004E009000E3004000E0C220007F
:105F80000080400090407800E0C8B30080CF50000F
:105F900006003200CE009000E0C2200000804000E9
:105FA000104078000004E000E8FF3A00CE009000C6
:105FB000E0C2200000804000104078000004E000B3
:105FC000040032004E0090006400400060618800D0
:105FD00002003700900020003007980033618000F5
:105FE000030F780060618000306188009E007800B7
:105FF000E0C2200000804000104078008080FB005C
:10600000F0FB2F000084400053FB070000017800E4
:106010008800440060BC2000008040000208780036
:1060200030618000606188001E00E80030618800F7
:1060300061618000E0C22000008040009040780054
:10604000C0C2B30080CF500003003A0060618000FE
:106050000000E8006061880061618000E0C220000B
:10606000008040009040780000CEB30080CF500008
:106070000E00360060618000E3004000E0C22000B6
:106080000080400090407800E0C8B30080CF50000E
:10609000030032000000EB0060618800030037005D
:1060A000606180006400400060618800DEFA0700E3
:1060B0004601370010002000200798003161800061
:1060C0006E00900000804000630040003061880056
:1060D0003E0137001000200020079800306180004A
:1060E0006400400030618800A1408000E002200090
:1060F0000088B90080007800008320000080400004
:106100001000780000000100C7FA07002F013700D7
:1061100010002000200798003061800064004000DB
:1061200030618800A1408000E00220000088B900B2
:106130008080E8000083200000804000100078008C
:1061400000000100B8FA070020013700100020000D
:1061500020079800306180006400400030618800B2
:10616000A1408000E00220000088B900E400400067
:106170000083200000804000100078000000010033
:10618000A9FA07001101370010002000200798002D
:10619000306180006400400030618800A1408000D0
:1061A000E00220000088B900E600400000832000E3
:1061B0000080400010007800000001009AFA0700FB
:1061C0000201370010002000200798003061800095
:1061D0006400400030618800A1408000E00220009F
:1061E0000088B900E80040000083200000804000E3
:1061F00010047800D7FB0700080001008AFA0700A6
:10620000F200370010002000200798003061800065
:106210006400400030618800CEFB07000000E00011
:1062200003003200C65E02000000000002003700DA
:10623000E85E0200000000007BFA0700E300370080
:1062400010002000200798003061800064004000AA
:1062500030618800BFFB07000000E000050032004D
:10626000C082A900C282A800C8A2A900CAA2A80030
:1062700004003700C082A900C282A900C8A2A900F8
:10628000CAA2A90068FA0700D00037001000200059
:106290002007980030618000640040003061880071
:1062A000ACFB07000000E00007003200A09C2000CB
:1062B000104078000000A0000010A100A19C200068
:1062C0008048780006003700A09C2000104078002D
:1062D0000000A0000010A100A19C200080487800D0
:1062E00051FA0700B900370010002000200798007D
:1062F00030618000640040003061880095FB070039
:10630000504F8800504F80000000E00002003D0028
:106310000000EB00504F8800514F800000FA200031
:10632000808F50000200340000FA2000504F880097
:10633000604F8000E10F500002003C002000200070
:10634000604F8800614F800030062000808F500031
:106350000200340030062000604F8800705B0200AD
:106360000000000030FA07009800370010002000FD
:106370002007980030618000640040003061880090
:1063800074FB0700604F8800504F80000000E00061
:1063900002003D000000EB00504F8800514F80008C
:1063A00000FA2000808F50000200340000FA200024
:1063B000504F8800604F8000E10F500002003C0009
:1063C00020002000604F8800614F800030062000D0
:1063D000808F50000200340030062000604F88009B
:1063E000705B0200000000000FFA07007700370022
:1063F00010002000200798003061800064004000F9
:106400003061880053FB07000000E0000900320003
:10641000A1408000E00220000088B900F0004000A8
:106420000083200000804000100078000000010080
:1064300008003700A1408000E00220000088B90079
:10644000F20040000083200000804000100078002F
:1064500000000100F4F907005C0037001000200084
:10646000200798003061800064004000306188009F
:1064700038FB0700700798007E009000E10F500085
:1064800010003200FE009000E28F50001600320033
:106490007E0190000200E000010032001A00370087
:1064A000A1408000E00220000088B900EE0040001A
:1064B00000832000008040001000780000000100F0
:1064C00011003700A1408000E00220000088B900E0
:1064D000EC004000008320000080400010007800A5
:1064E0000000010008003700A1408000E002200009
:1064F0000088B900F60040000083200000804000C2
:106500001000780000000100C7F907002F003700D5
:1065100010002000200798003061800064004000D7
:1065200030618800316180006E0090000080400082
:106530000000E90030618800BBF907002300370044
:1065400010002000200798003061800064004000A7
:1065500030618800FFFA0700000F78001E00780005
:10656000E47D020000000000AFF9070017003700CB
:106570001000200020079800306180006400400077
:1065800030618800F3FA0700000F7800A140800016
:10659000E00220000088B900FC00400000832000D9
:1065A00000804000900078001E007800010001008B
:1065B0009DF9070005003700100020003007980003
:1065C0000200370030002000300798002E009000B5
:1065D0000000E00005003A00316180006E0090008C
:1065E0000080400063004000306188000000EB0044
:1065F000200798003E0090000000E000C8FB320039
:10660000D04080000080A100D04088003E00900073
:10661000E10F50001800320061002000A03A200075
:1066200028800200000000003E009000D0570200C9
:106630000000000081002000003B200028800200B4
:10664000000000005E009000D05702000000000033
:10665000B1002000803B20002880020000000000E4
:1066600030618000D05702000000000060792800EF
:10667000C2550200000000004F0478000080FA00BC
:10668000000006000200FA00000F780000C2B3000C
:10669000F2590200000000001E007800965502002A
:1066A0000000000000C2B300F25902000000000028
:1066B0000080FA00000006000400FA000000EB0071
:1066C000306188003F00370031618000E0C2200067
:1066D0000080400090407800214798002E409000B4
:1066E0000004E000040035002E409000F259020042
:1066F0000000000030003700AE40900000CEB30034
:1067000080CF50001C00360060792800C25502007E
:1067100000000000306180008000E800E0C220003E
:1067200000804000104078000080FB004801DD0040
:10673000306180008080E800E0C2200000804000DE
:10674000104078000080FB0000004100000F78003E
:10675000306180000080E800306188001E00780011
:10676000D05702000000000000C2B300F25902003E
:10677000000000001000370000C2B300F259020010
:10678000000000002E4090008080FB0000F82F00E9
:1067900000804000800040002097200000804000E2
:1067A00010007800965502000000000000C2B300FF
:1067B000F259020000000000306180000000E80093
:1067C0003061880031618000E0C22000008040001C
:1067D000104078000004E000BBFF3A006079280018
:1067E000C255020000000000306180000000E90096
:1067F000D05702000000000071002000303C200053
:10680000B2800200000000000080FA0000000600D4
:106810000600FA001007980080578000000F7800EB
:10682000150037001E00900010417800815780004D
:10683000E09E20000080400010407800804F510012
:10684000050032001E007800805788000000EB0031
:10685000200798000E003700805780008000E80075
:10686000F00F200000806000805788001E0090001C
:106870000000E800100798001E009000104078000B
:106880000004E000E7FF3A00100020002007980015
:106890002E0090000080FA00000006000400FA00BC
:1068A0000000EB00000F7800100037001E00780099
:1068B00080004000209720000080400010007800F9
:1068C000D3FF07000000E000070032001E00780040
:1068D0008040780000C8B30000C040000080FB008A
:1068E00010079800060037001E0FE8001002200075
:1068F0009E0F1000EDFF34000000EB001007980021
:106900001E0090000080FA00000006003600FA0029
:1069100080578000000F98001F0037008E089000FD
:10692000E09E2000008040009040780000C6B30048
:1069300080CF5000110034008E089000E09E2000AF
:106940000080400090407800A0C7B30080CF500086
:106950000A003C000E0990008E089000E09E200086
:106960000080400090407800F0CDB30080C060000F
:10697000E09E200000004100014878000E089000D1
:106980000000E800000F98008E089000F00F200033
:1069900000806000000F98008E0890007057800003
:1069A000808F5000DDFF3A000000EB00000F9800E0
:1069B00081578000E09E20000080400090407800D9
:1069C000F0C2B30080CF50002D0134008157800009
:1069D000E09E2000008040009040780090C3B3000B
:1069E00080CF500026013C000000EB00000F980013
:1069F000070037000E099000F20047000040EB004E
:106A000000F178000E0890000000E800000F9800E8
:106A10008E08900020022000808F5000F5FF340087
:106A20009C1B020000000000600798006E009000B0
:106A30004880DE00804078007200470011409800D6
:106A40006E0090008040780000C0EB0080C06000C5
:106A500072004700214098006E0090008AF80700FD
:106A6000500798005E009000E10F40002B003200BC
:106A7000DE009000E0C2200000804000104078005E
:106A80008080FB0030F22F0000804000300798002B
:106A90005E009000000F98000D0037000E09900076
:106AA0008E0890003E00900080804000E0C22000F0
:106AB0000080400090407800E0C2200000004100CB
:106AC000014878000E0890000000E800000F9800D0
:106AD000014020003E009000808050000E08900091
:106AE000808F5000EDFF3C00080037008E089000BA
:106AF000E0C22000808040000040EB008048780029
:106B00000E0890000000E800000F98008E0890002A
:106B1000F03F2000808F5000F4FF34003000200050
:106B2000000F98000000EB00200798006A1F020089
:106B300000000000430037002E0090000000E0003D
:106B400002003A006A1F0200000000002E009000C0
:106B50000000E00004003A0050FF07000080FB0046
:106B600060079800020037000000EB006007980003
:106B70006E00900090580200000000006E0090002F
:106B80000000E0000C0032000E0990006E00900042
:106B9000804078007200470001717800EE0090009C
:106BA00070082000808F50001A003A00100020006A
:106BB000200798001700370081578000E09E2000D2
:106BC000008040009040780020C2B30080CF500089
:106BD00003003A002E0090000000A2002007980059
:106BE0000E09900081578000E09E20000080400048
:106BF00010407800804078007200470001717800F2
:106C0000805780008000E800F00F200000806000C6
:106C1000805788000E0890000000E800000F9800E0
:106C20008E08900030022000808F50000500340054
:106C300091002000A03C2000B28002000000000073
:106C4000D40037008157800070578000808F50003B
:106C5000B9FF3A000E089000E30F5000CD0032005B
:106C60000E089000E40F5000CA0032000E08900099
:106C700080407800C0CDB30000C040008040780064
:106C800072004700014878000000EB00000F9800F8
:106C90000000EB00400798000000EB005007980050
:106CA000460037008E089000E0C2200000804000BF
:106CB0009040780000CEB30080CF50002E00360008
:106CC0008E089000E0C22000008040001040780054
:106CD0008080FB0000F22F00008040003007980009
:106CE0000E0890008000E800E0C220000080400014
:106CF000104078000080FB004801DD000E08900085
:106D00008080E800E0C22000008040001040780051
:106D10000080FB000000410010079800720047004F
:106D2000104090000080FB00C800DD0072004700AA
:106D3000204090000080FB0000804000000F7800A1
:106D40001E0090009E0F5000050031008E0890003C
:106D50003E00900000804000630040005007980013
:106D6000BE0090000E0890000080400063004000CC
:106D7000000F9800020037000E08900040079800AE
:106D80000E0890008000E800E0C220000080400073
:106D9000104078000080FB004801DD000E089000E4
:106DA0008080E800E0C220000080400010407800B1
:106DB0000080FB0000004100600798004E0090003A
:106DC0000000E000B7FF320072004700104078007A
:106DD0008080FB0030F22F000080400060079800A8
:106DE0004E009000000F98000D0037008E089000B4
:106DF0006E009000008140008E089000E0C22000EC
:106E00000080400090407800E0C220000000410077
:106E1000014878000E0890000000E900000F98007B
:106E20008E0890005E009000808F5000EFFF3D00C4
:106E30000000EB00000F98000C003700DE0090000F
:106E40000E089000008140008E08900072004700FC
:106E5000E1407800E0C220000000410001487800D5
:106E60000E0890000000E800000F98008E089000C7
:106E70006E009000808F5000F0FF35004500370015
:106E80007079280062FE07000000E0000500320073
:106E90007EF9070060792800C2550200000000005A
:106EA0003C003700B079280059FE07000000E000E0
:106EB0000200320000FE070036003700007A28008A
:106EC00053FE07000000E00004003200D0408000C4
:106ED0000090A100D04088002E003700507A280092
:106EE0004BFE07000000E000200032000000EB0035
:106EF000000F9800180037000000EB0070079800A2
:106F00000F0037008E0890007E00900080804000C7
:106F1000E0C2200000804000104078000080FB00AC
:106F2000905802000000000000C2B300F2590200B5
:106F3000000000007E0090000000E800700798004C
:106F40007E009000EF0F5000EEFF34000E0890001E
:106F500070004000000F98008E089000F03F200065
:106F6000808F5000E4FF34000A003700B07A280018
:106F700027FE07000000E0000200320007000700C3
:106F800004003700C1002000303D2000B280020024
:106F9000000000000080FA00000006000200FA0075
:106FA0000000EB00000F7800060037009E0078001C
:106FB000E0C22000808040000040EB008048780064
:106FC0001E0FE800F03F20009E0F1000F7FF340076
:106FD00011CEB300E0C220000148780080C0EB0071
:106FE000F0C220000148780080C0EB0000C3200000
:106FF0000148780011CAB30010C32000014878008E
:107000000080FA0000000600575249005445200055
:10701000424954003A2020002A6E6500787420000E
:10702000636C6F00636B2000285E29002077690085
:107030006C6C200075736500207468006973200013
:1070400076616C0075653100574952004520720029
:107050006F757400696E6500732028004329200055
:107060003230300030204D006963680061656C008B
:107070002050650061726300652047004E55200076
:1070800047504C004E6F20006465760069636500D0
:107090002C2074007279200028414C0041524D0090
:1070A0002920530045415200434820006D61630090
:1070B000726F20006669720073744100444452008C
:1070C00045535300204D410043524F0020203000D3
:1070D0002E4D610063726F00206D65006E754D006E
:1070E000616372006F20200020202000315749008A
:1070F000524520006164640072657300730D0A00DC
:10710000202020002A3157004952450020524F00CC
:107110004D2043004F4D4D00414E4400204D410055
:1071200043524F00733A0D000A203500312E5200B1
:107130004541440020524F004D2028003078330054
:10714000332920002A666F0072207300696E670081
:107150006C652000646576006963650020627500D7
:10716000730D0A00203835002E4D4100544348006D
:1071700020524F004D20280030783500352920005E
:107180002A666F006C6C6F0077656400206279007E
:107190002036340062697400206164006472650006
:1071A00073730D000A20320030342E00534B490017
:1071B000502052004F4D20002830780043432900D2
:1071C000202A66006F6C6C006F7765006420620097
:1071D000792063006F6D6D00616E64000D0A200000
:1071E000323336002E414C0041524D0020534500B1
:1071F00041524300482028003078450043290D00C3
:107200000A20320034302E005345410052434800DA
:1072100020524F004D202800307846003029410090
:107220004C4152004D20530045415200434820003C
:107230002830780045432900534541005243480017
:1072400020283000784630002944650076696300C4
:10725000652049004473200061726500206176005A
:1072600061696C0061626C006520620079204D00EC
:10727000414352004F2C20007365650020283000E8
:10728000292E52004541440020524F004D20280035
:107290003078330033293A00204D410054434800F0
:1072A00020524F004D2028003078350035295300FA
:1072B0004B49500020524F004D20280030784300A9
:1072C000432955006E6B6E006F776E00206D610074
:1072D00063726F002C207400727920003F206F00D1
:1072E0007220280030292000666F72002068650037
:1072F0006C70420055532000524553004554200005
:10730000576172006E696E00673A20002A53680068
:107310006F727400206F7200206E6F002070750015
:107320006C6C2D00757020002A4E6F002064650083
:1073300076696300652064006574650063746500A8
:107340006420440053313800533230002048690033
:107350006768200050726500732044006967200050
:1073600054686500726D4400533138004232300079
:10737000205072006F67200052657300204469003E
:1073800067205400686572006D4453003138320044
:1073900032204500636F6E0020446900672054006E
:1073A000686572006D44530032343000342045006B
:1073B000636F6E0072616D00207469006D6520005E
:1073C0004368690070445300323433003120310087
:1073D0004B204500455052004F4D55006E6B6E00DE
:1073E0006F776E0020646500766963006550570012
:1073F0004D20640069736100626C650064314B006C
:10740000487A2D00342C300030304B00487A200070
:1074100050574D0046726500717565006E637900C6
:1074200020696E00204B48007A205000726573007E
:1074300063616C00653A500052323A004475740042
:107440007920630079636C00652069006E20250057
:10745000205057004D206100637469007665450037
:1074600052524F00523A200050574D0020616300A5
:1074700074697600652C2000672074006F2064001A
:1074800069736100626C65004155580020467200C6
:1074900065717500656E6300793A200041555800AA
:1074A00020494E00505554002F4849002D5A4100A4
:1074B00055582000484947004841550058204C0085
:1074C0004F5756004F4C54004D4554004552200034
:1074D0004D4F440045564F004C5441004745200055
:1074E00050524F0042453A002056450072726F00DC
:1074F0007228290020406C00696E65003A20400027
:1075000070676D007370610063653A0020627900F6
:10751000746573002E546F006F206C006F6E6700EF
:10752000215379006E7461007820650072726F00DB
:10753000724E6F002045450050524F004D4572007D
:10754000617369006E6764006F6E65005361760059
:10755000696E670020746F0020736C006F742000E8
:10756000496E7600616C6900642073006C6F740072
:107570004C6F610064696E0067206600726F6D0079
:1075800020736C006F742000455252004F523A0035
:1075900020636F006D6D61006E6420006861730090
:1075A000206E6F00206566006665630074206800C9
:1075B0006572650041434B004E4143004B49320028
:1075C0004320530054415200542042004954490082
:1075D0003243200053544F00502042004954490088
:1075E000324320006D6F6400653A0D000A203100BF
:1075F0002E2053006F66740077617200650D0A00DB
:1076000020322E00204861007264770061726500AC
:107610005365740020737000656564003A0D0A00BC
:1076200020312E00207E35004B487A000D0A2000C4
:10763000322E20007E3530004B487A000D0A2000A3
:10764000332E20007E313000304B48007A0D0A0086
:1076500020342E00207E340030304B00487A570012
:1076600041524E00494E47003A20480041524400E2
:1076700057415200452049003243200069732000E1
:1076800062726F006B656E00206F6E002074680080
:1076900069732000504943002120280052455600BC
:1076A0002041330029536500742073007065650024
:1076B000643A0D000A2031002E20310030304B009A
:1076C000487A0D000A2032002E20340030304B0062
:1076D000487A0D000A2033002E2031004D487A00F0
:1076E0004932430020286D006F64200073706400ED
:1076F000293D2800202030002E4D610063726F006C
:10770000206D65006E750D000A2031002E37620075
:1077100069742000616464007265730073207300F3
:107720006561720063680D000A2032002E49320044
:10773000432073006E6966006665720053656100E0
:1077400072636800696E670020493200432061005F
:107750006464720065737300207370006163650078
:107760002E2046006F756E00642064006576690007
:1077700063657300206174003A536E0069666600A9
:107780006572280042415300494329005265610057
:10779000647961002F412F00402063006F6E7400F8
:1077A000726F6C00732041005558200070696E00A4
:1077B000612F41002F402000636F6E0074726F00D4
:1077C0006C7320004353200070696E00436F6D009E
:1077D0006D616E0064206E006F742000757365002B
:1077E000642069006E20740068697300206D6F006A
:1077F00064655000756C6C002D757000207265001A
:1078000073697300746F720073204F004646500016
:10781000756C6C002D7570002072650073697300C3
:10782000746F720073204F004E5365006C662D001C
:1078300074657300742069006E204800695A200046
:107840006D6F640065206F006E6C790052455300C7
:10785000455442004F4F54004C4F410044455200A4
:107860004155580020494E00505554002F484900BA
:107870002D5A2C002052450041443A0020506F0000
:10788000776572002073750070706C006965730015
:10789000204F4E00506F77006572200073757000A6
:1078A000706C6900657320004F46460044415400E7
:1078B0004120530054415400453A200044454C00B7
:1078C000415920007573570052495400453A200031
:1078D00052454100443A2000434C4F00434B2C009A
:1078E000203143004C4F43004B2C200030444100DA
:1078F000544120004F555400505554002C20310065
:107900004441540041204F005554500055542C0020
:10791000203020002A7069006E20690073206E00FC
:107920006F77200048695A00434C4F00434B2000BA
:10793000544943004B533A00205245004144200033
:10794000424954003A205300796E74006178200057
:10795000657272006F7220006174200063686100BC
:10796000722078002E2065007869740028776900FD
:1079700074686F0075742000636861006E6765004D
:10798000296E6F00206D6F006465200063686100E0
:107990006E6765004E6F6E006578690073746500F0
:1079A0006E74200070726F00746F63006F6C210042
:1079B000782E200065786900740D0A00496E760003
:1079C000616C690064206300686F690063652C0066
:1079D0002074720079206100676169006E4445007F
:1079E000564944003A68740074703A002F2F6400BE
:1079F000616E670065726F0075737000726F74005E
:107A00006F747900706573002E636F006D2A2D000E
:107A10002D2D2D002D2D2D002D2D2D002A4F7000E8
:107A2000656E200064726100696E20006F757400DD
:107A30007075740073202800483D4800692D5A0075
:107A40002C204C003D474E0044294E006F726D00C3
:107A5000616C20006F7574007075740073202800CD
:107A6000483D33002E3376002C204C003D474E001D
:107A700044294D0053422000736574003A204D00A4
:107A80004F5354002073690067206200697420001E
:107A90006669720073744C00534220007365740071
:107AA0003A204C0045415300542073006967200080
:107AB00062697400206669007273740020426F006E
:107AC0006F746C006F616400657220007620310075
:107AD0002E20480045580D000A2032002E20440078
:107AE00045430D000A2033002E204200494E0D0070
:107AF0000A2034002E205200415744006973700060
:107B00006C61790020666F00726D610074207300F3
:107B1000657456006F6C740061676500206D6F00BE
:107B20006E6974006F7273003A203500563A200077
:107B3000207C2000332E3300563A2000207C200089
:107B4000565055004C4C5500503A20005365740077
:107B500020736500726961006C2070006F727400A0
:107B600020737000656564003A202800627073001D
:107B7000290D0A0020312E0020333000300D0A007C
:107B800020322E002031320030300D000A20330028
:107B90002E203200343030000D0A2000342E200018
:107BA00034383000300D0A0020352E0020393600E0
:107BB00030300D000A2036002E20310039323000DE
:107BC000300D0A0020372E002033380034303000CA
:107BD0000D0A2000382E20003537360030300D00D9
:107BE0000A2039002E2031003135320030300D00AE
:107BF0000A3130002E204200524720007261770087
:107C0000207661006C75650041646A0075737400CC
:107C100020796F0075722000746572006D696E00C6
:107C2000616C410072652000796F750020737500EA
:107C300072653F002043460047313A00204346002A
:107C400047323A00285C2D002F5F5C002D29280068
:107C50005C5F2F002D295300656C65006374200064
:107C60006F757400707574002074790070653A0047
:107C70000D0A2000312E20004F7065006E20640038
:107C8000726169006E202800483D4800692D5A0045
:107C90002C204C003D474E0044290D000A203200A4
:107CA0002E204E006F726D00616C200028483D0050
:107CB000332E3300562C20004C3D47004E44290003
:107CC00052325700202873007064200068697A00DF
:107CD000293D2800202030002E4D610063726F0086
:107CE000206D65006E750D000A2031002E4953008D
:107CF0004F37380031362D003320410054520D00EB
:107D00000A2032002E4953004F37380031362D00FB
:107D1000332070006172730065206F006E6C790013
:107D200049534F002037380031362D0033204100B1
:107D3000545220002852450053455400206F6E00D5
:107D400020435300290D0A0052455300455420009A
:107D500048494700482C2000434C4F00434B20002B
:107D6000544943004B2C20005245530045542000F9
:107D70004C4F570049534F002037380031362D0003
:107D80003320720065706C007920280075736500DF
:107D90007320630075727200656E7400204C53008E
:107DA0004220730065747400696E6700293A2000F0
:107DB00050726F00746F63006F6C3A00207365003F
:107DC000726961006C3320007769720065322000AF
:107DD000776972006552460055756E006B6E6F00D4
:107DE000776E5200656164002074790070653A0016
:107DF00020746F0020656E00647661007269610016
:107E0000626C6500206C65006E67740068446100F8
:107E100074612000756E690074733A00206E6F0003
:107E200020696E0064696300617469006F6E4400CC
:107E30006174610020756E00697420006C656E00CD
:107E4000677468002028620069747300293A200072
:107E500043532000454E4100424C450044435300EB
:107E600020444900534142004C45440052335700DE
:107E7000202873007064200063736C002068690020
:107E80007A293D00282029000D0A44006973630007
:107E90006F6E6E006563740020616E00792064006F
:107EA00065766900636573000D0A43006F6E6E00AE
:107EB000656374002028560070752000746F2000E0
:107EC0002B355600292061006E64200028414400B3
:107ED000432074006F202B00332E330056294300BB
:107EE00074726C00415558004D4F440045204C00C1
:107EF00045445000554C4C0055502000485055000A
:107F00004C4C550050204800565245004741440013
:107F1000432061006E64200073757000706C7900FE
:107F200035565600505533002E3356004144430019
:107F3000427573002068690067684200757320000D
:107F400048692D005A2030004275730020486900AE
:107F50002D5A2000314D4F0044452000616E6400D1
:107F600020565200454720004C45440073207300C2
:107F7000686F75006C642000626520006F6E2100E0
:107F8000466F75006E64200020657200726F72008B
:107F9000732E4D004F534900434C4B004D49530045
:107FA0004F435300204F4B0020464100494C5300A3
:107FB000657420007370650065643A000D0A200046
:107FC000312E200033304B00487A0D000A20320059
:107FD0002E20310032354B00487A0D000A20330044
:107FE0002E20320035304B00487A0D000A20340034
:107FF0002E2031004D487A00436C6F00636B2000E7
:10800000706F6C006172690074793A000D0A20008B
:10801000312E200049646C0065206C006F772000D1
:108020002A646500666175006C740D000A203200D8
:108030002E204900646C65002068690067684F0065
:108040007574700075742000636C6F00636B2000A2
:1080500065646700653A0D000A2031002E20490052
:10806000646C650020746F002061630074697600A1
:10807000650D0A0020322E002041630074697600ED
:10808000652074006F206900646C6500202A64001C
:1080900065666100756C7400496E7000757420002F
:1080A00073616D00706C650020706800617365001D
:1080B0003A0D0A0020312E00204D690064646C00E6
:1080C00065202A006465660061756C00740D0A0005
:1080D00020322E0020456E006453500049202800B5
:1080E0007370640020636B00702073006B65200068
:1080F000736D7000206373006C206800697A29003A
:108100003D28200020302E004D616300726F20005A
:108110006D656E00750D0A0020312E00536E6900EA
:1081200066662000435320006C6F77000D0A200024
:10813000322E53006E696600662061006C6C200070
:108140007472610066666900632D7000202D660000
:10815000202A42007974650073206400726F7000F9
:10816000706564002A464100494C4500442C2000BB
:108170004E4F20004441540041446100746120008E
:1081800062697400732061006E6420007061720087
:10819000697479003A0D0A0020312E0020382C0035
:1081A000204E4F004E4520002A6465006661750030
:1081B0006C7420000D0A2000322E2000382C200084
:1081C000455645004E200D000A2033002E20380071
:1081D0002C204F00444420000D0A2000342E2000A3
:1081E000392C20004E4F4E00455374006F70200014
:1081F00062697400733A0D000A2031002E203100AC
:10820000202A640065666100756C74000D0A200008
:10821000322E2000325265006365690076652000C9
:10822000706F6C006172690074793A000D0A200069
:10823000312E200049646C0065203100202A640042
:1082400065666100756C74000D0A2000322E2000F6
:1082500049646C00652030005541520054202800CC
:1082600073706400206272006720640062702000F6
:108270007362200072787000206869007A293D00DE
:1082800028202000302E4D00616372006F206D00A9
:10829000656E75000D0A2000312E540072616E006B
:1082A0007370610072656E00742062007269640010
:1082B00067650D000A2032002E204C0069766500AB
:1082C000206D6F006E6974006F720D000A2033001C
:1082D0002E42720069646700652077006974680047
:1082E00020666C006F772000636F6E0074726F0001
:1082F0006C55410052542000627269006467650049
:108300005265730065742000746F20006578690001
:1083100074526100772055004152540020696E006C
:10832000707574005541520054204C004956450068
:108330002044490053504C0041592C00207D20001E
:10834000544F200053544F00504C490056452000D4
:1083500044495300504C410059205300544F5000A1
:1083600050454400574152004E494E00473A2000C4
:1083700070696E0073206E006F7420006F7065006E
:108380006E206400726169006E20280048695A00FE
:108390002920520045564900443A0D000A496E0012
:1083A00076616C006964200063686F006963650032
:1083B0002C2074007279200061676100696E6D0085
:1083C00073525300204C4F00572C2000434F4D0058
:1083D0004D414E0044204D004F4445005253200073
:1083E00048494700482C20004441540041204D009A
:1083F0004F444500416464007265730073206F0050
:108400006620500043463800353734003F5468003A
:10841000697320006D6F64006520720065717500DE
:1084200069726500732061006E20610064617000F4
:10843000746572004C4344002074790070653A0002
:108440000D0A2000312E2000484434003437380013
:1084500030202800757369006E6720005043460085
:1084600038353700342049004F20650078706100AE
:108470006E64650072294C00434420002874790022
:10848000702061006464720029203D0020282000D3
:1084900020302E004D616300726F20006D656E000C
:1084A000750D0A0020312E004C4344002052650017
:1084B000736574000D0A2000322E49006E69740045
:1084C000204C4300440D0A0020332E00436C65000D
:1084D000617220004C4344000D0A2000342E4300FA
:1084E000757273006F722000706F73006974690099
:1084F0006F6E200065783A002834290020300D0086
:108500000A2036002E5772006974650020746500D9
:10851000737420006E756D006265720073206500D3
:10852000783A28003629200038300D000A2037001C
:108530002E57720069746500207465007374200002
:108540006368610072616300746572007320650086
:10855000783A2800372920003830440069737000C9
:108560006C617900206C69006E6573003A0D0A0039
:1085700020312E00203120000D0A2000322E200054
:108580004D756C00746970006C6549004E4954006B
:10859000434C450041524300555253004F52200076
:1085A000534554004E6F200041434B002C20630084
:1085B000686563006B20610064617000746572001F
:1085C000434C4B00094D4F005349090043530900E8
:1085D0004D4953004F5069006E737400617465001B
:1085E000733A47004E440900332E330056093500D4
:1085F0002E305600094144004309560050550900E9
:108600004155580009500900500950000949090016
:1086100049092D00094F570044092D00092D2D004F
:108620000954780044092D0009527800445343004E
:108630004C095300444109002D092D0050474300C7
:108640000950470044092D00092D31002E28420011
:1086500052290900322E28005244290009332E00E5
:10866000284F5200290934002E28590057290900A3
:10867000352E2800474E290009362E0028424C008E
:10868000290937002E28500055290900382E2800C6
:108690004752290009392E00285754002909300073
:1086A0002E2842006C6B2900474E440009474E00BB
:1086B0004409410044430900352E30005609330077
:1086C0002E335600095650005509410055580900EF
:1086D000657865006375740065203A0020205400B9
:1086E000494D45004F55540020302E00204D61006B
:1086F00063726F00206D65006E750D000A203100F9
:108700002E204C006976650020696E00707574003B
:10871000206D6F006E6974006F7249006E70750095
:1087200074206D006F6E6900746F7200202A7300F0
:1087300074617200746269007420650072726F0067
:1087400072202A00706172006974790020657200DD
:10875000726F7200202A7300746F70006269740077
:1087600020657200726F7200204E4F004E4520004F
:10877000554E4B004E4F57004E20450052524F0071
:108780005220610075746F0072616E006765200091
:108790002B4D48007A292B006B487A002952610042
:1087A00077207600616C7500652066006F7220008E
:1087B0004252470020284D00494449003D313200D3
:1087C0003729570041524E00494E47003A20500089
:1087D0006F73730069626C006520620075666600E5
:1087E00065726F0076657200666C6F0077416E008F
:1087F00079206B0065792000746F2000657869002E
:10880000745370006163650020746F0020636F0013
:108810006E7469006E7565004E756D00626572005C
:10882000206F660020626900747320007265610029
:10883000642F770072697400653A200043533A0050
:108840000D0A2000312E200043530D000A20320073
:108850002E202F00435320002A64650066617500B6
:108860006C7450006F73690074696F006E2069004A
:108870006E20640065677200656573005365720061
:10888000766F2000616374006976650047656E004D
:10889000657261006C0909000909090050726F00D6
:1088A000746F63006F6C2000696E74006572610004
:1088B000637469006F6E2D002D2D2D002D2D2D0060
:1088C0002D2D2D002D2D2D002D2D2D002D2D2D008C
:1088D0002D2D2D002D2D2D002D2D2D002D2D2D007C
:1088E0002D2D2D002D2D2D002D2D2D002D2D2D006C
:1088F0002D2D2D002D2D2D002D2D2D002D2D2D005C
:108900002D2D2D002D2D2D002D2D2D002D2D2D004B
:108910002D2D2D002D2D2D002D2D3F0009546800EB
:108920006973200068656C0070090900092830002F
:1089300029094C0069737400206375007272650028
:108940006E7420006D616300726F73003D582F00DC
:108950007C580900436F6E007665720074732000C6
:10896000582F720065766500727365002058090003
:108970000928780029094D00616372006F20780092
:108980007E095300656C6600746573007409090004
:10899000095B090053746100727423000952650079
:1089A0007365740009090900095D090053746F00BB
:1089B000702409004A756D00702074006F206200F9
:1089C0006F6F74006C6F61006465720009097B0051
:1089D0000953740061727400207769007468200084
:1089E0007265610064262F0025094400656C6100F2
:1089F00079203100207573002F6D7300090909007B
:108A00007D095300746F7000612F41002F400900F1
:108A10004155580050494E0020286C006F772F00B8
:108A200048492F00524541004429090009226100AC
:108A300062632200095365006E6420007374720043
:108A4000696E6700620953006574200062617500F9
:108A500064726100746509000909310032336300F2
:108A60002F43090041555800206173007369670066
:108A70006E6D65006E74200028617500782F4300CC
:108A8000532909000930780031323300642F440043
:108A9000094D650061737500726520004144430013
:108AA00020286F006E6365002F434F004E542E0048
:108AB000290930006231310030095300656E6400CD
:108AC000207661006C75650066094D006561730074
:108AD000757265002066720065717500656E6300D1
:108AE000790909007209520065616400672F53001B
:108AF000094765006E65720061746500205057007B
:108B00004D2F5300657276006F0909002F0943004D
:108B10004C4B20006869680009436F006D6D61006F
:108B20006E646800697374006F7279000909090046
:108B30005C0943004C4B20006C6F690009566500CE
:108B4000727369006F6E69006E666F002F73740038
:108B50006174750073696E00666F0900095E090033
:108B6000434C4B0020746900636B6C002F4C090070
:108B7000426974006F72640065722000286D730092
:108B8000622F4C005342290009092D00094441007D
:108B900054206800696D0900436861006E676500D4
:108BA000206D6F006465090009095F0009444100F8
:108BB00054206C006F6F090053657400206F7500BE
:108BC00074707500742074007970650009090900DB
:108BD0002E094400415420007265610064702F002A
:108BE00050095000756C6C00757020007265730040
:108BF000697374006F72730020286F0066662F001F
:108C00004F4E290009210900426974002072650055
:108C10006164730009536300726970007420650019
:108C20006E6769006E65090009093A00095265001E
:108C300070656100742065002E672E0020723A0076
:108C400031307600095368006F772000766F6C0032
:108C500074732F00737461007465730009093B001D
:108C60000942690074732000746F2000726561000E
:108C7000642F770072697400652065002E672E00EE
:108C80002030780035353B0032772F0057095000EF
:108C900053552000286F6600662F4F004E290900AB
:108CA000093C78003E2F3C00783D20003E2F3C00E0
:108CB000303E090055736500726D610063726F008C
:108CC00020782F006173730069676E0020782F0091
:108CD0006C697300742061006C6C00000000FA0085
:108CE000808B280096550200000000000080FA00EA
:108CF000000006000000FA000040EB00CC6A020011
:108D0000000000000040EB00CC6A02000000000000
:108D10000040EB00CC6A0200000000000040EB00C5
:108D2000CC6A0200000000000000EB00086A0200AC
:108D3000000000000000EB00086A020000000000D4
:108D40000000EB00086A0200000000000080FA004A
:108D5000000006000C00FA00A09C200010407800E3
:108D60000040A000A19C200080487800A09C20002A
:108D7000104078000030A100A19C200080487800BD
:108D800011C0B300809B20000148780081C0B3006F
:108D9000909B20000148780021C0B300B0BA2000A9
:108DA0000148780080C0EB0020C0B300A868020032
:108DB00000000000C922A900C902A900C8E2A80059
:108DC00010C0B300386B020000000000C3FF0700B2
:108DD0000000370022C2BF00614060000004E000D4
:108DE000FCFF32003011800080407800F0BA200093
:108DF00001487800F0BA2000104078000080FB00A5
:108E00004400DE0080407800E0BA2000014878008D
:108E1000E0BA2000104078000080FB003007980086
:108E20003E009000E30F500017013200BE0090009A
:108E3000E38F50000A003C003E019000E10F51001A
:108E4000A5003200BE019000E18F5100FB003C0004
:108E50003E0090000000E00012003200E8023700FF
:108E6000BE009000E68F5000910232003E0190005B
:108E7000E60F510004003C00BE019000E48F510059
:108E800083023200DE0237003E009000E80F5000FF
:108E90009E023200BE009000EA8F50003401320082
:108EA000D7023700F0BA2000104078000080FB00A5
:108EB0006101B9004207980053079800D0002000D4
:108EC000010020004E019000DE019000800F510053
:108ED000818F59007C003E004E009000DE00900023
:108EE00000600100CA0237000C0037000D00370097
:108EF00012003700170037001D003700230037002D
:108F000044003700480037004C003700520037005B
:108F1000580037005E003700640037006FFF07001D
:108F2000ACFF3700366902000000000010C0B3003B
:108F3000F259020000000000A6FF37007669020027
:108F40000000000010C0B300F25902000000000051
:108F5000A0FF37000040EB00386B0200000000006B
:108F600010C0B300F25902000000000099FF370062
:108F700010C0B300386B02000000000010C0B30046
:108F8000F25902000000000092FF3700B0BA200042
:108F900010407800E24F500006003A005C6A020080
:108FA0000000000080407800D0BA2000014878001E
:108FB00006003700F00F2000966902000000000054
:108FC00080407800D0BA200001487800A09C2000A2
:108FD00010407800684060000004E00008003200A3
:108FE000D0BA2000104078000080FB00467E0200CE
:108FF0000000000080407800D0BA200001487800CE
:10900000D0BA200010407800F259020000000000A1
:1090100070FF3700AA6A020000000000F259020047
:10902000000000006BFF37004A6B020000000000E8
:10903000F25902000000000066FF370010C0B300C4
:10904000EE6A02000000000010C0B300F2590200F6
:10905000000000005FFF37000040EB00266B0200BD
:109060000000000010C0B300F25902000000000030
:1090700058FF370010C0B300266B0200000000004C
:1090800010C0B300F25902000000000051FF370089
:109090000040EB00146B02000000000010C0B300A1
:1090A000F2590200000000004AFF370010C0B30070
:1090B000146B02000000000010C0B300F25902005F
:1090C0000000000043FF37000040EB00F2590200AF
:1090D000000000003FFF3700F0BA20009040780009
:1090E000F0C0B30080C06000F0BA200001487800F2
:1090F000F0BA2000104078008040E800F0BA20006C
:109100000148780010C0B300F259020000000000CE
:109110008040EB00D0BA20000148780040003700C2
:1091200022C2BF00614060000004E000FCFF32008A
:109130003011800080407800C0BA200001487800DB
:10914000A09C200010407800684060000004E0000F
:1091500008003200C0BA2000104078000080FB00F8
:10916000467E02000000000080407800C0BA200067
:1091700001487800B0BA200010407800E24F50005B
:1091800009003A00C0BA2000104078000080FB00BF
:10919000086A02000000000010C0B300F25902008B
:1091A0000000000019003700C0BA2000104078000D
:1091B0000080FB00966902000000000080407800FB
:1091C000C0BA200001487800A09C20001040780020
:1091D000684060000004E00008003200C0BA2000CF
:1091E000104078000080FB00467E02000000000076
:1091F00080407800C0BA200001487800C0BA200042
:1092000010407800F259020000000000D0BA20009F
:10921000104078008040E800D0BA20000148780073
:10922000D0BA200090407800F0BA200010407800BA
:1092300080CF5000BAFF3900E6FE3700F0BA2000B8
:1092400090407800F0C0B30080C06000F0BA200009
:1092500001487800F0BA2000104078008040E80013
:10926000F0BA200001487800F0BA200010407800E1
:10927000EE6A02000000000010C0B300F2590200C4
:1092800000000000D3FE3700F0BA200090407800C4
:10929000F0C0B30080C06000F0BA20000148780040
:1092A000F0BA2000104078008040E800F0BA2000BA
:1092B0000148780010C0B300F2590200000000001D
:1092C00022C2BF00614060000004E000FCFF3200E9
:1092D0003011800080407800E0BA2000014878001A
:1092E0008040EB00D0BA200001487800160037001B
:1092F000E0BA2000104078000004E00004003D00C7
:1093000010C0B300CC6A0200000000000300370068
:109310000040EB00CC6A020000000000E0BA200030
:10932000104078000040400080407800E0BA200003
:1093300001487800D0BA2000104078008040E80052
:10934000D0BA200001487800D0BA200090407800C0
:10935000F0BA20001040780080CF5000E4FF3900C0
:1093600010C0B300F25902000000000099FE37005F
:10937000F0BA2000104078000080FB002007980021
:10938000400A2000AE009000808F5000150032008F
:10939000500A20002E019000800F5100C5003200BD
:1093A000000A2000AE019000808F510001003200C1
:1093B0003301370022C2BF00614060000004E000BA
:1093C000FCFF32003011800080407800A0BA2000FD
:1093D0000148780010C0B300F259020000000000FC
:1093E0007CFE3700A0BA2000104078000080FB000F
:1093F000100798001E009000E10F5000040032009A
:109400009E009000E28F50003B003200A500370024
:1094100022C2BF00614060000004E000FCFF320097
:1094200030118000405D8800405D80006300B9001D
:10943000405D88000000EB00305D88000C003700C4
:1094400022C2BF00614060000004E000FCFF320067
:1094500071408000305D80008080400030118000CD
:1094600080487800305D80000000E800305D8800B2
:10947000315D8000405D8000808F5000F0FF39003A
:109480000000EB00305D8800130037007140800061
:10949000305D8000008040000080E80010417800CE
:1094A00071408000305D8000008040000000E800D6
:1094B0009041780071408000305D80000080400065
:1094C000104078008340780053010700305D800031
:1094D00063004000305D8800315D8000405D8000A9
:1094E000808F5000E9FF390010C0B300F25902002C
:1094F0000000000037FE370022C2BF00614060005C
:109500000004E000FCFF320030118000405D880064
:10951000405D80004200DD00405D88000000EB00FF
:10952000305D88000C00370022C2BF00614060003F
:109530000004E000FCFF320071408000305D8000DC
:10954000808040003011800080487800305D8000CD
:109550000000E800305D8800315D8000405D8000E3
:10956000808F5000F0FF39000000EB00305D880074
:10957000440037000040EB00CC6A0200000000000D
:109580000040EB00CC6A0200000000000040EB004D
:10959000CC6A0200000000000040EB00CC6A020030
:1095A0000000000071408000305D800000804000BD
:1095B000104078000080FB00086A020000000000F4
:1095C00071408000305D8000008040000000E800B5
:1095D000104078000080FB00086A020000000000D4
:1095E00071408000305D8000008040000080E80015
:1095F000104078000080FB00086A020000000000B4
:1096000071408000305D80000080400063014000B8
:1096100071408000305D80000080400063004000A9
:10962000104078006F406000004978008040EB00F7
:10963000D0BA20000148780006003700ADFD0700D1
:10964000D0BA2000104078008040E800D0BA200056
:109650000148780071408000305D8000008040004B
:109660006300400090407800D0BA2000104078009D
:1096700080CF5000F1FF3E00305D8000640040006C
:10968000305D8800315D8000405D8000808F50003B
:10969000B8FF390010C0B300F2590200000000000A
:1096A000CCFD37000040EB00F25902000000000042
:1096B000C8FD3700A0BA2000104078000080FB00F1
:1096C000000F78001E017800E10F51000400320005
:1096D0009E017800E28F510045003200BDFD370049
:1096E00022C2BF00614060000004E000FCFF3200C5
:1096F00030118000405D880022C2BF0061406000E0
:109700000004E000FCFF320030118000804078004F
:10971000E0BA2000014878000000EB00305D8800CE
:109720002E003700E0BA200090407800C0BA200038
:10973000014878008040EB00D0BA20000148780052
:1097400019003700C0BA2000104078000080FB00EC
:10975000610060000004E0000400320010C0B300AB
:10976000CC6A020000000000030037000040EB005C
:10977000CC6A020000000000C0BA2000104078004F
:109780000080FB000000D10080407800C0BA2000BB
:1097900001487800D0BA2000104078008040E800EE
:1097A000D0BA200001487800D0BA200010407800DC
:1097B000E34F5000E3FF36005C6A02000000000047
:1097C0005C6A020000000000F25902000000000084
:1097D000305D80000000E800305D8800315D800071
:1097E000405D8000808F5000CEFF390079FD37004A
:1097F00022C2BF00614060000004E000FCFF3200B4
:1098000030118000405D88000000EB00305D880072
:109810001600370022C0B30060B92000A10B200061
:10982000B7000700EA00070022C0B30060BB2D00AC
:10983000A10B2000B200070022C0B300603D2D0044
:10984000A10B2000AE000700E100070022C0B3001A
:1098500060BB2000A10B2000A9000700DC0007006E
:10986000305D80000000E800305D8800315D8000E0
:10987000405D8000808F5000E6FF390055FD3700C5
:109880000040EB00F25902000000000051FD3700DB
:10989000F0BA2000104078000883020000000000A9
:1098A00010C0B300F25902000000000049FD37006B
:1098B000F0BA20009040780030C0B30080C0600053
:1098C000F0BA200001487800F0BA200090407800FB
:1098D000809B200001487800809B20009040780009
:1098E000B0BA200010407800A86802000000000014
:1098F00010C0B300386B02000000000010C0B300BD
:10990000F25902000000000032FD3700A09C200048
:10991000104078000040A100A19C20008048780001
:10992000F0BA2000104078000080FB004300DE0009
:109930000000A200610060000004E00005003200A9
:10994000A09C2000104078000040A000A19C2000B6
:109950008048780021C0B300B0BA200001487800E8
:10996000F0BA2000104078000080FB004200DE00CA
:10997000610060000004E0000300320031C0B30069
:10998000B0BA200001487800A09C20001040780068
:109990000030A100A19C200080487800F0BA20008F
:1099A000104078000080FB000000D10061006000E2
:1099B0000004E00005003200A09C20001040780068
:1099C0000030A000A19C200080487800809B2000EF
:1099D00090407800B0BA200010407800A8680200DB
:1099E0000000000010C0B300386B0200000000004F
:1099F00010C0B300F259020000000000F5FC37006F
:109A00000040EB00F259020000000000F1FC3700BA
:109A10000080FA00000006000600FA0020479800C7
:109A200031479800424798002E4090000080FB008C
:109A30004600DE00004F78000040EB001047980021
:109A4000220037001E409000E34F50000C003A0007
:109A50001E04E0000A00320010C0B300266B0200B2
:109A6000000000001E80FB00E47D020000000000FA
:109A70000040EB00266B02000000000010003700E1
:109A80002E4090000080FB00610060000004E000B8
:109A90000400320010C0B300CC6A020000000000D5
:109AA000030037000040EB00CC6A02000000000019
:109AB0002E4090000080FB000000D100204798005D
:109AC0001E4090000040E800104798001E409000A3
:109AD000E34F5000DBFF36003E4090000080FB006B
:109AE000086A0200000000004E4090000080FB0069
:109AF000086A0200000000000080FA000000060072
:109B00000800FA00100798002107980062479800A3
:109B10000040EB00CC6A0200000000000040EB00B7
:109B2000CC6A0200000000000040EB00CC6A02009A
:109B3000000000000040EB00CC6A020000000000C2
:109B40001E009000467E020000000000086A02002D
:109B5000000000001E009000AE0090004809DD00EB
:109B60004800DE0000007100C808DE00467E0200EA
:109B700000000000086A0200000000001E009000C3
:109B8000AE0090004008DE0001002000467E02008A
:109B900000000000086A0200000000006E40900013
:109BA0006F406000604798000040EB00004F780075
:109BB000020037004FFC07001E4FE8006E40900087
:109BC0009E4F1000FBFF39000080FA0000000600E5
:109BD0000000FA0010C0B300CC6A020000000000D0
:109BE0000040EB00CC6A0200000000000040EB00E7
:109BF000CC6A0200000000000040EB00CC6A0200CA
:109C0000000000000000EB00086A020000000000F5
:109C10005C6A020000000000F2590200000000002F
:109C20005C6A020000000000F2590200000000001F
:109C300030FC07002FFC07000080FA00000006003F
:109C40000200FA00D04E80000000E0001200320056
:109C500000C2B300F25902000000000031002000F1
:109C600010442000288002000000000000C2B30061
:109C7000F259020000000000C04E80000000E00029
:109C800003003A000040EB00CC6A02000000000034
:109C90000000EB00D04E8800C04E80000000E000C5
:109CA00003003A005C6A020000000000004F7800E8
:109CB00010002000D04E88001E80FB000080FA00BB
:109CC000000006000400FA00000F7800D04E80006B
:109CD0000000E0001200320000C2B300F25902009E
:109CE0000000000031002000104420002880020005
:109CF0000000000000C2B300F259020000000000A2
:109D0000C04E80000000E00003003A000040EB007D
:109D1000CC6A0200000000000000EB00D04E88007A
:109D2000C04E80000000E00007003A001E007800EE
:109D3000086A020000000000AA6A02000000000099
:109D40000080FB00000F780000C2B300F25902004F
:109D5000000000001E00E00007003A003100200073
:109D60001044200028800200000000000030200085
:109D700010079800060037004100200040442000F2
:109D8000288002000000000000102000100798004A
:109D90001E0090000080FA00000006000000FA009B
:109DA000D04E80000000E0000F0032004100200093
:109DB0004044200028800200000000006089280044
:109DC000C255020000000000C04E80000000E0000C
:109DD00003003A0010C0B300CC6A0200000000008B
:109DE0000000EB00D04E8800C04E80000000E00074
:109DF0000F003A0036690200000000000000E00099
:109E00000B00320091002000A023200028800200D7
:109E100000000000510120003024200028800200B2
:109E20000000000060892800C25502000000000008
:109E3000D100200080442000B28002000000000019
:109E40000080FA00000006000000FA00D04E8000FA
:109E50000000E0000F0032004100200040442000DC
:109E6000288002000000000060892800C25502001E
:109E700000000000C04E80000000E00003003A0037
:109E800010C0B300CC6A0200000000000000EB002C
:109E9000D04E8800C04E80000000E00002003A0072
:109EA0007669020000000000C1002000504520003B
:109EB000B2800200000000000080FA0000000600EE
:109EC0000000FA000101200020522000288002003A
:109ED000000000000040EB002E58020000000000CF
:109EE00000C2B300F259020000000000809B200075
:109EF000104078002E5802000000000000C2B3009D
:109F0000F25902000000000070892800C2550200CA
:109F1000000000000080FA00000006000400FA00C3
:109F20000000EB00100798000000EB00C04E880016
:109F30006A1F0200000000009C1B020000000000DD
:109F4000000F78001E00E0000900340040002000EF
:109F50009E0F100006003C001E0078000040E90043
:109F600080407800809B2000014878000200370084
:109F70000000EB00000F78001E00E0002D003A000A
:109F80000000EB00905788000000EB00C04E8800F6
:109F9000C04E80000000E0000F003A00B103200036
:109FA00060482000B2800200000000008001EB0049
:109FB0004200200011002000100020009620020026
:109FC000000000000040E90080407800809B2000F5
:109FD0000148780022003700C14080003000230093
:109FE000808F500004003E0051032000104C2000E0
:109FF0002880020000000000C1022000604F200005
:10A0000028800200000000008001EB0032002000E8
:10A010001100200010002000962002000000000027
:10A020000040E90080407800809B200001487800D3
:10A030000B003700C140800030002300808F5000AB
:10A0400004003E0051032000104C20002880020034
:10A05000000000009AFF07000000EB00D04E8800CF
:10A06000A09C2000104078000040A000A19C20008F
:10A0700080487800C04E80000000E00009003A00EF
:10A08000C922A800C902A800CB02A900CB22A900BE
:10A09000809B20009040780020C0B300A868020098
:10A0A000000000000080FA00000006000000FA0036
:10A0B0000000EB00D04E8800C04E8000E10F500041
:10A0C00001003A0007E2A9000080FA000000060043
:10A0D0000600FA00100798001E0090002007980064
:10A0E0002E009000E10F50000C0032002E00900076
:10A0F000E10F5000040039002E009000E20F5000E4
:10A100006500320073003700510320002053200007
:10A110002880020000000000720037008040EB0041
:10A1200000302000566B020000000000E102200019
:10A1300070562000B280020000000000CBC2BF00B9
:10A14000614060000004E00004003200CBC2BF00A8
:10A15000624060000004E0000C003A009100200022
:10A16000A0232000288002000000000051012000F0
:10A1700030242000288002000000000060892800B0
:10A18000C255020000000000560037000000EB003E
:10A19000000F780039003700C04E80000000E0005A
:10A1A00009003A0036690200000000001E00780035
:10A1B000086A020000000000AA6A02000000000015
:10A1C0000080FB00100798001E0090000000E000D7
:10A1D00024003A001E0078003E7D020000000000CE
:10A1E00080C2B300F2590200000000001E00780097
:10A1F0000080D1003E7D0200000000001E007800BB
:10A200000000A200610060000004E00004003200D1
:10A210009089280096550200000000000B003700CE
:10A22000C04E80000000E00005003A005C6A0200B9
:10A230000000000010C0B300CC6A02000000000063
:10A24000C08928009655020000000000708928008F
:10A25000965502000000000000C2B300F25902004F
:10A2600000000000C04E80000000E00002003A0044
:10A2700076690200000000001E0FE800F00F2000C9
:10A280009E0F1000C4FF340060892800C2550200F0
:10A290000000000013003700C04E8000E10F5000A6
:10A2A00001003A0007E2A900710020005059200087
:10A2B000B280020000000000F1002000C01E21005A
:10A2C000B28002000000000010C0B3000E000700C2
:10A2D0000400370041022000C0202000B2800200AC
:10A2E000000000000080FA00000006000000FA00F4
:10A2F000B1002000C0092100B2800200000000006F
:10A300000080FA00000006000A00FA00004F9800E2
:10A310000040EB00204798000040EB0010479800F9
:10A320000040EB00004F78009A5A02000000000045
:10A33000C922A800C902A800CB02A900CB22A9000B
:10A3400062A0A80062C0A8008660A900CBC2BF00BE
:10A350000080FB000000D100614060006047980071
:10A360006E40900050479800CBC2BF006140600033
:10A37000604798006E40900030479800000037001A
:10A3800086C0BF00684060000004E00012003A0090
:10A3900023C2BF00624060000004E0000E003A00EB
:10A3A000E45A02000000000022C2BF0061406000C9
:10A3B0000004E000F2FF320030118000004F78000E
:10A3C00062A0A90062C0A9000E4890000004E0004D
:10A3D00061003A00630037008660A900CBC2BF006D
:10A3E0000080FB000000D1006140600060479800E1
:10A3F000CBC2BF0061406000404798002E409000F3
:10A400000004E0002E0032003E4090000004E00016
:10A410002B003A004E4090000004E000280032007B
:10A420001E409000E74F50000B003E001E40780099
:10A4300000404000004F78006E4090000004E000B3
:10A44000010032001E04A0001E4090000040E80001
:10A45000104798003B0037000E4890000004E000D1
:10A46000040032001E80FB00BA5802000000000009
:10A4700006003700C0C5B300AE5A0200000000005D
:10A480001E407800AE5A0200000000006E409000AE
:10A490000004E00004003200D0C2B300AE5A020053
:10A4A0000000000003003700B0C2B300AE5A020043
:10A4B000000000000040EB0010479800210037002A
:10A4C0003E4090000004E0001E0032004E4090002C
:10A4D0000004E0001B0032005E4090000004E00039
:10A4E0000B0032006E4090000004E00008003A00CB
:10A4F00010C0B300204798000040EB0010479800C0
:10A50000B0C5B300AE5A0200000000000D003700D5
:10A510005E4090000004E0000A003A006E409000A7
:10A520000004E000070032000040EB0020479800E4
:10A530000040EB0010479800D0C5B300AE5A0200AF
:10A54000000000006E409000504798004E40900080
:10A55000304798008AFF370060892800C255020002
:10A56000000000000080FA00000006000000FA0071
:10A57000F089280096550200000000000080FA00D3
:10A58000000006000A00FA00881F7800C922A8000F
:10A59000C902A800CB02A900CB22A900C8C2A90009
:10A5A000A09C2000104078000040A000A19C20004A
:10A5B00080487800A09C2000104078000030A10066
:10A5C000A19C20008048780080C0EB0020C0B30030
:10A5D000A868020000000000E4FF07000000370048
:10A5E00022C2BF00614060000004E000FCFF3200B6
:10A5F0003011800080407800609D20000148780084
:10A60000609D2000104078000080FB004400DE00C8
:10A6100080407800509D200001487800509D200027
:10A62000104078000080FB00400798004E0090002A
:10A63000E10F5000EB0032004E009000E10F50009F
:10A6400004003C004E0090000000E00008003200D2
:10A65000240137004E009000E40F50001901320031
:10A660004E009000E60F5000070132001D01370038
:10A67000609D2000104078000080FB0030079800AB
:10A680003E009000E40F5000330032003E00900086
:10A69000E40F500011003C003E009000E10F50001C
:10A6A0001F0032003E009000E10F500004003C000B
:10A6B0003E0090000000E0000E013200C5003700AF
:10A6C0003E009000E20F5000170032003E00900064
:10A6D000E30F50001A003200BE0037003E00900029
:10A6E000E70F5000280032003E009000E70F5000B6
:10A6F00004003C003E009000E60F50001B003200BA
:10A70000B40037003E009000E80F500025003200F2
:10A710003E009000EF0F5000A8003200AD0037005F
:10A7200092FF0700AEFF370036690200000000000C
:10A7300010C0B300F259020000000000A8FF37006B
:10A74000766902000000000010C0B300F259020058
:10A7500000000000A2FF37005C6A02000000000059
:10A76000F2590200000000009DFF37000040EB009E
:10A77000CC6A02000000000010C0B300F2590200D1
:10A780000000000096FF370010C0B300CC6A020042
:10A790000000000010C0B300F259020000000000E9
:10A7A0008FFF370022C2BF00614060000004E0005C
:10A7B000FCFF320030118000100798001E0090004E
:10A7C0004800DD001007980022C2BF006140600011
:10A7D0000004E000FCFF3200301180009E00900079
:10A7E000008070001007980022C2BF006140600026
:10A7F0000004E000FCFF320030118000000F780000
:10A800001E0078004800DD00000F780022C2BF0063
:10A81000614060000004E000FCFF32003011800065
:10A820001E0F70009E00900000002100808F5000DD
:10A8300003003E00000021009E0F100004003600BF
:10A840000040EB00F25902000000000064FF3700F6
:10A850000000EB00200798000C00370022C2BF0068
:10A86000614060000004E000FCFF320071408000A5
:10A870002E009000808040003011800080487800D9
:10A880002E0090000000E80020079800AE00900025
:10A890001E009000808F5000F0FF390036690200E2
:10A8A000000000000000EB00200798000E003700B9
:10A8B000714080002E009000008040001040780021
:10A8C0000080FB00086A020000000000AA6A020083
:10A8D00000000000E14F5000D9FF32002E00900030
:10A8E0000000E80020079800AE0090001E009000D5
:10A8F000808F5000EEFF39001E00E900100798001D
:10A900000000EB0020079800140037007140800021
:10A910002E009000008440005C6A020000000000ED
:10A92000004C7800AE0090001E009000808F500018
:10A93000040031000040EB00CC6A0200000000007F
:10A940000300370010C0B300CC6A02000000000012
:10A950002E0090000000E800200798002E009000D4
:10A960009E0F5000E9FF39007669020000000000E8
:10A9700010C0B300F2590200000000000000EB001C
:10A980002007980009003700714080002E009000D9
:10A990000080400010407800F259020000000000E2
:10A9A0002E0090000000E800200798002E00900084
:10A9B0009E0F5000F4FF390009FF37000040EB0004
:10A9C00051FE070010C0B300F25902000000000061
:10A9D00003FF37000040EB00F259020000000000C6
:10A9E000FFFE3700609D200090407800F0C0B3006B
:10A9F00080C06000609D200001487800609D2000BC
:10AA0000104078008040E800609D200001487800F8
:10AA100010C0B300F2590200000000008040EB00BB
:10AA2000409D2000014878001000370022C2BF007E
:10AA3000614060000004E000FCFF32003011800043
:10AA4000086A020000000000AA6A0200000000007C
:10AA5000F259020000000000409D200010407800E4
:10AA60008040E800409D200001487800409D200083
:10AA700090407800609D20001040780080CF50000A
:10AA8000EAFF3900D6FE3700609D20009040780034
:10AA900030C0B30080C06000609D20000148780095
:10AAA000609D20009040780020C0B300A86802009C
:10AAB0000000000010C0B300F259020000000000C6
:10AAC000C7FE3700609D2000104078000883020018
:10AAD0000000000010C0B300F259020000000000A6
:10AAE000BFFE37000040EB00F259020000000000FA
:10AAF000BBFE37004F0478000080FA00000006001B
:10AB00000200FA00000F78001E00E000030032008F
:10AB100010C3B300330207000200370000C3B300C4
:10AB2000300207000080FA00000006000600FA006C
:10AB300010079800020037001E4078002902070025
:10AB40001E009000104F78001E407800404798008B
:10AB50004E4090000004E0000200320010C0B3003C
:10AB6000404798004E4090009E0090008100E80011
:10AB7000110798000004E000EFFF3A000080FA009F
:10AB8000000006000600FA001007980002003700D7
:10AB90001E407800130207001E009000104F78003E
:10ABA0001E407800404798004E4090000004E000AE
:10ABB0000200320010C0B300404798004E409000A1
:10ABC0009E0090008100E800110798000004E0005A
:10ABD000EFFF3A00D0C0B30002020700A0C0B300EC
:10ABE000000207000080FA00000006000400FA00DE
:10ABF0002047980000C8B300004F780080872800E5
:10AC0000CAFF07000040EB00104798000F00370014
:10AC10002E4090001E4060000004E000030032005F
:10AC200010C3B300EF0107000200370000C3B300F8
:10AC3000EC0107001E80FB000000D100004F7800EF
:10AC40001E4090000040E800104798001E40900011
:10AC5000E74F5000EEFF36000080FA0000000600CB
:10AC60000E00FA0050079800610798000040EB00C2
:10AC7000004F780000102E00515F20003007980030
:10AC8000410798000040EB00104798003200370061
:10AC90003E019000CE0190005E009000EE0090001A
:10ACA000A00502000000000010079800210798008E
:10ACB0001E04E00005003A001E009000AE00900067
:10ACC000E00F5000E08F5800180032001E00900086
:10ACD0000043B000C30107009E0090003E009000BA
:10ACE000000AB8009E0090004E0090000088B90055
:10ACF0000501780000014100BE0090002E00900088
:10AD00000088B90000014100820278005E009000D6
:10AD1000EE00900004005000858058005007980015
:10AD20006107980010C0B300004F78003E0090000B
:10AD3000CE009000A200200003002000A005020029
:10AD40000000000030079800410798001E40900066
:10AD50000040E800104798001E409000E74F500068
:10AD6000CBFF36005E0090000043B0009D0107005D
:10AD70000080FA00000006000C00FA00400798006E
:10AD8000510798000000EB00100798000000EB004E
:10AD9000000F78006000B800200798003107980085
:10ADA0004E019000DE019000F0232400F10020000D
:10ADB000800F5100818F5900210036004E00900015
:10ADC000DE00900002242400F3002000A005020011
:10ADD0000000000020079800310798002E00900026
:10ADE0006F000700C0C2B3007E0107004E00900054
:10ADF000DE00900002242400F3002000C0050200C1
:10AE00000000000040079800510798004E01900094
:10AE1000DE019000703E200001002000800F5100F4
:10AE2000818F590002003E00B08728003FFF0700D5
:10AE3000100020001007980010002000000F78007C
:10AE40004E019000DE019000703E200001002000C5
:10AE5000800F5100818F5900320036004E00900063
:10AE6000DE009000823E200003002000A0050200CA
:10AE70000000000020079800310798002E01900084
:10AE8000BE0190004006200001002000800F51000C
:10AE9000818F5900030036002E009000400007000B
:10AEA000140037001E0090000000E0000F00320088
:10AEB0002E019000BE019000A000200001002000A3
:10AEC000800F5100818F59000300360000C3B3008A
:10AED00044010700020037000088280013FF070024
:10AEE0002E0090002E000700020037002E00900078
:10AEF0002B000700C0C2B3003A0107004E009000CB
:10AF0000DE009000823E200003002000C005020009
:10AF10000000000040079800510798001000200032
:10AF2000000F78004E019000DE01900040062000E6
:10AF300001002000800F5100818F5900030036006E
:10AF40004E00900016000700130037001E00E000BE
:10AF50000F0032004E019000DE019000A0002000A2
:10AF600001002000800F5100818F5900030036003E
:10AF700000C3B3001B01070002003700008828004F
:10AF8000EAFE07004E0090000500070002003700AF
:10AF90004E009000020007000080FA00000006004A
:10AFA0000800FA00300798000040EB00004F7800DE
:10AFB00000712200200798000040EB001047980025
:10AFC0001E0037003E0090002E0190001100090085
:10AFD0000280D800100798001E04E00003003A0029
:10AFE0001E0090000000E0000C0032001E009000E7
:10AFF0000043B000FB0007009E0090002E00900070
:10B000000088B900800078003E00900001005000E8
:10B010003007980010C0B300004F78002E00900059
:10B02000A2002000110009000280D800200798002B
:10B030001E4090000040E800104798001E4090001D
:10B04000E34F5000DFFF36003E0090000043B000A9
:10B05000E40007000080FA00000006000600FA0085
:10B06000404798000040EB00004F780040C6B30016
:10B07000304798000040EB00204798002000370040
:10B080004E4090008080FB003E4090000081FB001D
:10B09000110009008280D800104798001E04E000CB
:10B0A00003003A001E4090000004E0000B00320054
:10B0B0001E4090000043B000CA0007004E419000BF
:10B0C0009E4090003E4090000088B9000040510032
:10B0D0004047980010C0B300004F78003E409000F9
:10B0E0000080FB00A2002000110009000280D800AF
:10B0F000304798002E4090000040E800204798001C
:10B100002E409000E14F5000DDFF36004E40900091
:10B110000043B000B30007000080FA000000060002
:10B120000400FA0010079800308928007FFE07000D
:10B130001E0090004400DE006F0F60009E0078004B
:10B14000308828000080400010407800A5000700EB
:10B150001E0090006F0F60009E007800308828006D
:10B1600000804000104078009E0007000080FA0038
:10B17000000006000400FA001007980000C3B300A6
:10B18000F600070080C7B300F40007001E0090001F
:10B190004400DE006F0F60009E00780030882800B9
:10B1A0000080400010407800EC0007001E00900076
:10B1B0006F0F60009E0078003088280000804000FB
:10B1C00010407800E50007000080FA00000006004B
:10B1D0000400FA00100798003089280053FE070089
:10B1E0001E0090004C00DE006F0F60009E00780093
:10B1F0003088280000804000104078007900070067
:10B200001E0090004800DE006F0F60009E00780076
:10B21000308828000080400010407800710007004E
:10B220001E0090004400DE006F0F60009E0078005A
:10B230003088280000804000104078006900070036
:10B240001E0090006F0F60009E007800308828007C
:10B250000080400010407800620007000080FA0083
:10B26000000006000800FA00300798003E00900039
:10B27000CF80DE006403020000000000926C220018
:10B28000B3312400C2030200000000001007980040
:10B29000210798001E009000AE009000C605020035
:10B2A00000000000004F78001E4078006BFF070090
:10B2B000E0C2B3004B0007001E009000AE009000FB
:10B2C000C605020000000000CF80DE00640302001B
:10B2D000000000000001BE001E009000AE009000C3
:10B2E00046040200000000001007980021079800A3
:10B2F00002002000031224001E009000AE00900007
:10B3000002050200000000001007980021079800C5
:10B310001E009000AE009000C60502000000000074
:10B32000004F78001E4078004CFF07001E00900080
:10B33000AE009000C605020000000000CF80DE00D5
:10B3400064030200000000000001BE001E00900027
:10B35000AE009000460402000000000010079800B4
:10B360002107980002002000031224001E00900014
:10B37000AE009000020502000000000010079800D7
:10B38000210798001E009000AE009000C605020044
:10B3900000000000004F78001E4078002FFF0700DB
:10B3A0000080FA00000006000000FA0022C2BF0080
:10B3B000614060000080FB000080FA000000060091
:10B3C0000000FA0022C2BF00614060000004E000FB
:10B3D000FCFF3200301180000080FB000080FA008A
:10B3E000000006000200FA00004F7800D040800004
:10B3F00001102000010060000000E00006003A009B
:10B4000023C2BF00624060000004E000FCFF3A007D
:10B410001E00FB00201188000080FA0000000600DA
:10B420000200FA00004F78001E80FB0040118800E7
:10B430000080FA00000006000000FA0095C0BF007E
:10B44000704060000004E00010003A0051408000AD
:10B4500040408000808F50000C00320023C2BF00AB
:10B46000624060000004E000FCFF3A008580A90013
:10B470009580A8003140800040408000008040005E
:10B48000104078000080FB00201188000080FA0046
:10B4900000000600809FBE000000FA00014080000E
:10B4A000204080008080400030118000804878007B
:10B4B000204080000000E8002040880021408000FB
:10B4C00010408000808F500001003A009560A90074
:10B4D0008560A9000080FA004F00BE000040060011
:10B4E000809FBE000000FA00404080000000E8009D
:10B4F000404088004140800050408000808F5000D4
:10B5000002003A009580A900060037003140800013
:10B510004040800000804000104078000080FB0028
:10B52000201188008580A9000080FA004F00BE002D
:10B53000004006000000FA000000EB00C05C88003C
:10B5400010002000B05C8800D040800000A0A10066
:10B55000D04088000080FA00000006000200FA00D7
:10B56000004F7800B15C8000C05C8000808F50008C
:10B5700005003A00CA82A900D040800000A0A000C7
:10B58000D04088000E00370071408000B05C800021
:10B59000808040001E40780080487800B05C8000C9
:10B5A0000000E800B05C8800B15C80000000210071
:10B5B000808F500002003A000000EB00B05C880071
:10B5C0000080FA00000006000200FA00C05C800063
:10B5D000000FE800000021009E0F100002003A005A
:10B5E0000000EB00000F7800B05C80009E0F1000A0
:10B5F0000C00320023C2BF00624060000004E00083
:10B6000008003A001E007800C05C8800714080008D
:10B61000C05C800000804000104078000080FB008B
:10B62000201188000080FA00000006000200FA00E5
:10B6300000003700C05C8000000FE800000021001F
:10B640009E0F100002003A000000EB00000F78008F
:10B65000B05C80009E0F10000D00320023C2BF00BE
:10B66000624060000004E000F2FF3A001E00780033
:10B67000C05C880071408000C05C80000080400099
:10B68000104078000080FB0020118800E9FF37009F
:10B690000080FA00000006000800FA002007980069
:10B6A0003107980090018000100798002E0090004C
:10B6B000900188003E0090001080BA00C800DD00B4
:10B6C0003E0090001000BA00008F70001E00900035
:10B6D000900188001E0078000080FA00000006003B
:10B6E0000600FA000000EB00800888000000EB0074
:10B6F000F00888000000EB00E00C8800504F80004C
:10B700000000E00008003A00A16C200091407800A1
:10B7100000CEB30000C06000CAE6B7000000EB0036
:10B72000E04E88003D003700504F8000E30F50008E
:10B7300005003C00E0032000000F780010A1A800E5
:10B740001081A80015003700504F8000FE0F5000F8
:10B7500005003C00A00F2000000F780010A1A800F9
:10B760001081A9000D003700514F8000400F2000CC
:10B77000808F500005003C00007D2000000F780005
:10B7800010A1A9001081A8000400370000E82300E0
:10B79000000F780010A1A9001081A900504F80006F
:10B7A000000178001E007800110009000280D80016
:10B7B0000000E900200798002E0090006008880033
:10B7C000604F8000800078002E0090000088B90053
:10B7D00042062000110009000280D80010079800DE
:10B7E000A16C20009140780000CEB30000C0600042
:10B7F0006041B300CAE6B7001E009000D00C88007C
:10B800001E009000C00C880060002000E00C880042
:10B8100011E1A80020002000E04E88000080FA001E
:10B82000000006001200FA000000EB00800888000B
:10B830000000EB00F00888000000EB00E00C88003E
:10B84000E04E8000E20F500014003A00A16C20008E
:10B850009140780000CEB30000C06000CAE6B70097
:10B86000C1002000C02E2000B280020000000000B5
:10B870000000EB00E04E8800805780008000E80068
:10B88000F00F200080806000E09E200000804000DB
:10B89000104078000004E000AC0032000000EB0033
:10B8A00020079800805780008000E800F00F2000FB
:10B8B00000806000805788006A1F020000000000BE
:10B8C0009C1B020000000000400798006A1F020055
:10B8D000000000009C1B020000000000CF80DE0082
:10B8E0006403020000000000008FBE004E009000C4
:10B8F0000000E00007003200CE009000F0F92000C8
:10B90000808F500003003E002E0090000000E800F1
:10B91000200798006011B8001E00BE00BA030200A4
:10B92000000000000000E00001003C000B003700B8
:10B9300002002000832C24001E00BE00BE03020073
:10B94000000000000000E0000100350003003700A7
:10B950002E0090000000E800200798002E009000C4
:10B96000E20F5000110032000000EB0090578800F9
:10B9700011012000802F2000B28002000000000092
:10B9800011012000903020002880020000000000FB
:10B990008001EB0002FA20001100200020032000AB
:10B9A0009620020000000000400798004E00900022
:10B9B000E30F500005003E00E00320003007980030
:10B9C00010A1A8001081A800150037004E009000BB
:10B9D000FE0F500005003E00A00F20003007980029
:10B9E00010A1A8001081A9000D003700CE00900022
:10B9F000400F2000808F500005003E00007D200099
:10BA00003007980010A1A9001081A8000400370099
:10BA100000E823003007980010A1A9001081A900B8
:10BA20003E0090004E019000110009000280D800F5
:10BA30000000E900600798002E009000E20F50001F
:10BA40000E00320001012000703220002880020028
:10BA5000000000008001EB00320620008000EB00B7
:10BA6000200320009620020000000000CF80DE00AE
:10BA70006403020000000000008FBE0002002000EE
:10BA8000832C24001E00BE00C20302000000000040
:10BA9000008FBE006E009000CF80DE0064030200C5
:10BAA0000000000070079800010F98006E009000E1
:10BAB0000000E00008003D000200200003782400A0
:10BAC0007E0090008E0890004804020000000000F4
:10BAD00070079800010F98001E01BE007E009000C4
:10BAE0008E08900002050200000000006A050200B6
:10BAF0000000000050079800A16C200091407800E1
:10BB000000CEB30000C060006041B300CAE6B700D9
:10BB10005E009000D00C88005E009000C00C880091
:10BB200060002000E00C88006E0090006008880033
:10BB300011E1A800A100200070332000B2800200B3
:10BB40000000000020002000E04E88000080FA0085
:10BB5000000006000000FA00E04E8000E20F5000F6
:10BB600005003A00F101200010342000B2800200EC
:10BB7000000000003E003700F100200000362000E9
:10BB800028800200000000000000EB00F0088800A0
:10BB90000000EB0080088800C942A800616820000E
:10BBA0009140780000CEB30000C06000A040B30018
:10BBB00086E6B700A0032000800888002E0007005A
:10BBC000F04E8800014F8800F24E8000034F800045
:10BBD000F00F200001002000800F5100818F5900DC
:10BBE00009003600F04E8000014F8000C808DD00DB
:10BBF0000080FD00804078000040EB00F04E88009F
:10BC0000014F880009003700B1002000B019210061
:10BC10002880020000000000A000200080088800AA
:10BC200015000700F04E8800014F8800F04E80009C
:10BC3000014F8000BC56020000000000C08A2800AE
:10BC40009655020000000000008B2800C25502003B
:10BC50000000000086C6BF00F041B30086E6B700D2
:10BC60000000EB00F00888000000EB00800888006E
:10BC70000080FA00000006000000FA000080EB00DF
:10BC8000700888000080EB00600888000000EB006E
:10BC9000400888000000EB00300888000000EB003E
:10BCA000B00888000000EB00A00888008000200099
:10BCB000F0088800400F2000E008880000402200C3
:10BCC000D00888008780A9001FE1A80011E1A80022
:10BCD00087C0BF00704060000004E000FCFF32003D
:10BCE00011E1A9001FE1A90030088000404F880041
:10BCF00040088000304F8800304F80000100200055
:10BD0000104F8800214F8800104F8000214F800085
:10BD1000C000DD0000002000104F8800214F880087
:10BD2000404F80006101B800104F8000214F80001B
:10BD30000200400083804800104F8800214F880097
:10BD4000104F8000214F80000080FA0000000600A4
:10BD50000000FA00A09C20001040780063406000C2
:10BD60000004E00002003A00C942A80001003700C8
:10BD7000C8C2A800E1002000F036200028800200A0
:10BD8000000000000080FA00000006000000FA0039
:10BD9000A09C200010407800634060000004E00098
:10BDA00003003A00C942A900CB42A80002003700B4
:10BDB000C8C2A900CAC2A80081002000D037200054
:10BDC000B2800200000000000080FA0000000600BF
:10BDD0000000FA00A09C2000104078006340600042
:10BDE0000004E00003003A00C942A900CB42A900C8
:10BDF00002003700C8C2A900CAC2A9007100200011
:10BE000050382000B2800200000000000080FA00DC
:10BE1000000006000200FA00A09C200010407800FC
:10BE2000634060000004E00009003A00C942A80035
:10BE30000000000000000000CBC2BF000080FB003B
:10BE40004200DE0061406000004F780008003700CB
:10BE5000C8C2A8000000000000000000CAC2BF0065
:10BE60000080FB004600DE0061406000004F78006B
:10BE70001E80FB000080FA00000006000C00FA00A3
:10BE80000000EB00800888000000EB00F00888004C
:10BE90000000EB00E00C8800E04E8000E20F500054
:10BEA00014003A00A16C20009140780000CEB3004D
:10BEB00000C06000CAE6B700C1002000C02E20000C
:10BEC000B2800200000000000000EB00E04E88009D
:10BED000805780008000E800F00F20008080600024
:10BEE000E09E200000804000104078000004E00048
:10BEF00064003200805780008000E800F00F2000CE
:10BF000000806000805788006A1F02000000000067
:10BF10009C1B020000000000CF80DE0064030200D2
:10BF200000000000008FBE00905780000000E0007D
:10BF300008003A0002002000433324001E00BE0027
:10BF4000BA030200000000000000E00001003C0015
:10BF5000100037000000EB009057880031012000EE
:10BF600040242100B2800200000000008001EB00AC
:10BF7000420B20008000EB00A0052000962002006C
:10BF800000000000CF80DE0064030200000000001B
:10BF9000008FBE0010A1A8001081A800204E200034
:10BFA0003007980002002C00A35524001E00BE009C
:10BFB000C203020000000000008FBE003E0090009F
:10BFC000CF80DE00640302000000000040079800FC
:10BFD000510798003E0090000000E00008003D007E
:10BFE00002002000037824004E009000DE00900044
:10BFF0004804020000000000400798005107980024
:10C000001E01BE004E009000DE00900002050200FE
:10C0100000000000020020008327240048040200E2
:10C02000000000006A0502000000000020079800E0
:10C03000A16C20009140780000CEB30000C06000E9
:10C040006041B300CAE6B7002E009000D00C880013
:10C050002E009000C00C880060002000E00C8800DA
:10C060003E0090006008880011E1A800C100200097
:10C0700070252100B2800200000000002000200096
:10C08000E04E88000080FA00000006000000FA0080
:10C09000208B280096550200000000000080FA0066
:10C0A000000006000200FA00CA82A800F2000700A1
:10C0B000F6FF070000003700E60007008040780028
:10C0C00040BA20000148780040BA200010407800B3
:10C0D0000004E000D900350040BA2000104078008C
:10C0E0000004E00002003A00E8FF0700F2FF37001A
:10C0F00040BA200010407800E14F500004003A00A0
:10C10000DD000700DC000700E0FF0700EAFF370062
:10C1100040BA200010407800E24F500004003A007E
:10C12000D5000700D4000700D8FF0700E2FF370062
:10C1300040BA200010407800E34F500004003A005D
:10C14000CD000700CC000700D0FF0700DAFF370062
:10C1500040BA200010407800E44F500004003A003C
:10C16000C5000700C4000700C8FF0700D2FF370062
:10C1700040BA200010407800E54F500006003A0019
:10C18000BD000700AA46020000000000BA00070038
:10C19000BEFF0700C8FF370040BA200010407800FB
:10C1A000E64F500004003A00B3000700B200070059
:10C1B000B6FF0700C0FF370040BA200010407800EB
:10C1C000E74F500004003A00AB000700AA00070048
:10C1D000AEFF0700B8FF370040BA200010407800DB
:10C1E000EF4F50000A003A0010C0B300F2590200AD
:10C1F00000000000CA82A90023C2BF0061406000A5
:10C200000004E000FCFF32000000FE00AAFF37003F
:10C2100040BA200010407800F24F500035003A003C
:10C220000000EB00800888000000EB00F0088800A8
:10C230000000EB00E00C8800A16C20009140780029
:10C2400000CEB30000C060006041B300CAE6B70092
:10C25000800007000080FB00000F78001E007800BF
:10C260000000D100610060000004E0000100320025
:10C2700010A1A8009E007800618060000004E0002A
:10C28000010032001081A800720007000080FB004E
:10C290004800DD00000F78006E0007000080FB0002
:10C2A0001E0F70001E007800D00C88009E007800E1
:10C2B000C10C880060002000E00C880065000700C9
:10C2C0000080FB004800DD00000F780061000700DF
:10C2D0000080FB001E0F70001E00780060088800C0
:10C2E00011E1A80010C0B300F259020000000000E4
:10C2F00071FF370040BA200010407800F34F500023
:10C300000D003A000000EB00800888000000EB0000
:10C31000E00C8800A16C20009140780000CEB300B2
:10C3200000C06000CAE6B70010C0B300F2590200B6
:10C330000000000060FF370040BA20001040780085
:10C34000F44F50000E003A0021E3A800C0C0B30033
:10C35000867C020000000000000F780021E3A900A5
:10C360001E0078004800DE00F259020000000000C4
:10C370001E007800F2590200000000004EFF370056
:10C3800040BA200010407800F54F500018003A00E5
:10C3900021E3A800C0C0B300867C020000000000BA
:10C3A000000F780023C2BF00614060000004E0007D
:10C3B000FCFF32001E0078004800DE00F259020047
:10C3C000000000001E007800F2590200000000008A
:10C3D00022C2BF00614060000004E000EDFF3200B7
:10C3E00031118000010F780021E3A90032FF3700EE
:10C3F00040BA2000104078000080FB004500DE00BD
:10C400000080FB000000D100610060000004E0003B
:10C410000600320040BA2000104078001F000700DC
:10C42000F25902000000000023FF37000040EB003B
:10C43000F2590200000000001FFF370040BA200040
:10C4400010407800A5000700F2590200000000002B
:10C4500019FF37000000FA0022C2BF0061406000EF
:10C460000004E000FCFF3200301180000080FB007F
:10C470000080FA00000006000000FA0000C0EB0097
:10C48000060007000040EB0094000700C962A90005
:10C49000CB62A9000080FA00000006000400FA0048
:10C4A000204798000040EB00004F78002E4090009D
:10C4B0000080FB004400DE00610060000004E0003A
:10C4C0000200320010C0B300004F78009E40780098
:10C4D00061C06000614060004201DD00912C2000DD
:10C4E00091407800B0CFB30000C0600002407000FF
:10C4F000C9E2B7000040EB00004F78002E409000EA
:10C500000080FB004300DE00610060000004E000EA
:10C510000200320010C0B300004F78009E40780047
:10C5200061C060006140600000414000912C20002B
:10C5300091407800D0CFB30000C06000024070008E
:10C54000C9E2B7000040EB00004F78002E40900099
:10C550000080FB004200DE00610060000004E0009B
:10C560000200320010C0B300004F78009E407800F7
:10C5700061C0600061416000912C20009140780012
:10C58000E0CFB30000C0600002407000C9E2B70015
:10C590000040EB00004F78002E4090000080FB0030
:10C5A0000000D100610060000004E00002003200E1
:10C5B00010C0B300004F78009E40780061C060005A
:10C5C000C700DD00C8C2BF000074A10001407000B8
:10C5D000C8E2B7000040EB00004F78002E4090000A
:10C5E0000080FB00610060000004E00002003200F7
:10C5F00010C0B300004F78009E40780061C060001A
:10C60000614060004601DD00812C200091407800EF
:10C61000F0CBB30000C0600002407000C8E2B70079
:10C6200050002000107E020000000000AE4090008C
:10C6300000CEB30000C0600020479800CBC2BF000E
:10C64000644060000004E000030032002E409000CF
:10C650000044A00020479800CBC2BF0062406000A9
:10C660000004E000030032002E4090000034A000DF
:10C6700020479800CBC2BF00614060000004E0008A
:10C68000030032002E4090000024A00020479800B4
:10C69000CAC2BF0001C8B300014060000004E0004E
:10C6A000030032002E4090000014A00020479800A4
:10C6B000CAC2BF000044B2000004E0000300320020
:10C6C0002E4090000004A000204798002E409000CB
:10C6D0000080FB000080FA00000006000400FA0061
:10C6E000204798002E4090000080FB004600DE00AE
:10C6F000610060000004E00005003200C082A90073
:10C70000C282A800C8A2A900CAA2A80004003700DB
:10C71000C082A900C282A900C8A2A900CAA2A90019
:10C720000040EB00004F78002E4090000080FB009E
:10C730004400DE00610060000004E00002003200FE
:10C7400010C0B300004F78009E40780061C06000C8
:10C75000614060004201DD00B12C20009140780072
:10C76000B0CFB30000C0600002407000CBE2B70061
:10C770000040EB00004F78002E4090000080FB004E
:10C780004300DE00610060000004E00002003200AF
:10C7900010C0B300004F78009E40780061C0600078
:10C7A0006140600000414000B12C200091407800C1
:10C7B000D0CFB30000C0600002407000CBE2B700F1
:10C7C0000040EB00004F78002E4090000080FB00FE
:10C7D0004200DE00610060000004E0000200320060
:10C7E00010C0B300004F78009E40780061C0600028
:10C7F00061416000B12C200091407800E0CFB3008F
:10C8000000C0600002407000CBE2B7000040EB00C7
:10C81000004F78002E4090000080FB000000D10007
:10C82000610060000004E0000200320010C0B300AC
:10C83000004F78009E40780061C06000C700DD00B6
:10C84000CAC2BF000074A10001407000CAE2B70074
:10C850000040EB00004F78002E4090000080FB006D
:10C86000610060000004E0000200320010C0B3006C
:10C87000004F78009E40780061C060006140600019
:10C880004601DD00A12C200091407800F0CBB300E0
:10C8900000C0600002407000CAE2B70050002000F3
:10C8A000107E020000000000AE40900000CEB300F9
:10C8B00000C0600020479800CBC2BF006440600009
:10C8C0000004E000030032002E4090000044A0006D
:10C8D00020479800CBC2BF00624060000004E00027
:10C8E000030032002E4090000034A0002047980042
:10C8F000CBC2BF00614060000004E00003003200D2
:10C900002E4090000024A00020479800CAC2BF001B
:10C9100001C8B300014060000004E00003003200E1
:10C920002E4090000014A00020479800CAC2BF000B
:10C930000044B2000004E000030032002E409000EA
:10C940000004A000204798002E4090000080FB00CB
:10C950000080FA00000006000000FA00A09C200001
:10C96000104078000040A000A19C20008048780082
:10C97000960007000080FA00000006000000FA00A0
:10C980003C0107005300070010032100104078000D
:10C990000080FB000080FA00000006000400FA009E
:10C9A000100798001E00900071010700004F7800EA
:10C9B0001E04E00005003A00310020001044200071
:10C9C00028800200000000000C00370010C0B300F7
:10C9D0009E4F100005003A00410020004044200016
:10C9E00028800200000000000400370081002000C1
:10C9F000001221002880020000000000001020002A
:10CA00000080FA00000006000400FA00000F780021
:10CA10001E007800100798001E0090000000E00043
:10CA2000040032001E009000E10F500006003200AA
:10CA3000220037006102200080122100B280020033
:10CA40000000000021003700D1002000E014210088
:10CA5000B280020000000000F1002000C01E210092
:10CA6000B280020000000000020107000004E000A4
:10CA700008003A0010032100104078000080FB00FD
:10CA80003E7D02000000000000C2B300F259020027
:10CA90000000000022C2BF00614060000004E0000E
:10CAA000F1FF320030118000000F7800408D280027
:10CAB000C2550200000000000400370041022000BF
:10CAC000C0202000B2800200000000000080FA00B8
:10CAD000000006000400FA00004F78001E80FB00F2
:10CAE000100798009E009000E28F50001A0032005C
:10CAF0001E009000E20F500007003C009E009000D6
:10CB00000100E0002F0032001E009000E10F5000F5
:10CB10000C003200270037009E009000E48F500088
:10CB2000170032001E009000E40F50000F00350087
:10CB3000F00F20009E009000808F500018003200FF
:10CB40001C00370001012000B0152100B280020056
:10CB5000000000001B003700E1002000B01621009B
:10CB6000B28002000000000016003700F100200033
:10CB700090172100B2800200000000001100370071
:10CB800000C2B300F2590200000000008100200042
:10CB90000012210028800200000000000900370078
:10CBA0005100200080182100B28002000000000027
:10CBB00004003700E1002000D0182100B2800200FC
:10CBC000000000000080FA00000006000000FA00EB
:10CBD000C922A800C902A900CB02A900CB22A90042
:10CBE0000080FA00000006000400FA000040EB009C
:10CBF000410107000004E000030032002000200093
:10CC0000100798000E003700CBC2BF000080FB0069
:10CC10000000D10061406000004F780010C0B300F8
:10CC2000350107000004E00003003200200020006E
:10CC300010079800020037001E80FB0010079800C4
:10CC40001E0090000080FA00000006000600FA00B6
:10CC50000040EB00204798000040EB001047980090
:10CC6000CBC2BF000080FB000000D100E1406000AB
:10CC7000000321001040780061C16000E1CFB300E3
:10CC800001406000024070000103210080487800EC
:10CC90000003210010407800614060000004E000C3
:10CCA0000300320010002000200798006E003700BB
:10CCB00010C0B300100107000004E00003003200C0
:10CCC0004100200021079800670037000040EB007A
:10CCD00030479800190037001E4090000080FB008C
:10CCE0000000D10010479800BFFF0700004F7800F8
:10CCF00020C0B3009E4F100003003A004100200006
:10CD0000210798005800370010C0B3009E4F100054
:10CD100007003A009E40900000C8B30000C04000E9
:10CD2000104798002E4090000004A2002047980071
:10CD30003E4090000040E800304798003E409000A0
:10CD4000E74F5000E4FF3600100321009E409000A2
:10CD500001487800A4FF0700004F780020C0B3000E
:10CD60009E4F100003003A00410020002107980068
:10CD70003D0037001E407800E140600020032100A4
:10CD80001040780061C16000E1CFB3000140600055
:10CD90000240700021032100804878002003210018
:10CDA00010407800614060008080FB002E409000C1
:10CDB0000080FB00808F500008003A002003210013
:10CDC000104078000020A000210321008048780056
:10CDD00021002000210798002300370020032100B4
:10CDE000104078000020A100210321008048780035
:10CDF0007DFF0700004F780020C0B3009E4F100059
:10CE000003003A0041002000210798001600370077
:10CE10001E407800614160002003210090407800AE
:10CE20006140610000414000D0CFB30080C060008D
:10CE300082C070002003210001487800C902A900C7
:10CE40002003210010407800624060000004E000F0
:10CE500003003A003100200021079800020037004B
:10CE60000000EB00200798002E0090000080FA00E0
:10CE7000000006000200FA0000C0EB00004F78003E
:10CE8000C922A800C902A8000040EB001047980082
:10CE900011003700CBC2BF00614060000004E00019
:10CEA00007003A0069FF0700004F78001E04E00009
:10CEB0000C00320040C0B3009E4F10000900320049
:10CEC00050002000107E0200000000001E40900074
:10CED0000040E800104798001E409000E14F4000DD
:10CEE000ECFF3A00C902A9001E80FB000080FA0096
:10CEF000000006000400FA00004F780010C0B300E4
:10CF00007D0007000004E000030032002000200044
:10CF100010079800130037009E40780061C0600041
:10CF20006140600000414000912C20009140780059
:10CF3000D0CFB30000C0600002407000C9E2B7006B
:10CF40000040EB006C0007000004E000030032002A
:10CF50002000200010079800020037008000EB003E
:10CF6000110798001E0090000080FA0000000600E3
:10CF70000800FA00404798000040EB002047980066
:10CF8000C902A900CB02A900C0032000107E020044
:10CF900000000000CB22A900C922A900C902A800F4
:10CFA00010002000107E0200000000000040EB0096
:10CFB000510007000004E0000300320040002000A0
:10CFC00030079800490037000000EB00000F7800A0
:10CFD0001C0037004E4090000080FB0061006000A4
:10CFE0000004E0000B00320010C0B300C1FF0700D6
:10CFF0000004E000030032004000200030079800E9
:10D000003A0037002E4090000004A200204798000C
:10D01000070037000040EB00B6FF07000004E00007
:10D020000300320040002000300798002F00370036
:10D030004E4090000080FB000000D1004047980067
:10D040001E0FE800700020009E0F1000E1FF360068
:10D050002E4090000004A200204798002E4090002F
:10D06000A4FF07000004E00003003200400020009D
:10D07000300798001D003700C922A800CB22A90064
:10D0800010C0B3001C0007000004E00003003200E1
:10D09000400020003007980014003700D2FE07003F
:10D0A000E24F500003003A00400020003007980093
:10D0B0000E003700CCFE07000080FB00000F780058
:10D0C000200020009E0F100003003A0040002000C6
:10D0D0003007980005003700C902A900CB02A9005B
:10D0E0001E0078000080FB00300798003E00900092
:10D0F0000080FA00000006000600FA0020479800B1
:10D100000080EB00000F7800CBC2BF0061406000E0
:10D110008080FB002E4090000080FB00808F50003C
:10D1200003003A000000EB002007980005003700DC
:10D130001E0FE9001E00E000F3FF3A00100020007F
:10D14000200798002E0090000080FA0000000600E2
:10D150000400FA00004F780011479800A0B92000A1
:10D160001E48780030C0B3009E4F100005003A0002
:10D1700000202000E05C880000082000F05C8800AF
:10D180000400370000202000E05C88000020200020
:10D19000F05C88001E4090000080FB0010079800A3
:10D1A0001E009000E10F5000110032001E009000A0
:10D1B000E20F5000180032001E0090000000E00056
:10D1C000010032001E00370041C1B30000BA200048
:10D1D0000148780041C6B30010BA20000148780029
:10D1E00021C3B30020BA2000014878001D00370099
:10D1F00021C0B30000BA200001487800A1C0B300EC
:10D2000010BA20000148780051C0B30020BA2000B5
:10D21000014878001300370011C0B30000BA2000A5
:10D220000148780051C0B30010BA200001487800CE
:10D2300021C0B30020BA200001487800090037005F
:10D240008040EB0000BA2000014878008040EB00ED
:10D2500010BA2000014878008040EB0020BA20007E
:10D26000014878000080FA00000006000200FA0081
:10D270000000EB00000F780010BA2000904078000A
:10D280000030200009010700CBC2BF0061406000F0
:10D290000004E00004003200CBC2BF006240600026
:10D2A0000004E00002003A0010002000000F7800A7
:10D2B00010BA2000904078000020200017010700DD
:10D2C00010BA2000904078000010200013010700E1
:10D2D00010BA20009040780000202000F3000700E2
:10D2E0001E0078000080FA00000006000000FA002E
:10D2F00010BA20009040780000302000070107009D
:10D3000010BA20009040780000102000E7000700CD
:10D3100010BA20009040780000202000E3000700B1
:10D320000000EB000080FA00000006000C00FA008C
:10D33000500798000000EB00000F7800909B200041
:10D34000104078000080FB008000E9001000200001
:10D350000100DD00300798005E0090002007980073
:10D360000000EB00400798002000370000BA2000C2
:10D3700010417800AE0090003E00900000806000F8
:10D3800001202000FC00070010BA20009040780027
:10D3900000102000C500070000082000260107003B
:10D3A0000080FB001007980010BA20009040780021
:10D3B00000102000D90007002E009000000040005F
:10D3C000200798001E00780000004000000F780041
:10D3D0001E0090000000E000010032001E0FE80077
:10D3E0004E0090000000E80040079800909B20004D
:10D3F000104078008080FB004E009000808F50002D
:10D40000DAFF3E001E0078000080FA0000000600EF
:10D410000800FA0030079800909B20001040780028
:10D420000080FB008000E900100020000100DD000A
:10D43000100798003E009000000F78000000EB00FD
:10D44000200798001400370000BA2000104178002F
:10D450001E0090001E00600001202000C600070092
:10D4600010BA200090407800001020008F000700C4
:10D4700010BA20009040780000102000A70007009C
:10D480001E00780000004000000F78002E00900081
:10D490000000E80020079800909B200010407800D2
:10D4A0008080FB002E009000808F5000E6FF3E0041
:10D4B0000080FA00000006000600FA000000EB0001
:10D4C000000F780000202000DB0007000000EB00C8
:10D4D000200798001600370010BA2000904078000E
:10D4E000001020007100070000202000D20007007B
:10D4F0000080FB001007980010BA200090407800D0
:10D5000000102000850007001E0078000000400089
:10D51000000F78001E0090000000E00001003200C3
:10D520001E0FE8002E0090000000E8002007980081
:10D53000909B2000104078008080FB002E0090001F
:10D54000808F5000E4FF3E001E0078000080FA004B
:10D55000000006000200FA00F05C8000B600070040
:10D5600010BA200090407800001020004F00070003
:10D57000F05C8000B0000700004F780010BA200077
:10D580009040780000102000640007001E80FB001F
:10D590000080FA00000006000200FA00004F780048
:10D5A00000BA200010417800E15C80001E80FB0082
:10D5B0007100070010BA2000904078000010200091
:10D5C0003A00070010BA20009040780000102000B8
:10D5D000520007000080FA00000006000400FA0074
:10D5E000204798000040EB00004F7800090037000A
:10D5F00010BA200090407800001020002B00070097
:10D6000010BA20009040780000102000430007006E
:10D610001E4FE8002E4090009E4F1000F4FF39008E
:10D620000080FA00000006000200FA00004F7800B7
:10D6300000BA200010417800E15C80001E80FB00F1
:10D640004D0007000080FA00000006000200FA000A
:10D65000004F780000BA2000104178001E80FB00C7
:10D6600001102000440007000080FA0000000600BE
:10D670000200FA00004F780000BA20001041780044
:10D680001E80FB00010420003B0007000080FA0020
:10D69000000006000000FA00F05C80006600070051
:10D6A0000080FB000080FA00000006000400FA0081
:10D6B000000F780021479800A09C200010407800BF
:10D6C000704060000004E0000B003A00601680002B
:10D6D0001E007000601688001E0078000080EA00BE
:10D6E0008180EA00800078004016800000806000A1
:10D6F0004016880003003700401680001E007000AE
:10D70000401688002E4090000080FB00107E020032
:10D71000000000000080FA00000006000400FA008B
:10D72000000F7800214798001E0078000080EA0072
:10D730008180EA0080007800601680000080600030
:10D74000601688001E0078000080EA008180EA00F0
:10D75000800078004016800000806000401688003D
:10D760002E4090000080FB00107E020000000000B0
:10D770000080FA00000006000600FA00000F7800A2
:10D7800011079800424798001E00E0000F003A0081
:10D790001E0090000080EA008180EA00800078008E
:10D7A0006016800000806000601688001E009000F7
:10D7B0000080EA008180EA00800078004016800046
:10D7C000008060004016880015003700A09C2000F3
:10D7D00010407800704060000004E0000C003A0047
:10D7E000611680001E0090000080700060168800A6
:10D7F0001E0090000080EA008180EA00800078002E
:10D800004016800000806000401688000400370049
:10D81000401680009E0090000100700040168800B5
:10D820004E4090000080FB00107E020000000000CF
:10D830000080FA00000006000400FA00000F7800E3
:10D84000401680001E007000401688000000000096
:10D850000000000000000000501680001E00600064
:10D860000000E000030032001000200010079800C4
:10D87000020037000000EB00100798001E00900027
:10D880000080FA00000006000000FA005C6A020056
:10D89000000000000080FA00000006000200FA000C
:10D8A000000F78001E007800086A020000000000E7
:10D8B000001020000080FA00000006000000FA00BE
:10D8C000366902000000000081002000D092200094
:10D8D0002880020000000000D100200080442000C9
:10D8E000B2800200000000000080FA000000060084
:10D8F0000000FA00766902000000000061002000CC
:10D90000509320002880020000000000C100200089
:10D9100050452000B2800200000000000080FA00A4
:10D92000000006000000FA00AA6A020000000000E1
:10D930000080FB000080FA00000006000000FA00F2
:10D940004A6B0200000000000080FB000080FA002B
:10D95000000006000000FA000040EB00266B020009
:10D96000000000000080FA00000006000000FA003D
:10D9700010C0B300266B0200000000000080FA0017
:10D98000000006000000FA0010C0B300EE6A0200BA
:10D99000000000000080FA00000006000000FA000D
:10D9A0000040EB00146B0200000000000080FA0051
:10D9B000000006000000FA0010C0B300146B020063
:10D9C000000000000080FA00000006000000FA00DD
:10D9D00001012000A0982000288002000000000023
:10D9E000809B2000104078002E58020000000000AC
:10D9F00000C2B300F259020000000000A09C200009
:10DA0000104078000080FB004400DE0061406000B0
:10DA10002E5802000000000000C2B300F2590200BC
:10DA20000000000031002000F0AD2000288002003E
:10DA3000000000000080FA00000006000400FA0068
:10DA40006A1F0200000000009C1B02000000000092
:10DA5000100798006A1F0200000000009C1B0200D3
:10DA600000000000000F78001E0090000000E000A1
:10DA7000090034001E009000E40F500006003C0036
:10DA80001E0090000040E90080407800809B20004C
:10DA900001487800020037000000EB0010079800F2
:10DAA0001E00E00010003400200020009E0F100037
:10DAB0000D003C001E0078000040EA00614160005B
:10DAC000A09C200090407800614061004401DD008E
:10DAD000F0CEB30080C0600082C07000A09C200027
:10DAE00001487800020037000000EB0010079800A2
:10DAF0001E0090000000E00026003A000000EB004D
:10DB000090578800B103200060482000B2800200D6
:10DB1000000000008001EB00420020001100200006
:10DB20001000200096200200000000000040E900E4
:10DB300080407800809B200001487800F10420009C
:10DB4000B0932000B2800200000000008001EB00D2
:10DB5000220020001100200010002000962002006A
:10DB6000000000000040EA0061416000A09C20002D
:10DB700090407800614061004401DD00F0CEB300C8
:10DB800080C0600082C07000A09C20000148780026
:10DB9000010037008DFF0700CB02A900CB22A900AE
:10DBA000C922A800C902A900809B200090407800EB
:10DBB00020C0B300A8680200000000000080FA0046
:10DBC000000006000400FA00000F78001E00780034
:10DBD000100798001E009000E10F50000C0032006A
:10DBE0001E009000E10F5000040039001E0090005C
:10DBF000E20F5000070032000800370081032000C8
:10DC0000A0992000288002000000000007003700D3
:10DC10001000070025000700040037004102200023
:10DC2000C0202000B2800200000000000080FA0046
:10DC3000000006000200FA00000F7800B10020008A
:10DC4000C0092100B2800200000000000080FA003C
:10DC5000000006000000FA00F1032000209D2000D3
:10DC6000B2800200000000000040EB00386B0200B0
:10DC700000000000F00F2000107E020000000000F5
:10DC800010C0B300386B02000000000010C0B300E9
:10DC9000EE6A0200000000000040EB00386B02005A
:10DCA000000000000080FA00000006000A00FA00F0
:10DCB000881F7800D102200010A1200028800200D7
:10DCC000000000000000EB00000F7800100037009B
:10DCD0001E0478005C6A02000000000080407800AA
:10DCE00063004700017478009E00780063004700DD
:10DCF000614078000080FB009058020000000000A6
:10DD000000C2B300F2590200000000001E0FE8003C
:10DD1000300020009E0F1000EDFF3600C08C280060
:10DD2000C255020000000000A1002000E0A3200076
:10DD300028800200000000006300470010407800C7
:10DD40000080FB004400DE000080FB0040079800DC
:10DD50004E009000E90F5000130032004E0090007A
:10DD6000E90F500004003C004E009000E80F500006
:10DD7000080032001B0037004E009000EA0F5000F0
:10DD80000E0032004E009000EF0F500010003200E5
:10DD9000140037006100200080A4200028800200C9
:10DDA000000000001300370061002000E0A4200004
:10DDB00028800200000000000E00370061002000F3
:10DDC00040A5200028800200000000000900370064
:10DDD00031002000A0A520002880020000000000E3
:10DDE0000400370071002000D0A520002880020028
:10DDF00000000000C08C2800C25502000000000096
:10DE0000B100200040A62000288002000000000091
:10DE100063004700104090000080FB004700DE00D8
:10DE20000004E00005003A0061002000F0A6200098
:10DE3000288002000000000004003700F1002000EC
:10DE400050A720002880020000000000C08C28009D
:10DE5000C255020000000000C100200040A82000C0
:10DE6000288002000000000063004700104090007E
:10DE70008080FB0080F72F00008060004380DE0080
:10DE8000204798002E4090000004E00005003A0072
:10DE9000D100200000A9200028800200000000001E
:10DEA0001E0037002E409000EF4F500005003A0052
:10DEB00031002000A0A52000288002000000000002
:10DEC0001600370000042000000F7800E300470030
:10DED0000040EB0080487800080037001E00780002
:10DEE00000004000000F78006300470010407800F9
:10DEF0008040E80063004700014878006300470065
:10DF0000904078002E40900080CF5000F3FF390001
:10DF10001E007800D057020000000000C08C2800CE
:10DF2000C25502000000000091012000D0A920008D
:10DF3000288002000000000063004700904090002D
:10DF400070C0B30000C0600020479800100020009F
:10DF5000000F7800E30047000040EB0080487800A5
:10DF6000080037001E00780000004000000F780015
:10DF700063004700104078008040E80063004700DD
:10DF80000148780063004700904078002E409000E0
:10DF900080CF5000F3FF39001E0078002E58020099
:10DFA00000000000C08C2800C255020000000000E4
:10DFB0004F0478000080FA00000006000200FA001A
:10DFC000000F78001E00780080407800E0022100F9
:10DFD000104078000080FB000000D100614060002C
:10DFE00044010700001020000080FA000000060035
:10DFF0000000FA00E0022100104078000010A100AB
:10E00000E10221008048780041012000B0EC2000AE
:10E01000B2800200000000000080FA00000006004C
:10E020000000FA00E0022100104078000010A0007B
:10E03000E10221008048780021012000F0ED20005D
:10E04000B2800200000000000080FA00000006001C
:10E050000000FA00A09C2000104078000040A000C2
:10E06000A19C200080487800E00221001040780048
:10E070000010A000E102210080487800816A2000A1
:10E080009140780000CEB30000C060007040B30043
:10E09000A8E6B700916C20009140780000CEB30054
:10E0A00000C060007040B300C9E6B700816C20007A
:10E0B0009140780000CEB30000C060000034A000A2
:10E0C000C8E6B700CAC2A900C8C2A900C902A9000F
:10E0D000C8E2A800C922A900D013200010128800AD
:10E0E0000000EB00201288000000EB000012880006
:10E0F00041E2A800D101200040F02000B2800200DF
:10E10000000000000080FA00000006000800FA008D
:10E1100020079800805780008000E800F00F200062
:10E1200000806000805788006A1F02000000000025
:10E130009C1B020000000000100798000000EB008C
:10E14000905788002E009000300798003E00900005
:10E15000E30F50003C0032003E009000E30F5000FF
:10E1600004003E003E0090000000E0000B00320082
:10E170000F0037003E009000E60F500048003200CC
:10E180003E009000E70F50006A0032003E00900011
:10E19000E40F5000370032008B0037008109200067
:10E1A00060F62000B2800200000000008A00370004
:10E1B0005100200030632000B28002000000000007
:10E1C000AC0007002E009000E10F500082003200EA
:10E1D0001E0090000000E000030034001E009000CC
:10E1E000E20F50001300340041022000E0FF200045
:10E1F000B2800200000000008001EB00220020003D
:10E2000011002000200020009620020000000000E5
:10E21000100798001E009000E10F500003003A0024
:10E220000040EB00750007000200370080C0B3001B
:10E23000720007004100200020022100B28002008D
:10E24000000000006400370011C0B3000040EB0084
:10E25000A8000700F0002000E47D0200000000009C
:10E260005100200060022100B28002000000000086
:10E27000590037001E0090008040780000C8B300AD
:10E2800080C070000040EB009A000700A100200051
:10E29000B0022100B2800200000000004E003700F2
:10E2A00011C0B3000040EB0092000700F000200016
:10E2B000E47D020000000000000320002007980019
:10E2C0001E0090000000E00002003A00000520005F
:10E2D000100798000000EB00000F780011003700D5
:10E2E000AE00900090032000808F500002003600A6
:10E2F00000032000200798002E0090008040780046
:10E3000010C0B3007B0007002E009000F2590200FD
:10E31000000000002E0090000000E8002007980098
:10E320001E0FE8001E0090009E0F1000ECFF35004D
:10E330002900370011C0B3000040EB006D0007005A
:10E34000F0002000E47D0200000000001002200028
:10E35000200798001E0090000000E00002003A0034
:10E3600000052000100798000000EB00000F780067
:10E3700011003700AE009000F0072000808F5000A1
:10E380000200360010022000200798002E009000A6
:10E390008040780010C0B300560007002E009000A7
:10E3A000F2590200000000002E0090000000E8007A
:10E3B000200798001E0FE8001E0090009E0F10001E
:10E3C000ECFF35000400370041022000C02020008F
:10E3D000B2800200000000000080FA000000060089
:10E3E0000000FA00B1002000C0092100B280020044
:10E3F000000000000080FA00000006000200FA00A1
:10E40000004F78001E4078000042B0008040780045
:10E410000040EB0037000700F0002000E47D020020
:10E420000000000081C0B3000040EB003100070095
:10E43000F0002000E47D02000000000011C0B300E5
:10E440000040EB002B000700F0002000E47D0200FC
:10E4500000000000E1C0B3000040EB002500070011
:10E46000F0002000E47D0200000000000080FA00BF
:10E47000000006000000FA000040EB006C000700FE
:10E48000F0002000E47D02000000000031C0B30075
:10E490000040EB002600070050002000E47D020051
:10E4A0000000000031C0B3000040EB002000070076
:10E4B000000A2000107E02000000000031C0B300FE
:10E4C0000040EB001A000700000A2000107E020046
:10E4D0000000000021C0B3000040EB001400070062
:10E4E000000A2000107E0200000000000080FA00F8
:10E4F000000006000200FA00004F78001147980063
:10E500001E4090000080FB004400DE008040780048
:10E510001E407800060007001E409000EF4060009B
:10E520001E407800020007000080FA00000006008C
:10E530000200FA00004F7800114798001E4090003A
:10E540004400DD00104798001E4090000004A00029
:10E550001047980010C0B3009E4F100003003A000F
:10E560001E4090000014A000104798001E4090002C
:10E570002F0007001E4090000034A00010479800B4
:10E580001E4090002A0007009E40900070CFB3000C
:10E5900000C06000104798001E4090002400070053
:10E5A0000080FA00000006000200FA00004F780028
:10E5B0001E80FB004012880085C0BF0064406000E0
:10E5C0000004E000FCFF320040128000004F7800A1
:10E5D0008540A9001E80FB000080FA0000000600B4
:10E5E0000000FA0041E2A900A8C6BF00F041B30054
:10E5F000A8E6B700916C20009140780000CEB300EF
:10E6000000C06000C9E6B700816C2000914078002E
:10E6100000CEB30000C06000C8E6B700CEE2A9009B
:10E62000CF02A900CEC2A9000080FA0000000600B7
:10E630000200FA00004F78001E407800DAFF070061
:10E64000CAC2A800CAC2A9000080FA0000000600E1
:10E650000000FA0040168000017C200001007000DC
:10E66000401688001100070020C0B3002D000700ED
:10E67000D4590200000000000004E0000500320050
:10E68000E059020000000000260007000004E0003E
:10E6900004003A00360107000004E00001003A00DF
:10E6A000F3FF37000080FA00000006000000FA00C7
:10E6B000CA82A9000000EB00400388000000EB00C4
:10E6C000500388000000EB00000388000000EB000E
:10E6D000100388000000EB00F0088800D10A200039
:10E6E00091407800F0C8B30000C06000ADE0B70012
:10E6F0000000EB00E008880000642000D0088800DB
:10E7000000002100205E88008040EB0020BC20003B
:10E71000014878000000EB00805D88000080FA006E
:10E72000000006000A00FA00004F7800D05D80006B
:10E7300040079800CE009000E18F50004400320066
:10E740004E019000E10F5100040039004E0090008E
:10E75000E20F50004F003200000137009E80FB00A6
:10E76000310798003E019000E20F51001500320081
:10E770003E009000E20F500007003C00BE009000F9
:10E780000100E0000B0032003E019000E10F51005B
:10E7900010003200230037003E009000F10F5000BF
:10E7A000EE003200BE009000F38F5000EB0032000C
:10E7B0001C003700BDFF0700120020002207980050
:10E7C000E8003700E08B28009655020000000000AA
:10E7D000E2003700CA82A8000000EB00F0088800C1
:10E7E0000000EB00B00888000000EB00A0088800E3
:10E7F00080002000F00888008660A9009660A900CB
:10E80000D10A200091407800F0C8B30000C0600039
:10E810000044A000ADE0B70010002000805D88003B
:10E82000CE00370020BB20001E48780041C0B30056
:10E8300070BB2000014878008040EB0080BB2000C6
:10E840000148780010002000D05D8800C300370028
:10E8500080BB2000104078008040E80080BB200092
:10E860000148780080BB2000104078008080FB00C9
:10E8700020BB2000008040001E48780080BB2000A4
:10E880009040780070BB20001040780080CF50008E
:10E89000B200390020BB2000104078000080FB004F
:10E8A00010079800100820009E009000808F5000F4
:10E8B0003E003200000C20001E019000800F51002D
:10E8C00005003200000820009E009000808F50005C
:10E8D0004E0032009F00370030BB2000104078000F
:10E8E0000080FB004400DE00610060000004E000E6
:10E8F00003003200100380000000A0001003880015
:10E9000030BB2000104078000080FB004300DE0098
:10E91000610060000004E000040032001003800089
:10E9200001022000010070001003880030BB2000AD
:10E93000104078000080FB004200DE0061006000B3
:10E940000004E000040032001003800001042000F5
:10E95000010070001003880030BB200010407800D8
:10E960000080FB000000D100610060000004E000B6
:10E970000400320010038000010820000100700034
:10E980001003880030BB2000104078000080FB009E
:10E99000610060000004E000040032001003800009
:10E9A00001102000010070001003880040BB20000F
:10E9B000104078000080FB00205E8800205E800010
:10E9C0004800DD00205E880030BB20001040780049
:10E9D0008080FB00205E800000807000205E880048
:10E9E000205E80004200DD0064004000205E880060
:10E9F000215E800000002100808F5000550036000D
:10EA000000002100205E88005200370050BB20002B
:10EA1000104078000080FB0001002000E05D8800CD
:10EA2000F15D8800E05D8000F15D8000C808DD00D8
:10EA30000080FD00804078000040EB00E05D880031
:10EA4000F15D880040BB2000104078000081FB0091
:10EA500003002000E05D8000F15D80000000710097
:10EA600081807100E05D8800F15D8800E05D8000DC
:10EA7000F15D8000C808DD000080FD008040780066
:10EA80000040EB00E05D8800F15D880030BB2000B5
:10EA9000104078000081FB0003002000E05D800052
:10EAA000F15D80000000710081807100E05D8800F0
:10EAB000F15D8800E05D8000F15D80004209DD00CD
:10EAC000CE00DE00810071004200DD0064004000E5
:10EAD000E08048009201200003002000A005020011
:10EAE00000000000E05D8800F15D8800E25D8000CC
:10EAF000F35D80000001200001002000800F510024
:10EB0000818F590007003600E05D8000F15D8000D4
:10EB100070005000E0805800E05D8800F15D8800E2
:10EB2000040037001000200001002000E05D880094
:10EB3000F15D8800E05D8000F15D80004008DE004E
:10EB400001002000E0088800E05D8000F15D8000A9
:10EB5000D00888000000EB00D05D88000000EB00CA
:10EB6000200798002E0090000080FA0000000600A8
:10EB70000200FA00805D8000E10F500001003200C9
:10EB80003600370086C0BF00684060000004E00027
:10EB900003003A00100380000000E0002F003A005C
:10EBA0001FE1A8008780A9000000EB00005E88003C
:10EBB0000E00370071408000005E800080804000C1
:10EBC000501680004600DE008048780087C0BF00F5
:10EBD000704060000004E000FCFF32008780A90064
:10EBE000005E80000000E800005E8800015E80009A
:10EBF000205E8000808F5000EEFF39000000EB00A7
:10EC0000100388000000EB00F0088800205E800000
:10EC1000005E88000A00370071408000005E8000BE
:10EC2000008040000000E90010407800F259020026
:10EC300000000000005E80000000E900005E880027
:10EC4000005E80000000E000F3FF3A0097FE07003E
:10EC500010002000000F7800020037000000EB00D9
:10EC6000000F78001E0078000080FA000000060007
:10EC70000000FA00408C28009655020000000000B9
:10EC80000080FA00000006000A00FA0070408000D0
:10EC90003007980010002000A0818800F4FF0700D2
:10ECA00000003700E0590200000000001047980003
:10ECB0001E4090000080FB0040079800CE009000AE
:10ECC000E38F5000200032004E009000E30F500010
:10ECD0000A003C00CE009000E18F50005B00320043
:10ECE0004E009000E10F50005E003C00CE0090000E
:10ECF0000100E000E7003200DB0037004E0090002A
:10ED0000E60F50000E003200CE009000E68F50005B
:10ED100004003C004E009000E50F500095003200CA
:10ED2000D1003700CE009000E78F50006400320021
:10ED30004E009000E80F500054003200CA00370027
:10ED4000CBFF0700D7FF3700BE00900030C0B300F4
:10ED5000804878003E0090008000E80080C0B3004A
:10ED60008048780021E3A800C0C0B300867C020080
:10ED700000000000200798003E0090008080E8001E
:10ED80002E0090004800DE00804878003E00900091
:10ED9000E30040002E00900080487800B0C0B3002F
:10EDA000867C020000000000200798003E009000D2
:10EDB000E40040002E0090004800DE00804878000B
:10EDC0003E009000E50040002E0090008048780052
:10EDD000A0C0B300867C020000000000200798005D
:10EDE0003E009000E60040002E0090004800DE004B
:10EDF000804878003E009000E70040002E00900020
:10EE00008048780090C0B300867C020000000000BB
:10EE1000200798003E009000E80040002E0090007F
:10EE20004800DE00804878003E009000E900400085
:10EE30002E0090008048780021E3A900A100200066
:10EE40003E009000BA00070096FF3700E05902002C
:10EE500000000000104798001E4090008F0007003F
:10EE600090FF3700E05902000000000010479800B2
:10EE7000E059020000000000004F78009E4078003A
:10EE80001E409000BC00070086FF3700E0590200DA
:10EE90000000000010479800E05902000000000048
:10EEA000004F78001E4090000080FB00C800DD008D
:10EEB0001E80FB0000807000A081880079FF370071
:10EEC000E059020000000000104798001E4090002A
:10EED0000080FB00200798001E409000E14F50008A
:10EEE00004003A0030C0B300105A020000000000D5
:10EEF0000300370020C2B300105A020000000000D7
:10EF0000E05902000000000010479800E05902009C
:10EF100000000000004F78009E409000A0CAB3009F
:10EF200080CF500003003A0050C5B3009E4F100040
:10EF3000050032000000EB002007980020C2B3005B
:10EF4000105A020000000000BE00900070C0B30024
:10EF5000804878003E0090008000E8002E0090007D
:10EF600080487800210020003E00900070000700DB
:10EF70004CFF3700E05902000000000010479800E5
:10EF8000E059020000000000004F78008560A900F1
:10EF90001E4090000080FB00C800DD001E80FB00CA
:10EFA00000807000100798009E0090000000220072
:10EFB000808F5000020036000000220010079800E9
:10EFC0001E009000670040004300DE00200798000C
:10EFD000BE00900050C0B300804878003E00900012
:10EFE0000000E8009E409000014878003E0090003C
:10EFF0000080E8001E487800310020003E009000AC
:10F000004B00070070408000004088002E009000F8
:10F0100000004000104088000000EB002040880005
:10F020007140800040832000008040003040880014
:10F030000000EB00404088000000EB0050408800DA
:10F040009560A800A08180003140800004408000CD
:10F05000800178001E019000040078009283020075
:10F06000000000000FFF3700BE0090000040EB00E2
:10F07000804878003E0090008000E8000040EB00EF
:10F0800080487800110020003E0090002800070012
:10F0900004FF37000080FA00000006000200FA00BA
:10F0A000004F7800CAC2A900CB22A900CB02A90058
:10F0B000CB42A90020C0B3009E4F100005003A00CB
:10F0C000CAC2A800CB02A800CB22A800CB42A8004D
:10F0D00004003700CAC2A900CB02A900CB22A900B4
:10F0E000CB42A90010C0B3009E4F100003003200B5
:10F0F00020C0B3009E4F100006003A00C8C2A9000D
:10F10000C922A900C902A900C942A900C8E2A800F1
:10F1100005003700C8C2A800C922A800C902A8007B
:10F12000C942A800C8E2A8000080FA00000006005A
:10F130000600FA0010079800210798000000EB0075
:10F14000000F7800070037009E0078001E00900036
:10F150000080400010407800F259020000000000DA
:10F160001E0FE8002E0090009E0F1000F6FF3900E1
:10F170000080FA00000006000400FA00004F78004A
:10F18000114798001E80FB00100798001E00900099
:10F19000E20F5000170032001E009000E20F5000F6
:10F1A00004003C001E009000E10F500005003200FA
:10F1B000270037001E009000E80F50001A003200B0
:10F1C00023003700C882A9001E4090006140600003
:10F1D000614060004401DD00A12C200091407800D6
:10F1E000F0CEB30000C0600002407000CAE2B70079
:10F1F000170037001E4090000004E00005003200B8
:10F20000C082A900C282A800C8A2A900CAA2A80000
:10F210000F003700C082A900C282A900C8A2A900BD
:10F22000CAA2A9000A0037001E4090006140600099
:10F23000614060004201DD00B12C20009140780067
:10F24000B0CFB30000C0600002407000CBE2B70056
:10F250000080FA00000006000000FA00F00F200015
:10F2600096690200000000000080FA00000006001D
:10F270000400FA00000F78001E0078009669020072
:10F2800000000000000F7800A09C200010407800D3
:10F290000044B2000004E000030032001E007800C9
:10F2A00010079800020037000000EB0010079800DC
:10F2B0001E0090000080FA00000006000000FA0026
:10F2C000A09C2000104078000060A000A19C2000BD
:10F2D00080487800209D2000104078006140600048
:10F2E0000004E000040032000040EB00386B020034
:10F2F000000000000300370010C0B300386B0200AC
:10F3000000000000209D2000104078006140600057
:10F310000004E00003003200F0C2B300F259020022
:10F3200000000000A100200060AB2000B2800200BD
:10F33000000000000080FA00000006000000FA0053
:10F34000A09C2000104078000060A100A19C20003B
:10F3500080487800209D20001040780061406000C7
:10F360000004E000040032000040EB00386B0200B3
:10F37000000000000300370010C0B300386B02002B
:10F3800000000000209D20001040780061406000D7
:10F390000004E00003003200F0C2B300F2590200A2
:10F3A00000000000A100200060AB2000B28002003D
:10F3B000000000000080FA00000006000000FA00D3
:10F3C000A09C2000104078000060A100A19C2000BB
:10F3D00080487800209D2000104078006140600047
:10F3E0000004E0000400320010C0B300386B0200DB
:10F3F00000000000030037000040EB00386B020003
:10F4000000000000209D2000104078006140600056
:10F410000004E00003003200F0C2B300F259020021
:10F4200000000000B100200000AC2000B28002000B
:10F43000000000000080FA00000006000000FA0052
:10F44000AA6A0200000000000080FB000080FA00B1
:10F45000000006000000FA004A6B020000000000F5
:10F460000080FB000080FA00000006000000FA00A7
:10F4700010C0B300EE6A0200000000000080FA0035
:10F48000000006000000FA0010C0B300266B020066
:10F49000000000000080FA00000006000000FA00F2
:10F4A0000040EB00266B0200000000000080FA0024
:10F4B000000006000000FA0010C0B300146B020048
:10F4C000000000000080FA00000006000000FA00C2
:10F4D0000040EB00146B0200000000000080FA0006
:10F4E000000006000000FA0041012000B0AC20003E
:10F4F0002880020000000000809B2000104078005F
:10F500002E5802000000000000C2B300F2590200B1
:10F5100000000000209D2000104078006140600045
:10F520002E5802000000000000C2B300F259020091
:10F5300000000000A09C2000104078000080FB002C
:10F540004400DE00614060002E5802000000000010
:10F5500000C2B300F259020000000000E08C280055
:10F56000C2550200000000000080FA000000060002
:10F570000600FA006A1F0200000000009C1B020047
:10F5800000000000200798006A1F02000000000031
:10F590009C1B020000000000000F78006A1F0200A0
:10F5A000000000009C1B02000000000010079800F3
:10F5B0002E0090000000E000090034002E009000B2
:10F5C000E40F500006003C002E0090000040E900CF
:10F5D00080407800809B20000148780002003700BE
:10F5E0000000EB00200798001E00E0000F00340030
:10F5F000200020009E0F10000C003C001E00780030
:10F600000040E900E1406000209D200010407800AB
:10F6100061C16000E1CFB3000140600002407000B2
:10F62000219D200080487800020037000000EB0098
:10F63000200798001E0090000000E0001000340039
:10F640001E009000E20F50000D003C001E009000D4
:10F650000040EA0061416000A09C200090407800DA
:10F66000614061004401DD00F0CEB30080C0600065
:10F6700082C07000A09C2000014878000200370082
:10F680000000EB00200798002E0090000000E00032
:10F690003A003A00B103200060482000B280020026
:10F6A000000000008001EB0042002000110020005B
:10F6B0001000200096200200000000000040E90039
:10F6C00080407800809B200001487800D101200014
:10F6D00070222100B2800200000000008001EB00D7
:10F6E00022002000110020002000200096200200AF
:10F6F000000000000040E900E1406000209D200083
:10F700001040780061C16000E1CFB30001406000AB
:10F7100002407000219D200080487800F104200004
:10F72000B0932000B2800200000000008001EB00D6
:10F73000220020001100200010002000962002006E
:10F74000000000000040EA0061416000A09C200031
:10F7500090407800614061004401DD00F0CEB300CC
:10F7600080C0600082C07000A09C2000014878002A
:10F770000000EB00905788000100370059FF070098
:10F78000A09C2000104078000060A100A19C2000F7
:10F7900080487800A09C2000104078000050A10014
:10F7A000A19C200080487800809B20009040780039
:10F7B00030C0B300A868020000000000C922A90000
:10F7C000C902A900C8E2A800209D200010407800CE
:10F7D00061406000386B0200000000000080FA0009
:10F7E000000006000000FA0001012000A004210032
:10F7F000B2800200000000000080FA000000060055
:10F800000000FA00A09C2000104078000040A100F9
:10F81000A19C2000804878008040EB00809B200065
:10F8200001487800A09C2000104078000020A10032
:10F83000A19C200080487800A09C20001040780007
:10F840000000A1000010A100A19C200080487800C9
:10F85000A09C2000104078000030A100A19C200056
:10F86000804878000080FA00000006000000FA00DE
:10F87000C922A800C902A800C8E2A800C8C2A800FE
:10F88000C942A800CA82A900C882A900C962A8000A
:10F89000C262A800C062A900A16C2000914078005B
:10F8A00000CEB30000C06000CAE6B7000000EB0065
:10F8B000A0408800D2FF0700C082A900C282A90030
:10F8C000C8A2A900CAA2A9002D83A9002D43A9009E
:10F8D0002D23A9002D63A90001322000914078005A
:10F8E00000CEB30000C0700020E3B7000000EB00C2
:10F8F0008019880020F02100201988000000EB000A
:10F90000101988000080FA00000006000200FA00CA
:10F91000004F78001E80FB00401988002023A800BB
:10F920002003A90020C3BF00614060000004E00084
:10F93000FCFF3200001880000080FA000000060082
:10F940000000FA0021E3A800C0C0B300EFFF0700E9
:10F95000325902000000000021E3A9000080FA00F3
:10F96000000006000200FA00E1002000C03820007C
:10F97000B280020000000000F1002000C01E210043
:10F98000B280020000000000F1002000A039200039
:10F9900028800200000000000000EB003259020045
:10F9A0000000000011002000903A20002880020092
:10F9B000000000000F00370021E3A800C0C0B30022
:10F9C000D2FF0700000F780021E3A900408A280039
:10F9D00096550200000000001E0078003259020017
:10F9E0000000000011002000903A20002880020052
:10F9F00000000000D4590200000000000004E000F4
:10FA0000EDFF3200E059020000000000A08A28004B
:10FA1000C2550200000000000080FA00000006004D
:10FA20000000FA000081200010407800E94F5000EB
:10FA30000800320000812000104078000080FB00A8
:10FA400080004000E081200000804000100078002D
:10FA5000401188000000EB00001188002062A8001F
:10FA60000000EB001011880021E2A8002342A8004A
:10FA70008560A9000080FA00000006000400FA007A
:10FA8000000F7800909B200010407800EF4F50004E
:10FA900007003E00909B2000104078000080FB0093
:10FAA000EF001000F0FF27000180DE001E0F600055
:10FAB00090408000100798001E009000E10F500059
:10FAC000170032001E009000E10F500007003900BF
:10FAD0001E009000E20F50001E0032001E00900039
:10FAE000E30F50002A00320035003700A09C2000B0
:10FAF000104078000042B2000004E0000400320030
:10FB00001E007800E8580200000000002C003700BA
:10FB10001E00780090580200000000002800370006
:10FB2000A09C2000104078000042B2000004E000D9
:10FB3000040032001E007800D057020000000000D0
:10FB40001F0037001E0078002E5802000000000041
:10FB50001B003700A09C2000104078000042B2003B
:10FB60000004E000060032001E007800F655020096
:10FB70000000000000C2B300F259020000000000C3
:10FB80001E007800F6550200000000000C0037004F
:10FB9000A09C2000104078000042B2000004E00069
:10FBA000040032001E0078004800DE00F259020016
:10FBB000000000001E007800F25902000000000062
:10FBC0000080FA00000006000600FA0020079800F6
:10FBD0000000EB00000F78000C0037000000EB0085
:10FBE0001007980005003700A00F20000C00070048
:10FBF0001E0090000000E800100798001E00900012
:10FC0000E30F5000F8FF34001E0FE8002E009000B4
:10FC10009E0F1000F1FF35000080FA000000060082
:10FC20000400FA00100798000000EB00000F7800B5
:10FC3000110037000000000000000000000000007C
:10FC400000000000000000000000000000000000B4
:10FC500000000000000000000000000000000000A4
:10FC60000000000000000000000000000000000094
:10FC7000000000001E0FE8001E0090009E0F100004
:10FC8000ECFF35000080FA00000006000600FA00D4
:10FC9000200798000000EB001007980010002000DB
:10FCA000000F78000D0037001E009000000040009B
:10FCB000100798002E0090001E0060000000E00079
:10FCC000030032001E0090000000A0001007980002
:10FCD0001E00780000004000000F78001E00E000C9
:10FCE000F1FF3A00909B200010407800F04F500048
:10FCF00007003200909B2000104078000080FB003D
:10FD0000F00010001E0090000100DE0010079800B7
:10FD10001E0090000080FA00000006000C080000A1
:10FD20001200000002000000000036001000000079
:10FD300000000000000000000000000000000000C3
:10FD4000B80900001A000000000000003610000092
:10FD50000010000000000000D209000002000000B6
:10FD6000000000001E080000120000000200000059
:10FD7000143404000D8206004003A00001CF0000EF
:10FD80006700440000220000D409000008000000C1
:10FD900000000000DC09000012000000000000006C
:10FDA0003008000042010000020000007282720070
:10FDB0008272820072828400829A82007282720051
:10FDC0008272820072829A00827282009A829A0003
:10FDD00082AE8200C282D80082EE8200FC8248009D
:10FDE000695A000000000000005E6C005E6C780044
:10FDF0006C786C004E6C44006CB66C00AA6CDA0037
:10FE00006CCE6C009E6CC2006C926C009A82E20018
:10FE10006D1E6D00D8821A006EE66C0032574900E4
:10FE20005245000000009E00795E7900DE79DE0018
:10FE3000793879002C7942007A4E7A005A7A660035
:10FE40007A2A7A00367A1E007A9A8200AE82B80048
:10FE50007AD88200F27B72007A335700495245000B
:10FE60000000000072827200827282007282CE00F4
:10FE700064BE6400728272008272820072829A0092
:10FE8000827282009A829A0082046500AC64D80073
:10FE900082EE8200FC824B004559420000000000C7
:10FEA00000F86F00F86F100070107000DE6F9A009D
:10FEB0008272820072827200827282009A82720062
:10FEC000829A82009A82860070287000F072F00098
:10FED00071FC82004C4344000000000000007200EE
:10FEE000827282007282720082A284009A847200FE
:10FEF0008272820072827200829A820072829A00FA
:10FF0000829A8200AE82940084D88200EE82FC0045
:10FF1000824449004F000000000000000000000083
:10FF200000000000000000000000000000000000D1
:10FF300000000000000000000000000000000000C1
:10FF400000000000000000000000000000000000B1
:10FF5000000000000000000000000000EE090000AA
:10FF6000A801000000000000960B00000400000043
:10FF700000000000000800000C000000000000006D
:10FF80009A0B00000A00000000000000A40B000013
:10FF90000200000000000000A60B00000A000000A4
:10FFA00000000000B00B0000160000000000000080
:10FFB000720900004600000002000000E486E8002C
:10FFC00086EB8600F086F50086FA8600008707003B
:10FFD000870B870011871700871B87001E87230068
:10FFE000872887002D873400873A8700408745009F
:10FFF000874A870052875600875A870062876600C3
:020000040001F9
:10000000876D870071877800877E870082878700E9
:10001000878C87009287000000000000C60B00005C
:1000200068040000000000002E1000000200000024
:10003000000000003010000004000000000000007C
:10004000341000000200000000000000000000006A
:100050000600FA0010079800210798001E00900083
:10006000000F7800380037001E00780032002000B2
:10007000110009000200D8008000FD000000E0002F
:100080000B003A001E007800320020001100090029
:100090000200D8000000400080007800408023006B
:1000A000008040001000BA00F25902000000000079
:1000B0001E00780032002000110009000200D80064
:1000C0008000FD00E10F50000C003A001E00780097
:1000D00032002000110009000200D800000040009A
:1000E0008000780040802300008040001000BA00AB
:1000F0004800DE00F2590200000000001E007800F7
:1001000032002000110009000200D8008000FD002C
:10011000E20F50000B003A001E0078003200200071
:10012000110009000200D8000000400080007800A3
:1001300040802300008040001080BA00F259020085
:10014000000000001E0FE8001E009000AE009000AE
:10015000010040009E0F5000C3FF3C000080FA00E9
:10016000000006000400FA00000F78001107980054
:100170009E0090001E007800B5FF0700208D28002B
:10018000C2550200000000000080FA0000000600D6
:100190000000FA000102200030262100F1FF0700D4
:1001A000B104200030282100EEFF0700510220009A
:1001B000E02C2100EBFF070071022000302F21000E
:1001C000E8FF070041012000A0312100E5FF070002
:1001D00011012000E0322100E2FF0700710220003F
:1001E000F0332100DFFF0700A1012000603621006D
:1001F000DCFF0700D102200000382100D9FF0700F2
:1002000041012000D03A2100D6FF07002102200042
:10021000103C2100D3FF0700D1022000303E210016
:10022000D0FF0700B101200000412100CDFF0700F1
:1002300001022000B0422100CAFF0700B1012000E6
:10024000B0442100C7FF07004102200060462100A2
:10025000C4FF070001022000A0482100C1FF0700E1
:1002600081012000A04A2100BEFF0700E10120001B
:10027000204C2100BBFF070081022000004E21001E
:10028000B8FF07004102200080502100B5FF0700A1
:1002900051032000C0522100B2FF0700D10320000B
:1002A00010562100AFFF07000080FA000000060092
:1002B0000400FA00E10020004091200064FF0700E4
:1002C000D4590200000000000004E000FCFF3200EE
:1002D000E059020000000000004F78001E40780046
:1002E000F259020000000000208D2800C2550200D3
:1002F0000000000090C7B3009E4F100003003200C2
:1003000090C5B3009E4F100003003A00100020007B
:1003100010079800020037000000EB00100798005B
:100320001E0090000080FA00000006000600FA009F
:10033000000F780021479800324798004347980003
:10034000544798002E40900061406000614060007A
:1003500000414000F12C200091407800D0CFB30044
:1003600000C0600002407000CFE2B700616A200068
:100370009140780000CEB30000C060007040B30030
:10038000A6E6B700916C20009140780000CEB30043
:1003900000C060005040B300C9E6B7001E007800FE
:1003A000C01188000000EB00801188003062A800B6
:1003B0003E40900061406000614060004401DD000B
:1003C0000123200091407800F0CEB30000C060000F
:1003D0000240700030E2B7004E4090006340600081
:1003E00063406000004140000123200091407800FC
:1003F00090CFB30000C060000240700030E2B70050
:100400005E40900061406000614160000123200077
:1004100091407800E0CFB30000C06000024070005F
:1004200030E2B7000000EB00901188000080FA0075
:10043000000006000000FA0031E2A8003342A800E4
:1004400087C0A9000080FA00000006000000FA0042
:1004500031E2A9003342A900A6C6BF00F041B300B3
:10046000A6E6B700616C20009140780000CEB30092
:1004700000C06000C6E6B700CF22A9000080FA00E5
:10048000000006000200FA00000F780033C2BF002F
:10049000624060000004E000FCFF3A001E007800AB
:1004A000A01188000080FA00000006000000FA0099
:1004B00032C2BF00614060000004E000FCFF320077
:1004C000B01180000080FA00000006000000FA0071
:1004D00032C2BF00614060000080FB000080FA0073
:1004E000000006000000FA00110220000042200077
:1004F000B280020000000000100020009057880029
:100500000080FA00000006000200FA00000F7800E8
:100510001102200000422000B28002000000000012
:100520001000200090578800001020000080FA0082
:10053000000006000000FA00110220000042200026
:10054000B2800200000000001000200090578800D8
:100550000000EB000080FA00000006000200FA0034
:10056000000F78001102200000422000B28002003B
:100570000000000010002000905788000080FA0062
:10058000000006000000FA0081C0B300909B20002C
:1005900001487800A09C2000104078000050A10085
:1005A000A19C2000804878000080FA00000006002E
:1005B0000000FA0081C0B300909B20000148780041
:1005C000A09C2000104078000050A100A19C2000B9
:1005D000804878000080FA00000006000000FA0061
:1005E00001012000A0042100B280020000000000F0
:1005F0000080FA00000006000000FA00008D2800CC
:10060000C2550200000000000080FA000000060051
:100610000200FA00004F78001E80FB004300DE005D
:10062000610060000004E00005003200C082A90003
:10063000C282A800C8A2A900CAA2A800040037006C
:10064000C082A900C282A900C8A2A900CAA2A900AA
:100650001E80FB004200DE00610060000004E0003C
:1006600003003200C962A800CB62A9000200370073
:10067000CB62A900C962A9001E80FB000000D10066
:10068000610060000004E00003003200C942A900DC
:10069000CB42A80002003700C942A900CB42A90002
:1006A0001E80FB00610060000004E00013003200C7
:1006B000A09C200010407800704060000004E00022
:1006C0000500320040168000010420000100700087
:1006D00040168800110037006116800000042000D9
:1006E000008070006016880041168000F0FB2F002B
:1006F0000080600040168800080037006116800006
:10070000F0FB2F000080600060168800411680001A
:10071000F0FB2F0000806000401688000080FA0087
:1007200000000600889FBE008A9FBE008C1F7800D4
:100730008002EB000203E9008003780001047800E6
:1007400003067800A92C20009A0020006B002000EE
:1007500010408000E48242000028E6000500780096
:100760000408E300FEFF350037017800B701780088
:100770000280FD0003026900F40FB2000401690069
:10078000848169000280FD00F00020000030E60056
:1007900006007800800078000C800900000000004E
:1007A0001980A1000281D3001950AD008381D300CC
:1007B0001958AD000C800900000000001980A0004D
:1007C0001970A3000482D3008100E900F2FF310018
:1007D000EF0010000122DE00041C78004300DE0060
:1007E0000000E8000A28B4009580AB000800320041
:1007F000404080000A08E300050032008580A9001F
:100800009580A8000608B400100078002011880028
:1008100070035300CEFF31004F0678004F05BE0035
:100820004F04BE001C5A0400000000000000FA0043
:1008300005000700D6080200000000000000EB00E1
:100840000080FA00000006000000FA004507A90039
:100850000080EB00601988004227A900416A20004F
:100860009140780000CEB30000C060003040B3007B
:10087000A4E6B700216C20009140780000CEB300C0
:1008800000C060003040B300C2E6B70081C0B300D2
:1008900000812000014878000000EB0090408800B3
:1008A000367C020000000000107D02000000000005
:1008B0008000EB00F00F20004C5B02000000000005
:1008C000B040880021002000F00F20004C5B0200A7
:1008D00000000000C04088008040EB00A0812000A4
:1008E00001487800D04080000080A100D0408800FE
:1008F00081C0B300909B200001487800CE370200F1
:10090000000000000000EB0090018800A08C28008F
:10091000C255020000000000142202000000000086
:100920000080FA00000006000000FA000080FA00D3
:10093000000006000000FA00501680000080FA0057
:10094000000006000400FA00000F78001E00780086
:100950004700DE000000A200610060000004E0002B
:10096000060032001E0078004E6202000000000007
:100970000080FB0010079800050037001E0078007B
:100980006E630200000000000080FB00100798006A
:100990001E0090000080FA00000006000000FE002B
:1009A000FFFFFF00FFFFFF00FFFFFF00FFFFFF0053
:1009B000FFFFFF00FFFFFF00FFFFFF00FFFFFF0043
:1009C000FFFFFF00FFFFFF00FFFFFF00FFFFFF0033
:1009D000FFFFFF00FFFFFF00FFFFFF00FFFFFF0023
:00000001FF
